:10200000008000104B210000092100000B2100007E
:102010000D2100000F2100001121000074B9FEEF16
:10202000000000000000000000000000712500001A
:102030001521000000000000D12500001526000039
:102040001B2100001B2100001B2100001B210000A0
:102050001B21000009AA00001B2100001B21000019
:1020600019AA00001B210000158500001B2100009B
:102070001B2100001B2100001B2100001B21000070
:102080001B2100001B2100001B2100001B21000060
:102090001B2100001B2100001B2100001B21000050
:1020A0001B2100001B2100001B2100001B21000040
:1020B0000D2C0000398A00001B2100001B210000AC
:1020C0001B2100001B2100001B2100002426010011
:1020D00040000010B80000002426010000C00720C6
:1020E0000000000024260100000000100000000095
:1020F000F8000010A062000000C0072000000000EF
:102100000000001000000000FEE7FEE7FEE7FEE72B
:10211000FEE7FEE7FEE7FEE7FEE7FEE70023934269
:1021200009D210B404680C600433043004319342C3
:10213000F8D310BC70477047002303E00022026010
:10214000043304308B42F9D3704710B50E4B07E0CF
:1021500003F10C049A6859681868FFF7DFFF2346FB
:102160000A4A9342F4D306E01C46596854F8080B17
:10217000FFF7E2FF2346064A9342F5D308F0CAFB75
:102180000BF0FDFAFEE700BFCC200000F0200000BD
:1021900008210000FFFFFFFFFFFFFFFFFFFFFFFF22
:1021A000FFFFFFFFFFFFFFFFFFFFFFFFFFFFFFFF3F
:1021B000FFFFFFFFFFFFFFFFFFFFFFFFFFFFFFFF2F
:1021C000FFFFFFFFFFFFFFFFFFFFFFFFFFFFFFFF1F
:1021D000FFFFFFFFFFFFFFFFFFFFFFFFFFFFFFFF0F
:1021E000FFFFFFFFFFFFFFFFFFFFFFFFFFFFFFFFFF
:1021F000FFFFFFFFFFFFFFFFFFFFFFFFFFFFFFFFEF
:10220000FFFFFFFFFFFFFFFFFFFFFFFFFFFFFFFFDE
:10221000FFFFFFFFFFFFFFFFFFFFFFFFFFFFFFFFCE
:10222000FFFFFFFFFFFFFFFFFFFFFFFFFFFFFFFFBE
:10223000FFFFFFFFFFFFFFFFFFFFFFFFFFFFFFFFAE
:10224000FFFFFFFFFFFFFFFFFFFFFFFFFFFFFFFF9E
:10225000FFFFFFFFFFFFFFFFFFFFFFFFFFFFFFFF8E
:10226000FFFFFFFFFFFFFFFFFFFFFFFFFFFFFFFF7E
:10227000FFFFFFFFFFFFFFFFFFFFFFFFFFFFFFFF6E
:10228000FFFFFFFFFFFFFFFFFFFFFFFFFFFFFFFF5E
:10229000FFFFFFFFFFFFFFFFFFFFFFFFFFFFFFFF4E
:1022A000FFFFFFFFFFFFFFFFFFFFFFFFFFFFFFFF3E
:1022B000FFFFFFFFFFFFFFFFFFFFFFFFFFFFFFFF2E
:1022C000FFFFFFFFFFFFFFFFFFFFFFFFFFFFFFFF1E
:1022D000FFFFFFFFFFFFFFFFFFFFFFFFFFFFFFFF0E
:1022E000FFFFFFFFFFFFFFFFFFFFFFFFFFFFFFFFFE
:1022F000FFFFFFFFFFFFFFFFFFFFFFFFFFFFFFFFEE
:1023000010B4134A00E01A4613688342FBD35168A5
:102310005418844209D041684418A3420AD003608B
:10232000904200D0106010BC70474068014451607A
:102330001046F0E7074C2468A34206D05B681944B6
:10234000416013681B680360EAE70460E8E700BFC8
:1023500008010010F800001070B5054604F08AFD71
:102360002B4B1B681D420FD135B1083515F0070FF7
:1023700002D025F0070508356DB1264B1B68AB422E
:102380000DD3254A146810E004F002FE002605F083
:1023900017FD304670BD04F0FBFD0026F7E704F0A2
:1023A000F7FD0026F3E722461C466368AB4202D2E3
:1023B0002368002BF7D1194B1B68A3421DD0166868
:1023C00008362368136063685B1B102B19D862689A
:1023D00010490B689B1A0B60114909688B4201D2A6
:1023E0000F490B600A4B1B68134363600023236093
:1023F00004F0CEFD002ECCD1C9E704F0C9FD0026C3
:10240000C5E7601943606560FFF77AFFDFE700BF4B
:10241000FC0000100001001008010010F80000107E
:1024200004010010F8B138B50446A0F1080550F8D1
:10243000042C0D4909680A4202D050F8080C00B17A
:1024400038BD22EA010244F8042C04F013FD54F8CC
:10245000041C064A13680B4413602846FFF750FF1C
:1024600004F096FDECE77047FC000010000100103E
:10247000014B1868704700BF00010010F0B402461D
:1024800000210E4614E0194C25681344083B23F044
:102490000703236000245C601C6014469F1A576089
:1024A000136005B12A6063681E44013100EBC1026C
:1024B000536883B1126812F0070F05D0D41D24F0C1
:1024C0000704121B134422460029DCD1084C226069
:1024D00000256560D7E7074B1E60074B1E60074B62
:1024E0004FF000421A60F0BC704700BFF8000010C7
:1024F000080100100401001000010010FC00001091
:1025000082B0002301934FF0280383F31188BFF3B7
:102510006F8FBFF34F8F019B002BFCD002B0704731
:1025200006480068006880F3088862B661B6BFF3A9
:102530004F8FBFF36F8F00DF00BF000008ED00E09A
:102540004FF0807340F8043C21F0010140F8081C72
:10255000034B40F80C3C40F8202C4038704700BF3B
:1025600001250000FFFFFFFFFFFFFFFFFFFFFFFF51
:10257000074B19680868B0E8F00F80F30988BFF3CB
:102580006F8F4FF0000080F311884EF00D0E7047F2
:102590006C0400104FF0280383F31188BFF36F8F92
:1025A000BFF34F8F024A136801331360704700BFB7
:1025B00040000010034A1368013B13600BB983F31A
:1025C0001188704740000010FFFFFFFFFFFFFFFF73
:1025D000EFF30980BFF36F8F0D4B1A6820E9F00FFE
:1025E00010602DE908404FF0280080F3118804F0B6
:1025F0005BFD4FF0000080F31188BDE808401968CA
:102600000868B0E8F00F80F30988BFF36F8F704758
:102610006C04001008B54FF0280383F31188BFF352
:102620006F8FBFF34F8F04F033FC18B1034B4FF0A3
:1026300080521A60002383F3118808BD04ED00E086
:10264000084A0023136008490B60084B1B680849BF
:10265000A1FB03135B09013B06490B6007231360D1
:10266000704700BF10E000E018E000E09463001045
:102670001F85EB5114E000E010B50B4B1A6842F4D3
:1026800078021A601A6842F078421A60FFF7D8FFA1
:102690000024064B1C60FFF743FF04F005FDFFF725
:1026A0002FFF204610BD00BF20ED00E040000010CD
:1026B00082B00E4B1A6892090D4BA3FB0232920AAC
:1026C0004FF47A7303FB00F0009006E000BF019B1B
:1026D00001330193019B9A42F8D8009B013B009380
:1026E00013B100230193F5E702B070479463001023
:1026F0001791650210B504464FF0A040D0F82C2188
:10270000032392B20749098809F011FB022807D078
:10271000044B1A88044B1B6843F83240012010BD5B
:102720000020FCE74201001020010010F8B5394BF1
:102730001B7803B1F8BD1820FFF70EFE364F386046
:102740000C20FFF709FE354E30602020FFF704FE15
:10275000334D28602020FFF7FFFD324C2060182207
:10276000002138680BF016F80C22002130680BF0BD
:1027700011F82022002128680BF00CF820220021FB
:1027800020680BF007F80024274B1C80274B1C8087
:1027900015E019214FF4107000F00AFB8069E30086
:1027A0001F4A1268D11842F83400214A4A601D4A73
:1027B00011680B44002241F834205A600134032C84
:1027C000E7DD00230DE0144A126802EBC30119484B
:1027D00042F8330000224A601049096841F823207A
:1027E0000133022BEFDD03230C4A12680A49096802
:1027F0004FF0A04009F061FA04230A4A1268084920
:1028000009684FF0A04009F075FA024B01221A70D6
:1028100090E700BF380100102001001024010010D3
:10282000180100101C0100104001001042010010AE
:102830003F020080EFBEADDE08B508F0A9FE10F043
:10284000080F14D00F4B1B68834210D00D4B18603B
:1028500010F0100F0CD04FF0A0434FF480729A612B
:1028600010F0200F09D14FF0A04009F00CFA08BD7C
:102870004FF0A04300229A61F2E74FF0A04009F028
:10288000E8F9F4E73C010010F0B583B04FF0A04345
:10289000D3F8E42F4FF0FF32C3F8E42F624B282225
:1028A00083F81C234FF080521A60AAE05F4A137825
:1028B00003F0FE0313705D4B1B7813F0020F78D109
:1028C0005A4B1B78002B00F09680584B1B7813F066
:1028D000010FF0D001238DF800300023019321E097
:1028E00019214FF4107000F063FA0746002843D016
:1028F000304600F012FD0646C461B9694C4B1A8897
:102900004C4B1B6843F8321001900021684600F0E0
:1029100091FF002837D04FF0A04009F050FA444B07
:1029200018802B465A1CD5B2022BC4D84FF0A040B9
:10293000D0F8141104233E4A128889B209F0F7F93D
:102940000028B3D03A4B1B883A4A126852F83360D9
:10295000394A126852F83320C2F30A03DC1E04D04D
:10296000002ABDDA12F0806FBAD14FF0A04009F012
:1029700026FA2F4B1880D4E74FF0A04009F01FFA39
:102980002B4B1880CDE7304600F0F0F9C3E7002369
:102990001A4619462948006803F046FE284A13687B
:1029A00001331360274A13780133DBB21370022B13
:1029B00017D8244B1A7891B24FF0A043D3F82C319A
:1029C0009BB2994211D0204B53F822000028DED050
:1029D00000F0CCF91B4B1A781B4B002143F8221056
:1029E000D5E7134600221A70E3E7104A137803F084
:1029F000FD03137064E704F045FA144B1B6883422F
:102A00000CD3FFF735FD124B18604FF0A043D3F8FD
:102A10002C313221012004F09BFD51E732300B4B69
:102A20001860FFF709FFECE700E100E03901001052
:102A300040010010180100101C0100104C01001092
:102A4000100100103A010010500100104401001064
:102A50001401001010B582B001214FF0A04009F020
:102A600022F82E494FF0A04009F086F801220146D5
:102A70004FF0A04009F05EF8294B59791A7942EAE3
:102A800001224FF0A0442264D9789A7842EA0122C8
:102A900062645A781B7843EA0223A36400231A462F
:102AA0002049012008F004FDFFF740FED4F8003172
:102AB00043F00203C4F80031D4F8003143F00103BD
:102AC000C4F80031236843F001032360D4F80031D7
:102AD00023F08003C4F80031D4F8003243F022031D
:102AE000C4F80032104B01930623009300234FF4E7
:102AF00096720E490E4804F053F904460D4B1B68BC
:102B000023B1FFF799FE204602B010BD022108460E
:102B100003F07FFD074B1860F3E700BFA0252600F8
:102B20008C000010B126000048010010D8100100F0
:102B3000892800004C01001070B584B004460E4690
:102B40000A230393C369002B48D02B4B1868002835
:102B50004BD00A2103F0B2FE012802D000231D460B
:102B60003EE001A804F092FBA069FFF7C3FD38B96D
:102B700003A901A804F0A8FB0028F5D0012300E078
:102B800000230BBB3EB14FF0A043D3F828319BB2DA
:102B90001A4A42F82340E369013BC3F30A03184D84
:102BA0002988184A126802EBC10243F0404353607F
:102BB0004FF0A04009F0E5F82880134A136801336C
:102BC000136001231D460BE000231A4619460A48EC
:102BD000006803F029FD00231D4601E000231D4687
:102BE00003B92EB9284604B070BD00231D46F7E78F
:102BF000204600F0BBF8F5E74C0100105001001032
:102C000042010010200100102C01001010B582B00C
:102C10000023019320E02B4A1368013313602A4AF2
:102C2000137843F00103137001A9284B186804F0CE
:102C3000CBFC1DE0264A136801331360224A137847
:102C400043F00203137001A9204B186804F0BCFC88
:102C500011E014F0100F1BD14FF0A043D3F8E04F58
:102C600024B34FF0A043C3F8E84F14F0080FD2D1BB
:102C700014F0800FDED114F0010FEAD04FF0A04223
:102C8000136843F480631360124B00221A80E0E75C
:102C9000114A1368013313604FF0A042136843F4E4
:102CA000807313600D4B00221A80D5E7019B3BB166
:102CB0000B4B4FF080521A60BFF34F8FBFF36F8FF3
:102CC00002B010BD280100103901001048010010A9
:102CD00030010010400100103401001042010010CA
:102CE00004ED00E038B5184B1B6823B1164B1B6888
:102CF00043B3012038BD0C21084603F08AFC124C76
:102D00002060124903F088FE2368002BEED01048A3
:102D100003F02BFB00250FE0EB002B449A000D4C39
:102D200014440023A361204603F02AFBE4602146FB
:102D3000074803F034FB01350B2DEDDD064B0C226B
:102D40001A60D3E70020D5E724030010E410010047
:102D500060010010740100105C01001020B108B582
:102D60000A38FFF75FFB08BD7047FFFF38B5044620
:102D70008069FFF7F3FF0023A361FFF70BFC2569D0
:102D8000094B9D4203D02146184603F0FCFAFFF799
:102D900011FC054B9D4206D000231A4619460348F4
:102DA000006803F041FC38BD6001001024030010EE
:102DB00070B5431E402B00D84220841C14F0030F32
:102DC00002D044F003040134164B186803F076FD7A
:102DD000012824D1FFF7DEFB134EF368DD68284697
:102DE00003F0F7FAFFF7E6FB3368104A12689A42DD
:102DF00001D90E4A13600CB9284670BD04F10A00CF
:102E0000FFF7AAFAA86128B10560AB690A33AB6184
:102E1000EC61F1E72846FFF7A9FF0025ECE7002564
:102E2000EAE700BF24030010600100105C010010FD
:102E30000023052B21DC10B503EB4304A200104C4A
:102E4000A258824204D00133052BF5DD002010BDCD
:102E500003EB4302900022460244D27A5AB108465C
:102E600003EB43039A0021461144062204310AF081
:102E70008DFC0120EBE70220E9E70020704700BF4E
:102E8000280300102DE9F04705460E46474B5B69C5
:102E9000474A52685940114246D0002B40F0848086
:102EA0004FF0FF094FF0000A4FF0FF37B846544685
:102EB0000EE0002D41D004EB440293003D4818443D
:102EC0000622294604300BF0E5F908B3A046013488
:102ED000052C33DC04EB44029300364AD358B3424A
:102EE000E7D055B104EB440293003248184406225F
:102EF000294604300BF0CEF9A0B104EB44039A004C
:102F00002C4B13449B7A4B45E1D29946A246DEE70F
:102F1000284A630018198100114496208872012301
:102F2000CB7241E02746D2E74FF0FF094FF0000A8D
:102F30004FF0FF37B8465446CAE7A046002F1FDBC4
:102F4000B8F1000F12DA07EB47029300194AD65086
:102F5000EDB9B8F1000F27DA164A7B00D8198100C5
:102F60001144052088720023CB721DE008EB480253
:102F700093000C2200210F4818440AF00BFCE2E7F2
:102F8000B8F1000F01DB4746DDE75746DBE77C0081
:102F9000E3199E00164406222946301D0AF0F6FB6E
:102FA0009623B3720123F372BDE8F087440000104A
:102FB000AC0300102803001070B582B0044600F185
:102FC0001C05042229460DEB02000AF0DFFBD4F8B1
:102FD00026602A4B5B69002B4DD0A28AB2F5807F18
:102FE00004D0B2F5007F3FD0002045E0B34201D0CD
:102FF000002041E0019904F11600FFF743FF002390
:10300000237502236375019BB34218D0062204F195
:10301000160104F120000AF0B9FB019BC4F8263028
:10302000164E0622314604F116000AF0AFFB0422C8
:1030300006F1140128460AF0A9FB02201CE0062232
:103040000F49A0180AF0A2FB0622002104F120007B
:103050000AF0A0FB002384F8263084F8273084F897
:10306000283084F82930DBE7019904F11600FFF7D6
:1030700009FF002000E0002002B070BD44000010F5
:103080002811010038B5054608462C68B4F1FF3F09
:1030900018D0124B1B699C4214D0114B5B69C3B111
:1030A0000E4A52686340134203D00C4B9B6803B135
:1030B0001C4684B101462046FFF7BAFE034630B9EC
:1030C0002C6004E0062207490AF060FB0123184641
:1030D00038BD0223FBE70223F9E700BFAC03001071
:1030E000440000102811010070B5054684692622AD
:1030F0000E4920460AF04AFB0D4E06223146A01822
:103100000AF044FB0622314604F116000AF03EFBA9
:10311000042206F1140104F11C000AF037FB6B696C
:10312000C4F826302A23EB6170BD00BFF010010007
:103130004400001038B5054600212A20FFF738FE6C
:1031400038B104464561FFF7CFFF01212046FFF764
:10315000F3FC38BD10B5002411E0204A1058FFF7E9
:10316000E9FF04EB44039A001C4B13449B7A2BB9F0
:1031700004EB44029300194A0021D1500134052C7C
:103180001ADC04EB44039A00144B13449B7A002B83
:10319000F4D0013BDBB21046104A02449372D27A5B
:1031A000002ADAD0032BDCD804EB440293000B4A4C
:1031B000D058FFF7BFFFD4E703F064FE0446084B86
:1031C0001B681BB1C31AB3F5FA6F05D9054B5869D3
:1031D000FFF7B0FF024B1C6010BD00BF28030010BA
:1031E00070030010440000100C4B1B7813F0010F0B
:1031F00007D00A4BDB68B3F57A7F09D2074B1B690E
:1032000001E04FF47A73064AD068984203D27047BF
:103210004FF47A73F7E71846F9E700BF7803001018
:10322000D4030010002380F82230D0F81A30C0F800
:103230001E30084B5B69C0F81A30838C4FF6F6726B
:10324000934203D8083383840220704703F58473C4
:103250008384F9E74400001008B590F82230082B69
:1032600002D1FFF7DFFF00E0002008BD38B50446BB
:103270000D46043004F00AF8E56045B123786FF399
:1032800041032370237843F00103237038BD237872
:1032900043F002032370F5E708B50161FFF7E6FF8D
:1032A00008BD037813F0010F10D010B5044613F0D9
:1032B000020F05D100F10C01043004F005F838B11B
:1032C00021692046FFF7D2FF012010BD0020704782
:1032D0000020FAE708B504F029F8044B1B68834284
:1032E00001D0002008BD0120FCE700BFA4030010AE
:1032F00038B5054608460021FFF75AFD044650B18F
:103300006B6943612B8C03846B8C4384EA69A969E4
:1033100080690AF03BFA204638BD38B1A0F10A02B4
:1033200012F0030F04D150F80A0C704700207047C8
:1033300000207047F0B583B005460F4616461C4680
:1033400000220821112003F04AF92F4B18600028B1
:1033500057D02E4903F060FBFFF7C4FC012806D0CC
:10336000294C206803F082FB002020604AE0EA78C4
:10337000AB781B0443EA02636A7843EA02232A78A3
:103380001343234D2B60F978BA78120442EA0162A4
:10339000797842EA012239780A436A60F078B17894
:1033A000090441EA0061707841EA00213078014364
:1033B000A960E078A178090441EA0061607841EAF7
:1033C000002120780143E96063EA02032B611422A3
:1033D000294610480AF0DAF92B680F4843610622A3
:1033E00008990AF0D3F900F08FFC0C4B01930523E8
:1033F000009300234FF4617209490A4803F0D0FC9E
:1034000000E0002003B0F0BDC4030010181101005B
:10341000AC0300109003001044000010A40300103F
:10342000201101009D39000010B504460622014616
:103430000C480AF02FFF48B9A289130A43EA022375
:103440009BB2B3F5C06F0AD8002010BD06222146FA
:1034500005480AF01FFF0028EED00020F5E7012004
:10346000F3E700BF440000102811010008B5064B27
:1034700001221A60002004F0A5FC4FF47A71034881
:10348000FFF70AFF08BD00BFC80300107803001053
:10349000F0B40502ADB245EA1025ADB22B460026C8
:1034A0000C4601F0030011F0010705D022B114F819
:1034B000011B61F30F26013A411E012906D922F0B2
:1034C000030CACF10C0CA444002508E0012AF6D949
:1034D00034F8020B2B18023AF1E701F110042146EF
:1034E000A44510D92068181800D301354B68C018BE
:1034F00000D301358C68001900D30135CB68C3189F
:10350000EBD30135E9E798B200EB1340431902F021
:103510000E00014402E034F8020B0344A142FAD841
:1035200012F0010F02D0227862F30706981983B2D5
:1035300003EB10439AB202EB13432FB11A0292B27B
:10354000C3F3072042EA0003180220F07F4222F072
:10355000FF02C3F30720104380B2F0BC7047F8B5F8
:10356000837B03F00F039B00A3F114060644C47D84
:10357000112C08D0062C2CD0621ED2B2012A48D8B9
:1035800006F1240501E006F1280529B300222A806E
:10359000B0F810C04FEA1C2242EA0C2292B2D21AB2
:1035A000072A39D9C3F51073934238D30F46022C3A
:1035B0001AD806F122010020FFF76AFFC04383B248
:1035C000EFB91BB3180A40EA032080B237B3288052
:1035D00024E006F13205D8E72A88002AD8D1112C38
:1035E000D6D14FF6FF7019E093B22344083200F1B0
:1035F0001A0198B2FFF74CFFC04383B2E0E7002BFB
:10360000E0D1112CDED14FF6FF73DBE74FF6FF73ED
:10361000D8E744F2213001E041F23420F8BD41F214
:103620003420FBE738B5D0F81E40838A23F0F0033E
:103630009BB25BBB837B453BDBB20A2B28D8164B86
:103640005B69A34207D0B4F1FF3F04D0134D2D694D
:10365000A54200D0F3B90C46C37D012B0AD000F17E
:103660000E010020FFF714FF4FF6FF73984201D0C0
:1036700000200CE00021A069FFF771FF4FF6FF73F7
:10368000984201D0002002E0012000E0002038BD77
:103690000020FCE70020FAE744000010AC03001013
:1036A0002DE9F0470546884600F10E09847BA40009
:1036B00004F03C04C77D2246FFF7B4FF064601280C
:1036C00002D03046BDE8F087142C13D8112F25D135
:1036D000062F42D0112F27D0012FF2D1D8F8180091
:1036E000D5F81E20234B5B699A42EAD1FFF7B4FD5F
:1036F0000646E6E7A4F1140AD8F81C20A2EB0A0259
:10370000223A09EB040105F122000AF041F8D8F849
:103710001C30A3EB0A03C8F81C30D7E7D5F81A1001
:10372000A81DFFF7AFFBD3E7D8F81820D18C0B0A00
:1037300043EA01239BB2083BC8F81C30538CA8F81D
:103740002030D2F81A30C8F81430918C404602F07C
:1037500015FD0128B5D10326B3E7404602F008FB6A
:10376000012804D0044A136801331360A9E7032633
:10377000F8E700BF44000010CC03001070B5044609
:103780000D4681B174B1A069861D0622314609F04B
:10379000FDFF06220749304609F0F8FF294620467A
:1037A000FFF7CAF970BDC169FFF7A2FD0446012504
:1037B000E8E700BF4400001010B582B004468069FD
:1037C000FFF732FE8DF80700A0699DF80730DBB2E5
:1037D000012B0AD09DF80730DBB2022B1AD0032B45
:1037E0001CD02046FFF7C2FA18E08389082B07D0C7
:1037F000B3F5C16F0AD1FFF7DFFB8DF80700E9E7EA
:103800002146FFF74DFF8DF80700E3E700238DF811
:103810000730DFE701212046FFF7B0FF02B010BDFF
:1038200008B5FFF7C9FF08BD014B1868704700BF16
:10383000A803001038B504460D46FFF7F5FF10B990
:1038400094F9003003BB94F90030052B0BD0FFF73F
:1038500041FD012814D000232A4621460B48006868
:1038600002F0E2FE38BD0A4A137843F002031370F7
:10387000064B186803F0C6F80028E8D00120F1E7ED
:10388000002DE8D00025E6E70020EBE7C403001098
:10389000D403001008B500210648FFF7CBFF01282C
:1038A00003D0054B01221A6008BD034B00221A60A9
:1038B000FAE700BF30110100C003001008B50F4B3C
:1038C0001A786FF300021A700D4B1B68012B0DD094
:1038D0000B4B01221A60FFF7BDF801280AD04FF404
:1038E000967003F0C7FBFFF7D5FF08BD012004F079
:1038F00069FAEDE7FFF7BAFDF7E700BF78030010BC
:103900008C03001000B583B08DF8000000210191F8
:103910006846FFF78FFF03B05DF804FB10B5194848
:10392000FFF7BFFC38BB184B186803F06BF830BBCF
:10393000012403F0A7FA154B1B683BB1C31A03EB34
:1039400083035902124A13680B4413600F4B18602B
:103950001048FFF7A6FC104B1B6803B104B948B12F
:10396000204600F0E9FD01460A48FFF77FFC0A4BBC
:1039700000221A6010BD0220FFF7C4FFD3E7002425
:10398000D7E700BF78030010C4030010D003001075
:1039900018040010D4030010CC03001010B584B03C
:1039A000FFF778FF64213E48FFF776FC3D4B01228C
:1039B0001A6008E03C4B00221A60FFF77FFF3B4B88
:1039C0001B68002B68D1FFF7A9FFFFF70DFC04A9C6
:1039D000FF2301F8083D0246354B186802F0E8FE67
:1039E0009DF908300A2BEAD801A252F823F000BF53
:1039F000B53900001D3A0000253A0000613A000088
:103A0000BF390000713A00007D3A0000BF39000064
:103A10002B3A0000593A0000693A00000398FFF77A
:103A2000FFFECCE7FFF796FBC9E7039C0023019359
:103A3000A18C0A0A42EA0122ADF80220A3840822DE
:103A40006946204600F05AFA236843F010032360C9
:103A5000204600F02EFBB2E7039800F0A3FAAEE791
:103A6000039802F01FFBAAE7039800F09DFFA6E76A
:103A70000B4A137843F002031370A0E7039C20461F
:103A800002F010FA00289AD0236843F00403236060
:103A9000204600F00EFB92E7FFF7FCFE93E700BF25
:103AA000D4030010A8030010C8030010C0030010C6
:103AB000C4030010431E13F1030F0BD80AB183692E
:103AC00053B190F82730C9B28B4201D00020704723
:103AD000012070470020704700207047808C0C4BFD
:103AE000DB6800E05B680B4A93420FD0DA6892F81B
:103AF00053100129F6D1918C8142F3D1B2F84E10C6
:103B00000029EFD00139A2F84E107047704700BF6E
:103B1000EC030010F403001070B50E4614461D4669
:103B2000FFF782FEB0B1112C03D0062C09D0002083
:103B300011E0022E03D000204C232B600BE001206B
:103B4000FAE7012E04D000204FF49C732B6002E0B2
:103B50000120F9E7002070BD38B505460C46FFF797
:103B600063FE60B16DB105F10802E868904204D0CF
:103B70000368A34202D04068F8E7002038BD002067
:103B8000FCE70020FAE7FFFF70B5062802D0124ECE
:103B900000250EE0114E01250BE0114B33F81530D6
:103BA0001C0A44EA0324A4B221463046FFF7D4FF9E
:103BB00078B10B4A32F8153001339BB222F8153038
:103BC000B3F57F4FE9D313464FF4414223F8152054
:103BD000E3E7204670BD00BF00040010EC030010B6
:103BE000E803001010B584B004460A238DF80830AD
:103BF00003901021006802F067FB4FF0FF3102A82C
:103C0000FFF718FE58B14FF0FF3300930023012255
:103C10001021206802F0FEFAA06804B010BD002058
:103C2000FBE7FFFFF8B505460F46C9B1446EC36D0B
:103C30006BB9A3F13333A3FB04239B08C365B0F82E
:103C40004A20934203D2B4EB420F00D3C2652B6EDD
:103C50003BB9A300124AA2FB03239B082B6600E09A
:103C6000846E043424F0030404F11400FEF774FBA2
:103C7000064640B11422002109F08CFD34616FB971
:103C80002E673046F8BD95F8423043F0080385F8BA
:103C900042300821284601F0AFFBF2E7EE66F0E77C
:103CA000CDCCCCCC38B504460D4601220621FFF719
:103CB00001FFC8B194F8423013F0080F17D194F8FF
:103CC0005330BBB194F8413013F0400F15D1B5B16A
:103CD000236F0BB1012011E000212046FFF7A2FF66
:103CE000236F73B1012009E06FF0150006E06FF05B
:103CF0000B0003E06FF07F0000E0002038BD0020E3
:103D0000FCE76FF00B00F9E708B5074802F02DFB60
:103D1000064B4CF201021A800549012008605A80C6
:103D2000044802F022FB08BD00040010E803001064
:103D300018040010EC03001070B582B0154601ABFA
:103D4000FFF7EAFE20B94FF0FF34204602B070BD05
:103D50000198FEF701FB0446B0B302F04EFA0646A6
:103D600038B3019A0021204609F014FD6660112D38
:103D700025D004F1080002F003FB64614FF0FF332B
:103D8000E3612362022384F8263084F82750062D4D
:103D9000DBD140F20A23A4F84A30A4F84C3040F2B8
:103DA00014436366A3660123C4F8CC30C4F8D03052
:103DB000CBE72046FEF736FB4FF0FF34C5E704F1B2
:103DC000380002F0D2FAD4E74FF0FF34BDE710B567
:103DD0000C20FEF7C1FA044638B10C22002109F08C
:103DE000D9FC02F00AFA206008B1204610BD204636
:103DF000FEF718FB0024F8E708B502F00F02C36ACB
:103E00001A43C26212F00F0F00D108BD8162002375
:103E10004B600846FFF7E6FEF7E702F00F02C36AC1
:103E200023EA0202C26212F00F0F02D10023836262
:103E3000704781627047836A8B4201D000207047CF
:103E4000006B00F00F00704730B587B00446039157
:103E500004A803F01BFA039B009300231A460F21CA
:103E6000206802F0D7F9012363602046FFF7BAFE0D
:103E70000021206802F028FA054628B903A904A801
:103E800003F022FA0028E6D0284607B030BD431ED2
:103E900013F1030F26D883693BBB10B584B0082308
:103EA0008DF808300390D1B14A8822FA03F343EA2F
:103EB0000223838404464FF0FF3102A8FFF7BAFCC7
:103EC000B0B14FF0FF33009300230122102160684E
:103ED00002F0A0F9A36973B1002004B010BD002363
:103EE0008384E7E76FF0150070476FF015007047A7
:103EF0006FF08B00F1E76FF01500EEE7F0B583B0DF
:103F000005460C461F4690F8270006281DD0174E80
:103F1000ECB12CB36388FBB11FB195F82730062BA9
:103F200004D061883046FFF717FEE0B96388AB60C4
:103F30006288130A43EA0223AB8405F10801304684
:103F400002F021FA002003B0F0BD094EE0E70023A3
:103F5000ADF802306C46DCE7FFF716FE6080DBE769
:103F60006FF07C00EFE76FF06F00ECE700040010EB
:103F7000EC03001000B583B009238DF800300190E8
:103F8000013810F1030F03D9002003B05DF804FBE2
:103F900000216846FFF74EFC08B10120F5E74FF01D
:103FA000FF30F2E738B5044690F82730062B12D0E0
:103FB000A3691BB104F1080002F00BFA94F8273052
:103FC000112B1CD0606808B102F0BCF92046FEF746
:103FD00029FA002038BDC06E08B1FEF723FA206F21
:103FE00008B1FEF71FFA2046FFF778FDE0E7636CA3
:103FF000DD68284602F0EDF92846FEF7B7FEA36B10
:10400000002BF4D1DEE7FFFF08B501460348FFF7B8
:10401000A3FD08B1C06808BD0020FCE70004001043
:1040200070B483B0012600251AE003EB8303590026
:104030005318303B01342278A2F13001C9B209296A
:10404000F3D9844211D0FF2B13D802A9294401F8D7
:10405000043C022D0BD82E2A16D1601C5EB101350E
:10406000032D08D804460023E5E70026EBE72046A9
:10407000F4E720460026037803B10026042D06D07D
:10408000002003B070BC704720460026F3E70EB94D
:104090000020F6E79DF807309DF80600000440EA8E
:1040A00003609DF8053040EA03209DF80430184372
:1040B000E7E710B50446836A1BB10168C1F3032129
:1040C00049B9216801F07F012160606800B149B9F8
:1040D0000023236010BD026B0A430263186802F0DC
:1040E00000F9EEE702F0FDF8F2E72DE9F04389B0C0
:1040F00005460F46914601220621FFF7DBFC00280A
:1041000078D095F8403013F0080F0AD195F8533065
:10411000012B02D04FF0FF346EE04FF0000846460E
:104120002DE04FF00008464629E02C462FE002F033
:104130002FFF0024B8F1000F08D006238DF80C30B3
:1041400004954FF0FF3103A8FFF774FB002C53D107
:104150003EB9EB690793002B4ED005A803F096F803
:10416000012607A905A803F0AFF8002844D1079B52
:104170000093002301220421686802F04BF802F04A
:1041800079FE95F8403013F0080FCED16C6D64B114
:1041900000236B6594F8403013F0020FC7D094F8F9
:1041A00040306FF3410384F8403002F0F1FE002C00
:1041B000C0D08FB1A26B130203F47F0343EA026302
:1041C000110A01F47F410B4343EA12637B60A28F23
:1041D000130A43EA02237B80B9F1000F02D00823BF
:1041E000C9F8003095F8403013F0080FA2D14FF015
:1041F0000108A2E74FF0FF34204609B0BDE8F08384
:104200002DE9F04786B00446894690461E460122B5
:104210000621FFF74FFC002800F09680E36E002B8C
:104220005FD09D681A681B691D44AD1AAB4200D867
:10423000ED1A0027002D36D006E094F8423013F036
:10424000080F50D06FF00B05002D16DD16F0010F92
:104250004CD0E26E10689568136811690D44EB1A32
:10426000994200D85B1A02F114010144C9F8001008
:1042700015692D1A9D4228BF1D46284606B0BDE887
:10428000F08705A903A803F01FF882460028DBD1B8
:10429000059B0093002301226121606801F0BAFFB1
:1042A000E36E5546A3B994F85330002BC5D0083BB4
:1042B000012BC2D9002FE4D1E3690593002BC3D0B1
:1042C00016F0100FC0D103A802F0E0FF0127D8E7D5
:1042D0009D681A681B691D44AD1AAB42AAD8ED1A35
:1042E000A8E70025A5E76FF07F05ADE7C6F38006D8
:1042F000009643464A460021E06E00F05EFC05460B
:1043000094F94030002BB8DAE26ED1681368126974
:1043100013445B1A013B9A4200D89B1A226E9A42C0
:10432000ABD894F840306FF3C71384F8403094F85A
:10433000413043F0010384F841300123A4F84830B0
:104340000520FFF7DFFA98E76FF0150595E72DE9EF
:10435000F04F87B006460F46924699461146FFF742
:10436000A1FC002876DD336F9A681C681B691C4429
:10437000A41A013CA34200D8E41A55464FF00008A5
:1043800041E002F077FD96F8403043F0400386F8B4
:1043900040304FF0010B01E04FF0000B23463A464E
:1043A0000021306F00F0B4FB0446BBF1000F3BD19D
:1043B0000123A6F84830FEF78DFF002837D02D1BCB
:1043C0003FD02744B8F1000F35D1336A0593002B55
:1043D00037D019F0100F34D103A802F057FF4FF077
:1043E0000108059B0093002301222221706801F03F
:1043F00011FF336F9A681C681B691C44A41A013CA6
:10440000A34200D8E41A002D1BDD002CDADDAC42FB
:1044100000DD2C4696F8403013F0100FBCD0AC42B3
:10442000AFD04FF0000BB9E702F0B2FDC0E70520B6
:10443000FFF768FAC3E705A903A802F045FF0028C3
:10444000CFD0BAEB050005D196F85330052B04D92F
:104450006FF07F0007B0BDE8F08F6FF01B00F9E749
:1044600038B504460D4601220621FFF723FB00283C
:104470003CD094F853300BB1082B3AD14FF6FF7370
:104480009D42A8BF1D46A4F8505094F8403013F048
:10449000080F25D0E36E23B100229A601A60DA601B
:1044A0005A60236F23B100229A601A60DA605A6062
:1044B0004222002104F17A0009F06CF96022002107
:1044C00004F1D40009F066F90422002104F140004F
:1044D00009F060F994F8403043F0080384F8403064
:1044E0000121204600F088FF002038BD6FF05E00FB
:1044F000FBE76FF05E00F8E710B5044601220621E5
:10450000FFF7D8FA88B194F85330052B10D194F8FE
:10451000403043F0200384F840300123A4F84830B1
:104520000520FFF7EFF9002010BD6FF05E00FBE7FC
:104530006FF05E00F8E7FFFF2DE9F041804602F0E2
:10454000A1FC1B4B1E681B4AD4681860861B29D02F
:104550006427194B9C4227D0E5686468B5F8483059
:10456000002BF6D0B34210D99B1BA5F848302B681E
:104570001BB1B8F1000F11D10027B5F84830002B5E
:10458000E7D0BB42E5D21F46E3E70023A5F8483059
:10459000284601F007F90028E9DADAE72846FFF7AC
:1045A00088FDEAE70126D3E73846BDE8F08100BF81
:1045B00014040010EC030010F4030010F0B40F48D2
:1045C000C468002001E0284664680D4DAC4210D05C
:1045D000E568AF8C8EB2B742F6D195F85360012EE4
:1045E000F1D0AF8F9EB2B742EED1AE6B9642EBD117
:1045F00000E0002505B12846F0BC7047EC03001030
:10460000F40300102DE9F04104460E461746984683
:10461000C56E35B343463A463146284600F078FA2F
:104620000546DEB994F94030002B0CDBE26ED16810
:104630001368126913445B1A013B9A4200D89B1A13
:10464000E26D9A4216D2236843F001032360E26AC6
:1046500012F0010F02D043F4807323602846BDE8B6
:10466000F0810121FFF7DEFA05460028D2D14FF094
:10467000FF35F3E794F8403043F0800384F840308E
:1046800094F8413043F0010384F841300123A4F849
:1046900048300520FFF736F9D5E790F82730062B8C
:1046A00015D110B4826B130203F47F0343EA026353
:1046B000140A04F47F44234343EA12634B60828F5D
:1046C000130A43EA02234B80082010BC70476FF0A6
:1046D0001500704790F82730062B0DD1036F4BB1B2
:1046E0009A6818681B691844801A0138834205D8F3
:1046F000C01A7047806E70476FF01500704790F8D1
:104700002730062B0AD1036F5BB198681A681B69C2
:104710001844801A834205D8C01A70476FF01500FC
:1047200070470020704770B582B004461D460F2ABE
:1047300000F20481DFE812F01000160025000201EB
:104740003600360002010201020102010201890065
:104750009F005C00B400E1002B68C3610023184691
:1047600002B070BD2B68036290F82720112A01D097
:104770000023F4E7022B40F2E480022303620023CB
:10478000EDE73DB190F8263043F0020380F8263083
:104790000023E4E790F8263023F0020380F8263067
:1047A0000023DCE790F82730062B40F0CC80042A69
:1047B00007D0052A0BD02B68042A0ED0636600238D
:1047C000CDE7036F002BF4D06FF01503C7E7E36E5E
:1047D000002BF0D06FF01503C1E7B4F84C20134460
:1047E000013BB3FBF2F303FB02F3A3660023B6E73E
:1047F00090F82730062B40F0A980036F002B40F083
:10480000A880C36E002B40F0A780042600962B469C
:1048100032460021FFF787FF009605F108030522C5
:1048200000212046FFF77FFF0123C4F8CC30C4F8F5
:10483000D03094F8D43013F0010F00F09080B4F829
:104840004C30C4F8D830002389E790F82730062B85
:1048500040F087802B683BB190F8403043F008036C
:1048600080F8403000237AE790F840206FF3C302CD
:1048700080F8402073E790F82730062B74D12B681E
:104880003BB190F8403043F0100380F840300023F3
:1048900065E790F840206FF3041280F840205EE74F
:1048A00090F82730062B62D12B6883B190F8D43072
:1048B00043F0020380F8D43094F8D43013F0020FA0
:1048C00058D194F85330042B08D8002347E790F8C8
:1048D000D4306FF3410380F8D430EDE72046FFF782
:1048E0000EFF034600283FF43AAF0123A4F84830F6
:1048F0000520FFF707F8002331E790F82730062B53
:104900003AD12B689BB190F8423043F0040380F811
:10491000423094F8413043F0010384F841300123E0
:10492000A4F848300520FEF7EDFF002317E790F8C4
:1049300042306FF3820380F84230EAE76FF06C0395
:104940000DE700230BE76FF0150308E76FF0150381
:1049500005E76FF0150302E76FF01503FFE600238C
:10496000FDE66FF01503FAE66FF01503F7E66FF05A
:104970001503F4E60023F2E66FF01503EFE690F876
:104980002730062B0AD1C36E5BB198681A681B6981
:104990001844801A834205D8C01A70476FF015007A
:1049A000704700207047FFFF2DE9F84F8046002335
:1049B00083609A46994685E0534F8BE095F84030E6
:1049C00013F0040F05D113F0020F36D04FF0000B97
:1049D00001E04FF0000BEE6A16F001060BD095F8DF
:1049E0005320012A2CD003F00A030A2B3ED0BBF13E
:1049F000000F2ED10026EB6A13F0040F06D095F8B5
:104A00005320082A00D00AB946F0040613F0020F1A
:104A10003FD0BBF1000F2BD195F8413013F0080FB8
:104A20002DD095F85320042A2ED913F0100F2DD134
:104A300043F0100385F8413023E04FF0010BCAE743
:104A40006B6D7BB193F8403013F0020F0CD1002650
:104A5000D1E72846FFF793FF002801DD0126CAE7CA
:104A60000026C8E70026C6E70126C4E70126C2E7FC
:104A70002846FFF72FFE0028CEDD012300E00023AB
:104A80003BB146F0020604E00023F9E70023F7E714
:104A900001262E634AEA060A6468BC4210D0E56823
:104AA000AB6A4345F8D195F82730062B86D0EE6ADD
:104AB00016F00106EDD0AB6B002BE9D10026E8E73C
:104AC00009F10109B9F1010F06DCB9F1000F3FF45A
:104AD00073AF0E4F7C68E0E70021D8F8000001F0CA
:104AE000F3FB20EA0A0010F00F0107D14AF0100191
:104AF000D8F8000001F0F5FBBDE8F88FD8F8000009
:104B000001F0E2FBF2E700BF08040010F40300101C
:104B10002DE9F04784680568066935442D1B6C1E35
:104B2000A64200D8A41BA1423CD2641A9C4228BFD2
:104B30001C46A4B3856819B10D44B54200D3AD1B22
:104B40001746884681466AB1761BA64228BF26468C
:104B500000F1140A324639460AEB050008F016FE49
:104B6000B44221D8B8F1000F07D12544D9F810304C
:104B7000AB4200D8ED1AC9F80850D9F80C20D9F882
:104B800000309A422CBF002001209D422CBF002102
:104B9000012188420ED09D4201D2C9F80C50204616
:104BA000BDE8F0870024C1E7A21BB919504608F000
:104BB000EDFDD7E7AA42F0D9F1E72DE9F047856886
:104BC0000468066935442C1BA64200D8A41BA142E8
:104BD0002ED2641A9C4228BF1C4634B3D0F8008001
:104BE00021B18844B04501D3A8EB060817460D460D
:104BF000814672B1A6EB0806A64228BF264600F100
:104C0000140A32460AEB0801384608F0BFFDB442E8
:104C100010D8089B4BB945B908EB0403D9F810200C
:104C20009A4200D89B1AC9F800302046BDE8F087A8
:104C30000024CFE7A21B5146B81908F0A7FDE8E70A
:104C40000B2809D8DFE800F006080808080808065D
:104C50000606080600207047012070478A6902F1A5
:104C6000360392F82E100909053903EB810104E09F
:104C7000013302E05A7852B313448B4227D21A7898
:104C80002AB3012AF4D0022AF4D15A78042AF1D1A5
:104C90009A78DB7843EA0223B0F84C209A4216D97E
:104CA00090F8402042F0010280F84020D0F8D8204F
:104CB000B2FBF3F203FB02F2C0F8D820A0F83231C5
:104CC000A0F83031A0F84C30A0F84A307047704757
:104CD000B0F84C30022281F83620042081F83700E9
:104CE0001A0A81F8382081F83930704770B4846925
:104CF00094F82E309B0803F03C0303F12202224477
:104D00000A60C5690E3D268A300A40EA062080B254
:104D1000854200DC28461433834212DAC01A94F824
:104D20002F3013F0200F0AD0A48E230A43EA042365
:104D30009BB21A440A609842D4BF001AC01A70BCD1
:104D400070470020EBE70346896990F8100193F85B
:104D50005320042A04D993F8402012F0010F00D107
:104D6000704793F840206FF3000283F8402002223E
:104D700081F83620042081F83700B3F84A20120A5F
:104D800081F8382093F84A3081F83930602381F86F
:104D90002E30E5E740F20A23A0F84A30A0F84C3064
:104DA000704710B5026F9168546813691944091B64
:104DB0008B4200D8C91A00291BDD04465268D43042
:104DC00001F0EAF8002814DD226F93685468116935
:104DD0000B441B1B994200D85B1A984200D803462B
:104DE0005068034453605368994202D85368591A73
:104DF000516010BD70B5184C246834B179B11A44B3
:104E00003632CA610D46284670BDD5183635422D5A
:104E1000B8BF422529B1CC69AC42F0D201E040F2E2
:104E200056250C46064600212846FDF7C1FF0546DB
:104E30000028E8D044B1E269A169806908F0A6FCC5
:104E40002046FDF793FFDEE7422206F17A018069F2
:104E500008F09CFCD7E700BFE010010010B582B05D
:104E6000D0F8CC40D0F8D020B0F84C3040F20A2135
:104E70000193D0F800310093D0F8E43001FB02F246
:104E800001FB04F1D43001F06CF802B010BDFFFF5B
:104E900030B585B00446826B130203F47F0343EA06
:104EA0000263110A01F47F410B4343EA1263039347
:104EB00001A903A8FEF7E6F801280AD094F85230B9
:104EC000013384F852300398FEF734F9002005B01E
:104ED00030BD002584F8525094F8413043F0080367
:104EE00084F841304222294604F17A0008F052FC4D
:104EF000062201A904F1800008F048FC082384F888
:104F0000863084F88750452384F8883084F88A50A6
:104F1000342384F88B30802384F89030062384F87F
:104F200091301C4B5B69C4F89830A26B130203F4F8
:104F30007F0343EA0263110A01F47F410B4343EA12
:104F40001263C4F89430A28F130A43EA0223A4F830
:104F50009C30A28C130A43EA0223A4F89E30C4F8C2
:104F6000E4500D4A1368C4F8003103F581731360EF
:104F7000502384F8A830022384F8A9302046FFF794
:104F800009FFB4F84C30C4F8C8302046FFF766FF7C
:104F900001209CE744000010180400102DE9F041A6
:104FA0008AB005461746002900F0CC8098460E4688
:104FB00033B9F1693046FEF79BF906464FF0010818
:104FC000002E00F0BC80B469002D00F0CB80EB6EA9
:104FD000002B00F0C280D9681A681B691A44521A63
:104FE000013A934200D8D21AD5F8C810D5F8D83073
:104FF0008B4228BF0B46286C6649014001B1002353
:10500000B5F84A10994202D9914200D80B464FF6A2
:10501000FC72934200F2A3801A46110221F07F41F4
:1050200021F0FF01C2F307220A43228695F84120AE
:105030006FF3000285F84120D5F8E42013446B6437
:10504000D5F80021130203F47F0343EA0263110A37
:1050500001F47F410B4343EA1263C4F8263094F80D
:105060002F3013F0010F0CD0A7F12801D5F8002143
:105070000A44D5F8F8108A4203D023F0010384F8DB
:105080002F30D5F8E420130203F47F0343EA0263D0
:10509000110A01F47F410B4343EA1263C4F82A303A
:1050A0008023A3753B029BB243EA1723238215B1E9
:1050B000394B5B690BB9D4F81E30D4F81A20C4F808
:1050C0001E20C4F81A30638CA28C6284A3843349F6
:1050D0000B881A0A42EA0322628201330B80002005
:1050E0002075607520766076142204F10E01FEF7BB
:1050F000CFF9030A43EA002080B2C0432083012194
:105100002046FEF72CFA638E2BB94FF0FF3384F85C
:10511000323084F833300E37F761A51D0622294658
:10512000204608F033FB06221B49284608F02EFBD8
:1051300041463046FDF700FDB8F1000F1BD00AB024
:10514000BDE8F081242201A808F024FB05F17A03D0
:1051500007934223089301AE2BE76A6E44E74FF6AC
:10516000FC725AE7D4F82630D4F82A20C4F8262056
:10517000C4F82A3094E7638CA28C6284A384D4F8A8
:105180001E30C4F81A3006222146284608F0FEFADE
:10519000D5E700BF80000400440000107403001035
:1051A00008B501468369142283F82F20502283F822
:1051B0002E20002328221846FFF7F0FE002008BD0D
:1051C00070B50D461C46D0F8D810D0F8E430D0F8B1
:1051D000EC209B1A1944C0F8C810C66E86B1F3685B
:1051E000326836693244D21A531E9E4200D89B1B45
:1051F0008B4228BF0B46C0F8C8301CB9204670BD92
:10520000436EF5E7012322462968FFF7C7FE002316
:105210002B60F3E710B582B0044644F62063019397
:1052200090F85330022B06D0B0F848305BB3B4F896
:10523000480002B010BD90F8413013F0080F0ED0B6
:1052400090F85230022B06D8013B40F6B83202FAF1
:1052500003F3019306E042F6F823019302E04FF4D2
:10526000FA730193019A642303FB02F3B3F57A7F87
:1052700007D3154AA2FB0323C3F38F13A4F84830C6
:10528000D5E70123FAE701AAD0F8C410D43000F022
:10529000D0FE019B13B980B101230193019A6423CD
:1052A00003FB02F3B3F57A7F0BD3074AA2FB032378
:1052B000C3F38F13A4F84830B9E744F62063019391
:1052C000ECE70123F6E700BFD34D621010B50446AA
:1052D00001F0D8FDA06510BD10B582B00446CB69C1
:1052E000C3610B6A036291F8263080F826304B6E5A
:1052F00043668B6E8366CB6DC3650B6E0366D1F818
:10530000CC30C0F8CC30D1F8D030C0F8D0308B6A77
:1053100023B18362CB6A43F00503C362114B5B691F
:1053200001938A8C130A43EA0223ADF8023094F801
:10533000403043F0040384F840306165B1F84E30EA
:105340000133A1F84E300123082269462046FEF7BA
:10535000D5FD10B9012002B010BD2046FEF722FE97
:105360000020F8E7440000102DE9F8439469D4F8D0
:1053700026502C0204F47F0444EA05642E0A06F445
:105380007F46344344EA156473B300F1D4071D46E5
:1053900090F85330032B27D9C66EEEB1D6F808C06B
:1053A000336836693344A3EB0C03013B9E4200D8BB
:1053B0009B1B9046894606462A462146384600F001
:1053C000DAFD011E16DB2B464A463046FFF71AF976
:1053D000854203D100200BE0436EEAE74046FFF729
:1053E000DFFE4FF0FF3003E0002380F81031184655
:1053F000BDE8F8830020FBE770B504460D4690F841
:105400005330042B05D9082B01D0012202E00022E1
:1054100000E00022042D05D9082D01D0012302E06F
:10542000002300E000239A4256D0002B43D094F88A
:10543000403013F0040F31D013F0080F2AD1666DFD
:1054400066B1736D43B3336843F004033360F26AAB
:1054500012F0010F02D043F48073336000236365C0
:1054600094F8403003F0FB0343F0020384F840302B
:1054700094F85300FFF7E4FB10B90023A4F8483078
:1054800084F853502046FFF721FF16B13046FEF74F
:1054900010FE70BD2646D3E77465D4E7236843F059
:1054A00008032360E26A12F0020F11D043F4007384
:1054B00023600026DCE7236843F020032360E26AD0
:1054C00012F0040F06D043F4806323600026CFE778
:1054D0000026CDE70026CBE775B994F8403013F0ED
:1054E000060F0BD013F0080F01D00026C8E72046A6
:1054F000FEF740FD0026C3E70026C1E70026BFE710
:105500002DE9F04784B00446884617460B68A3B3DC
:105510009D6904F1D4090023039395F82F3043F0DB
:10552000100385F82F30236F002B79D0B4F84A3060
:10553000012B25D80026002E03DB94F85330052BD1
:1055400070D0002E40F3968095F82F3003F0F703CB
:1055500007F11402D2B2920085F82E2043F0100316
:1055600085F82F301EB143F0080385F82F303E44F4
:105570002836304604B0BDE8F08700F17A05C8E768
:1055800003AAD4F8C410484600F020FD824606461F
:105590000028D0DD3B460246D8F800102046FFF731
:1055A00029FC002863D0C8F80000856907F136029D
:1055B0002A44206FD0F800E0036903991944A1EB55
:1055C0000E018B4200D8C91A012300935346FFF7FE
:1055D000F4FAB4F8403023F47E5323F03F035B0425
:1055E0005B0C402BA7D1226F936812691344039977
:1055F0005B1A9A4200D89B1A98429CD195F82F309A
:1056000043F0010385F82F30D4F800315344C4F837
:10561000F83094F8413043F0400384F841308AE791
:1056200000268AE794F8403013F0200F89D04846CE
:1056300000F0F9FC002884D094F840306FF3451353
:1056400084F8403095F82F3043F0010385F82F306F
:1056500094F8413043F0410384F84130D4F8F430F9
:10566000C4F8F83006212046FFF7C6FE69E74FF080
:10567000FF3666E794F8413013F0030F7FF464AF10
:1056800077E72DE9F04180460D4600273C46072C80
:1056900011D8002229464046FFF732FF061E0ADDD8
:1056A0000123324629684046FFF778FC00232B602F
:1056B00037440134EBE73846BDE8F08130B583B0BC
:1056C000044690F85330022B0ED190F85230022B42
:1056D00018D890F8413013F0080F18D1FFF7D8FB15
:1056E000012814D000250AE002A9002341F8043D56
:1056F000FFF7C7FF0546019808B1FDF737FB2846BD
:1057000003B030BD0821FFF777FE0025F7E704F16D
:105710007A012046FFF7DCFA00F128051430C0B208
:10572000800084F8A80094F85230013384F8523095
:1057300000232A4619462046FFF730FCDFE7FFFF2B
:1057400090F85330082B06D8DFE803F0252505052F
:1057500005250505250010B5044601F093FBA36D52
:10576000C01A0F4B984201D8012010BD08212046D5
:10577000FFF742FE94F8403013F0040F0DD013F001
:10578000080F02D04FF0FF30EFE72046FEF70AFC8B
:105790004FF0FF30E9E7002070470120E5E700BF48
:1057A000A086010010B5044690F85330042B03D9AD
:1057B000036F0BB1FFF7F5FA94F85330042B01D8BF
:1057C000022B02D12046FFF779FF2046FFF722FD8A
:1057D0002046FFF7B5FF10BDF8B505460E468F69A8
:1057E00090F8403013F0080F43D043F0040380F8E2
:1057F000403068650446002C39D07A8C130A43EA9D
:105800000223A387D7F81A20130203F47F0343EA85
:105810000263110A01F47F410B4343EA1263A3635D
:10582000244D2B68C4F80031D7F82620130203F466
:105830007F0343EA0263110A01F47F410B4343EA09
:105840001263C4F8E4302046FFF7A4FA2046FFF7BD
:1058500005FB2B6803F581732B6003212046FFF7BE
:10586000CBFD4222B16904F17A0007F08FFF204698
:10587000F8BDB0F84E20B0F850309A4210D206224F
:1058800001210220FEF758FA0446431E13F1030FCC
:105890000BD82946FFF720FD0028ACD10024E6E70D
:1058A0000846FFF77DFC0024E1E73046FFF778FC6F
:1058B0000024DCE7180400102DE9F04104461746E7
:1058C0001D460B689E69D43096F82F20D6F82680A6
:1058D0004FEA082303F47F0343EA08634FEA1821E1
:1058E00001F47F410B4343EA186894F853100229EE
:1058F0002CD04FF0100C02F01703634529D1A38F71
:10590000A4F82E31A38CA4F82C31022933D00FB97E
:10591000C4F8E480D4F8F0300133C4F8003194F8CE
:105920005330022B01D0002F40D0102386F82F30A7
:1059300005F128071435EDB2AD0086F82E5005218B
:105940002046FFF759FD3846BDE8F0814FF0120CB4
:10595000D1E708212046FFF74FFD96F82F3043F09E
:10596000040386F82F3005F128071435EDB2AD0099
:1059700086F82E50E7E7102384F8A930B4F84A30AF
:10598000D4F80021414600F0C3FA08F10103C4F83D
:10599000EC30C4F8E430D4F8F4300133C4F8F43017
:1059A000D4F808310133C4F80831B3E70027C6E75B
:1059B00038B504468D6995F82F00D5F82A201302D2
:1059C00003F47F0343EA0263110A01F47F410B43AE
:1059D00043EA126310F0010F04D0D4F8E82001323A
:1059E000C4F8E42094F8412012F0400F2AD1D4F8F2
:1059F000F430C4F8F83042F0400384F8413094F8B1
:105A0000422012F0010F29D0D4F8F8300133C4F845
:105A1000F43094F94130002B2CDB002385F82F3033
:105A2000D4F8F430C4F8003195F82F308BB394F8E3
:105A30001001283094F810311433DBB29B0085F844
:105A40002E3038BDD4F8F82001329A42D7D194F8DC
:105A5000423043F0010384F84230D0E7D4F8F83004
:105A6000C4F8F430112385F82F300A212046FFF7BF
:105A7000C3FCD5E712F0020F07D1102385F82F30B1
:105A800008212046FFF7B8FCCAE7002385F82F302D
:105A9000F6E70020CEE72DE9F04F83B004460E462E
:105AA00092461F460B689D6900F1D40995F82F8036
:105AB000D5F826B04FEA0B2303F47F0343EA0B63C8
:105AC0004FEA1B2202F47F42134343EA1B6B2A8EE8
:105AD000130A43EA02239BB2C0F8C43018F0100F37
:105AE00029D1236F13B12046FFF75BF9D4F8F430C6
:105AF000C4F8003194F8413013F0200F02D118F0AF
:105B0000010F6FD013F0400F3ED1484600F0C4FAA9
:105B10008046484600F087FAB8F1000F5DD00028B3
:105B20005DD00BEB0A03D4F8E4209B1A012B2BDD8C
:105B30000023984634E0D5F82A100B0203F47F03C3
:105B400043EA01630A0A02F47F42134343EA116104
:105B5000484600F094FA0346206F0028C1D0002B7D
:105B6000BFD0002100910A46FFF727F80028B8D0DF
:105B7000236843F002032360E26A12F0020FB0D000
:105B800043F400732360ACE794F8413043F0200302
:105B900084F8413031682046FFF70AFF8046012330
:105BA000BBB9102385F82F30BAF1000F10D007F1E0
:105BB000280807F11403DBB29B0085F82E3094F817
:105BC000413013F0400F03D0D4F8F830C4F8F4306B
:105BD0005FB1404603B0BDE8F08F0023E0E78046A8
:105BE0000023DDE74FF00008DBE73A463146204668
:105BF000FFF786FC0028ECDD8046EAE72DE9F04F50
:105C000083B004460E4608688769D7F826301D021F
:105C100005F47F0545EA03651A0A02F47F4215433D
:105C200045EA136597F82FA001A9FFF75FF88046B2
:105C300094F85330042B04D9D4F8E4206B1C9A4216
:105C40003ED005EB080BD4F8EC30ABEB0303002B94
:105C500001DDC4F8ECB04346326801992046FFF7F5
:105C600083FB00287EDB31682046FFF76CF8814615
:105C700094F85330042B2AD01AF0010F14D094F961
:105C80004130002B10DBC4F8E8B094F8413043F009
:105C9000800384F8413013F0400F05D194F842306E
:105CA00043F0020384F8423094F85330023B082B4F
:105CB0005BD8DFE803F04115414951515A5A510070
:105CC00094F8413043F0010384F84130B9E70AF019
:105CD0001F03022BD0D103212046FFF78DFBCBE71A
:105CE00039462046FEF7F4FF122387F82F3000F1E3
:105CF00028091430C0B2800087F82E000421204605
:105D0000FFF77AFB0135C4F8EC50C4F8E450D4F83E
:105D1000F0300133C4F80831C4F8F430B9F1000FA1
:105D200006DD4B46424631462046FFF749FA81469A
:105D3000484603B0BDE8F08F4B4642463146204608
:105D4000FFF7BAFD8146E9E74B4642463146204619
:105D5000FFF7A1FE8146E1E731682046FFF728FE04
:105D60008146DBE74FF0FF39E2E74FF00009DFE75C
:105D7000F0B583B00190846994F82F50D4F81E6078
:105D8000330203F47F0343EA0663300A00F47F40E2
:105D90001843A18C0B0A43EA0121D4F81A703B0284
:105DA00003F47F0343EA07633A0A02F47F421A438B
:105DB000B4F822C04FEA1C2343EA0C239BB242EA08
:105DC000176289B240EA1660FEF7F8FB30B106466A
:105DD00090F853703846FEF733FF70B905F01F0393
:105DE000102B5AD015F0040F02D0002003B0F0BDE4
:105DF0000198FFF7D5F90020F8E7002386F8523024
:105E0000012F28D015F0040F3CD105F01F05022DFD
:105E100001D1042F43D8019B99691422223106F144
:105E20009C0007F0B3FC3046FFF750FA94F82E3090
:105E300003F0F003502B2BD801A93046FFF7DEFE0C
:105E4000019818B1FCF792FF002301933046FFF749
:105E5000E1F90120CAE705F01F03022B09D015F074
:105E6000040F01D00020C1E70198FFF799F9002045
:105E7000BCE701993046FFF7AFFC06460028D2D1B7
:105E80000020B3E700213046FFF7B6FA0020ADE767
:105E900001993046FEF7E2FECEE70020A6E700209B
:105EA000A4E7FFFF838C190A41EA032189B2124B50
:105EB000DB680BE092F8404014F0020F12D042650C
:105EC000012000E0002010BC70475B680B4A934241
:105ED00010D01A688A42F8D110B4DA6892F82740D4
:105EE000062CE7D05B68054A9342EBD01A688A42D9
:105EF000F8D1F2E700207047EC030010F403001023
:105F0000B0F85E308B4201D9002070470120704705
:105F100010B4002404600124047093B11C46B0F84E
:105F20005E300BB1A0F85E40B0F85C30A34200D800
:105F30003BB94368B3FBF4F304FB03F34360A0F8FD
:105F40005C40B0F85C3043644FF4FA738363C16023
:105F500001618161C261026242638262C26210BCFD
:105F6000704738B51D4641608260059B049A2946FA
:105F7000FFF7CEFF38BD10B404698C4206D19342BE
:105F800007D314440461002010BC70474FF0FF3069
:105F9000FAE74FF0FF30F7E770B5836C002B02DDB6
:105FA0000026304670BD456C8D4200D30D46044638
:105FB000436B03642E468564C2640023436500F08E
:105FC00061FF2065636B1D446563EAE7F8B5856C86
:105FD0002DB31646044690F8563013F0010F0CD03E
:105FE000876B90F854309F4000F04CFF236DC01A2F
:105FF00000EB800043009F4213D894F8563043F0E2
:10600000010384F8563094F85430013384F8543046
:1060100000F038FF2065236CE362E36C33602846B0
:10602000F8BD0025FBE7836C0BB100207047012011
:10603000704738B500231360836CE3B115460446FE
:1060400090F8563013F0010F04D1FFF759FF98B1C3
:10605000012011E000F016FF236DC01A00EB800054
:106060004200A36B94F854108B40934205D99B1ABD
:106070002B60012000E0002038BD0120FCE7836C8C
:1060800033B1026A1A448A4204D80262002282644E
:10609000184670470023FBE703698069181AC0435C
:1060A000C00F70472DE9F04182B00446436902A851
:1060B00040F8043DA5692946FCF7E4FF064602289E
:1060C0000BD0012811D050B901990020FCF7DAFE5D
:1060D000019B63612046FDF707F8022E47D1204659
:1060E000FCF744FE02B0BDE8F081238CAB84638CE6
:1060F0006B84E36908339BB21A0A42EA0323EB84F8
:10610000002785F8287085F82970A36993F8068020
:1061100018221949A81D07F039FBE3691C339BB20B
:106120002B820E33E3612A8A130A43EA02232B826D
:106130006369C5F81E302F766F76142205F10E01C3
:106140003846FDF7A5F9030A43EA00239BB2DB4377
:106150002B8318F0020F05D1002385F8283085F82D
:106160002930BAE701212846FDF7F9F9B5E7012101
:106170002046FCF7E1FCB5E74400001070B5054689
:1061800086690846FDF740FF28B30446D6F81A1082
:10619000B01DFCF777FE00F06DFEFCF7FBF9294619
:1061A00004F1380000F0EFF8FCF704FA00F0F0FE1C
:1061B000606810B1012100F094F8A36A6BB1E26A43
:1061C00012F0010F01D1012006E00121186800F052
:1061D00088F8012000E0002070BD0120FCE71AB91A
:1061E000084206D10020704731EA000303D00020A6
:1061F0007047012070470120704710B51C20FCF744
:10620000ABF8044620B1002340F8043B00F0ADF8A1
:10621000204610BD2DE9F84307460E4691469846A4
:10622000089D00F027FE3C68424631462046FFF7B5
:10623000D6FFE8B1B9F1000F2FD024EA06033B6086
:10624000002500F0A5FE85B138B91E4B4FF08052F5
:106250001A60BFF34F8FBFF36F8F01F05FF90446F1
:1062600010F0007F1BD024F07F442046BDE8F88367
:10627000002DE6D0B9F1000F0CD10021B8F1000FCC
:1062800001D041F080612A463143381D00F072FF91
:106290000024D6E74FF08071F0E70025D1E7FCF746
:1062A00079F93C68424631462046FFF798FF28B10D
:1062B000B9F1000F02D024EA06063E60FCF77AF935
:1062C000D1E700BF04ED00E070B506460C46FCF7D0
:1062D00061F9356825EA04043460FCF76BF9284657
:1062E00070BDF8B504460D4600F10C0600F0C2FD85
:1062F000206921682943216000270AE0216832EAE9
:10630000010105D111E0216841F0007100F092FF18
:106310002846B0420ED04568036823F07F4213F050
:10632000806FEBD121681142F2D013F0807FEAD068
:106330001743E8E7236823EA0707276000F028FEF1
:106340002068F8BD10B5044600F094FD04E04FF05D
:106350000071206900F06EFF6368002BF7D12046C2
:10636000FCF760F800F014FE10BD00F10803436074
:106370004FF0FF328260C360036100230360704707
:1063800000230361704743684B609A688A609A688B
:10639000516099600861036801330360704730B44D
:1063A0000D68B5F1FF3F02D000F1080202E002697A
:1063B00004E01A4653681C68AC42FAD953684B6033
:1063C00099608A605160086103680133036030BCE2
:1063D00070470369426881689160826841685160D2
:1063E0005A68824206D0002202611A68013A1A6095
:1063F0001868704782685A60F5E7436A23B1036BF7
:106400001868C0F1070070470020704710B50446B7
:10641000FCF7C0F8A26BE36B9A4204D00024FCF7AF
:10642000C9F8204610BD0124F9E710B50446FCF771
:10643000B1F8A36B23B10024FCF7BCF8204610BDD3
:106440000124F9E770B504461646856B026C5AB90B
:1064500003681BB100200135A56370BD406800F0E2
:10646000D7FF00236360F6E76EB9806807F08EF906
:10647000226CA3681344A3606268934219D3236813
:10648000A3600020E7E7C06807F080F9226C524261
:10649000E3681344E36021688B4202D263681A44C4
:1064A000E260022E01D00020D5E725B1013D002099
:1064B000D1E70020CFE70020CDE7026C72B110B524
:1064C000C3681344C3604468A34201D30368C36034
:1064D0000C46C168204607F059F910BD704738B521
:1064E0000546FCF757F895F8454064B203E000F024
:1064F00017FF013C64B2002C08DD6B6A33B105F173
:10650000240000F05BFE0028F3D0F0E7FF2385F8BD
:106510004530FCF74FF8FCF73DF895F8444064B27D
:1065200003E000F0FDFE013C64B2002C08DD2B69A5
:1065300033B105F1100000F041FE0028F3D0F0E780
:10654000FF2385F84430FCF735F838BD38B50446EC
:106550000D46FCF71FF82168E26B236C03FB021069
:1065600060600020A063A160013A02FB0313E360B6
:10657000FF2384F8443084F84530A5B923691BB95A
:10658000FCF718F8012038BD04F1100000F016FEE9
:106590000028F5D0084B4FF080521A60BFF34F8FA0
:1065A000BFF36F8FECE704F11000FFF7DEFE04F19C
:1065B0002400FFF7DAFEE3E704ED00E038B51D46FE
:1065C000049C0B4649B12260E0632364012120460C
:1065D000FFF7BCFF84F84C5038BD2460F4E7F0B5F9
:1065E00083B0054617460E4689B100FB01F05030D6
:1065F000FBF7B2FE044638B100903B4600F1500272
:1066000031462846FFF7DAFF204603B0F0BD0020F0
:10661000EDE710B50C4602220021FFF7E0FF03462C
:1066200000B18463184610BDF0B585B004460F462E
:1066300001921E46002539E0324639462046FFF7D2
:1066400001FF636A6BB938B13C4B4FF080521A605E
:10665000BFF34F8FBFF36F8FFBF7ACFF012005B087
:10666000F0BD04F1240000F0A9FD0028F4D0334B64
:106670004FF080521A60BFF34F8FBFF36F8FEBE77D
:10668000FBF798FF0020EAE702A800F011FE0125C1
:1066900019E0002384F8443021E0002384F84530D9
:1066A00023E02046FFF71BFF00F072FCFBF772FFB0
:1066B000A26BE36B9A42BFD3022EBDD0019B002B8D
:1066C000DED0002DE0D0FBF775FF00F0D3FBFBF729
:1066D00061FF94F844305BB2B3F1FF3FD9D094F836
:1066E00045305BB2B3F1FF3FD7D0FBF763FF01A9A1
:1066F00002A800F0E9FDC8B92046FFF787FE002890
:10670000CFD0019904F1100000F026FD2046FFF7DC
:10671000E6FE00F03DFC0028C8D1084B4FF0805247
:106720001A60BFF34F8FBFF36F8FBFE72046FFF7AD
:10673000D6FE00F02DFC002091E700BF04ED00E044
:10674000F8B5EFF311864FF0280484F31188BFF3F6
:106750006F8FBFF34F8F856BC46BA54205D3022BA0
:1067600003D0002086F31188F8BD1746054690F83F
:10677000454064B21A46FFF765FEB4F1FF3F05D00D
:10678000013464B285F845400120EBE76B6A0BB930
:106790000120E7E705F1240000F010FD18B127B152
:1067A00001203860DEE70120DCE70120DAE7FFFFA7
:1067B000F0B585B004460F46019200263CE039460C
:1067C0002046FFF77AFE013DA563236923B9FBF755
:1067D000F1FE012005B0F0BD04F1100000F0EEFC68
:1067E0000028F4D0344B4FF080521A60BFF34F8F23
:1067F000BFF36F8FEBE7FBF7DDFE0020EAE702A8AF
:1068000000F056FD012621E0002384F8443029E001
:10681000002384F845302BE02046FFF760FE00F0AF
:10682000B7FB09E02046FFF75AFE00F0B1FB204617
:10683000FFF7FBFD00283DD1FBF7ACFEA56B002D5B
:10684000BDD1019B002BD6D0002ED8D0FBF7B2FED5
:1068500000F010FBFBF79EFE94F844305BB2B3F1FE
:10686000FF3FD1D094F845305BB2B3F1FF3FCFD0BA
:10687000FBF7A0FE01A902A800F026FD0028D1D157
:106880002046FFF7D2FD0028C6D0019904F124006C
:1068900000F062FC2046FFF722FE00F079FB0028A2
:1068A000CAD1054B4FF080521A60BFF34F8FBFF330
:1068B0006F8FC1E700208DE704ED00E070B584B074
:1068C000044601910026354648E0013BA363236856
:1068D0003BB123694BB9FBF76DFE0126304604B08E
:1068E00070BD00F027FE6060F3E704F1100000F0D7
:1068F00065FC0028EFD0424B4FF080521A60BFF386
:106900004F8FBFF36F8FE6E7FBF754FE0026E5E7F6
:1069100002A800F0CDFC01252AE0002384F84430D1
:1069200032E0002384F8453034E0FBF733FE606842
:1069300000F012FD0646FBF73DFE3BE02046FFF768
:10694000CEFD00F025FB09E02046FFF7C8FD00F072
:106950001FFB2046FFF769FD002840D1FBF71AFE18
:10696000A36B002BB1D1019B002BCDD0002DCFD03C
:10697000FBF720FE00F07EFAFBF70CFE94F84430A3
:106980005BB2B3F1FF3FC8D094F845305BB2B3F1CE
:10699000FF3FC6D0FBF70EFE01A902A800F094FC51
:1069A0000028D1D12046FFF740FD0028C6D023683B
:1069B000002BBAD0019904F1240000F0CDFB204651
:1069C000FFF78DFD00F0E4FA0028C7D10C4B4FF023
:1069D00080521A60BFF34F8FBFF36F8FBEE7002E58
:1069E0003FF47CAFFBF7D6FD2046FFF706FD0146DE
:1069F000606800F04DFDFBF7DDFD00266EE700BF8F
:106A000004ED00E010B50446FBF7C4FDA46BFBF7F2
:106A1000D1FD204610BDFFFF0023092B0CD8074AEB
:106A200052F833200AB10133F7E7044A42F8331031
:106A300002EBC30358607047704700BF1C0400108E
:106A40000023092B0FD8084A02EBC3025268824286
:106A500001D00133F5E7044A002142F8331002EB7C
:106A6000C3035960704770471C04001010B50446FA
:106A7000FFF7E6FF2046FBF7D5FC10BD70B50446D6
:106A80000D461646FBF786FD94F844305BB2B3F131
:106A9000FF3F0DD094F845305BB2B3F1FF3F0BD010
:106AA000FBF788FDA36B5BB12046FFF718FD70BDB7
:106AB000002384F84430EDE7002384F84530EFE705
:106AC0003246294604F1240000F066FBECE7FFFFA4
:106AD000084B1B681B683BB1064B1B68DB68DB6817
:106AE0005A68054B1A607047034B4FF0FF321A602B
:106AF000704700BF700400104805001010B5044630
:106B0000006BFBF78FFC2046FBF78CFC10BD2DE9DA
:106B1000F04781460D4617469A46089EDDF82480C8
:106B20000A9C9200A521206B06F034FE236B07F12E
:106B30008042013A03EB820727F007070023082B66
:106B400007D8E95CE21882F83410EA5C0AB1013334
:106B5000F5E7002384F83C30062E00D90626E662CD
:106B6000A6640025E564201DFFF70AFC04F1180067
:106B7000FFF706FC2461C6F10706A661646225657D
:106B800084F85450524649463846FBF7D9FC2060F9
:106B9000B8F1000F01D0C8F80040BDE8F087FFFF52
:106BA00038B5002407E004EB840293000E48184433
:106BB000FFF7DBFB0134062CF5D90C4D2846FFF717
:106BC000D4FB0B4C2046FFF7D0FB0A48FFF7CDFB68
:106BD0000948FFF7CAFB0948FFF7C7FB084B1D60D0
:106BE000084B1C6038BD00BF780400101C05001065
:106BF00030050010500500107C05001068050010DD
:106C0000700400107404001010B50446FBF7C2FCB9
:106C1000214A136801331360204B1B685BB1204B82
:106C20001B686BB91D4B1B68DA6AE36A9A4207D886
:106C30001A4B1C6004E0194B1C601368012B27D011
:106C4000184A1368013313602364E36A01229A40EF
:106C50001549086802430A6003EB83039A00211D6B
:106C600012481044FFF78FFBFBF7A4FC0C4B1B688A
:106C70006BB10A4B1B68DA6AE36A9A4207D20C4B83
:106C80004FF080521A60BFF34F8FBFF36F8F10BD6C
:106C9000FFF786FFD4E700BF040500106C04001066
:106CA0006405001014050010180500107804001089
:106CB00004ED00E00F4B1B68D3B110B5FBF76AFC85
:106CC0000D4BDB68DC68201DFFF783FB0B4A136864
:106CD000013B1360074A1368013B1360FBF76AFC32
:106CE0002046FFF70BFF034B1B68002BE6D110BDBE
:106CF000704700BF080500107C0500100405001057
:106D000008B5FFF7D7FFFCE770B504460E461D4BEC
:106D10001D681D4B18680430FFF75BFB50B91A4B18
:106D20001B68DA6A012303FA02F218490B6823EAA6
:106D300002030B60B4F1FF3F13D02C44124B1B68CD
:106D40005C60A54216D8124B18680F4B19680431C5
:106D5000FFF725FB0F4B1B68A34212D90D4B1C609C
:106D60000FE0002EE9D0084B196804310A48FFF7FC
:106D70000AFB06E0094B1868034B19680431FFF75A
:106D80000EFB70BD900500106C040010180500107B
:106D9000700400104805001068050010740400100D
:106DA0002DE9F04385B00746884615469946900080
:106DB000FBF7D2FAF8B106465820FBF7CDFA0446A5
:106DC000A8B10663D4B10023039302940D9B0193F1
:106DD0000C9B00934B462A4641463846FFF797FEE8
:106DE0002046FFF711FF012005B0BDE8F0833046D3
:106DF000FBF718FBE6E74FF0FF30F5E74FF0FF3009
:106E0000F2E7FFFF00B583B0144B0193002300931A
:106E10004FF4967212491348FFF7C2FF012804D0BD
:106E2000012805D003B05DF804FB00F081FCF7E712
:106E30004FF0280383F31188BFF36F8FBFF34F8F99
:106E4000094B4FF0FF321A60084B01221A60084BC1
:106E500000221A60FBF710FCE4E700BF44050010B5
:106E600038110100016D0000480500106405001094
:106E700090050010024A136801331360704700BF89
:106E800010050010014B1868704700BF90050010F6
:106E9000F8B5344B1B68002B58D1334B1D680135B6
:106EA0001D6085B1314B1B68AB4245D90027304B83
:106EB0001B68DB6A03EB83039A002E4B9B58012B64
:106EC00049D9012747E02C4A11682C4B18681060FB
:106ED00019602B4A136801331360FFF7F9FDE1E7EE
:106EE0000127254B1B681B6843B3234B1B68DB68DA
:106EF000DC6863689D4226D3261D3046FFF769FA99
:106F0000A36A1BB104F11800FFF763FAE36A0122D8
:106F10009A401C49086802430A6003EB83039A0005
:106F2000314614481044FFF72EFAE26A104B1B68F2
:106F3000DB6A9A42D4D2D4E70027D2E70B4B4FF05A
:106F4000FF321A60B3E7094A1360B0E70E4A1368CC
:106F50000133136000270D4B1B6803B1012738462E
:106F6000F8BD00BF10050010900500104805001086
:106F70006C040010780400107004001074040010F9
:106F80004C050010180500100C05001094050010A9
:106F900038B5FBF7FFFA2E4B1A68013A1A601B68E6
:106FA000002B4DD12B4B1B683BB300242A4B1B6895
:106FB0002BB3294BDB68DC6804F11800FFF709FAF2
:106FC000251D2846FFF705FAE36A01229A40234966
:106FD000086802430A6003EB83039A0029462048AD
:106FE0001044FFF7D0F9E26A1E4B1B68DB6A9A4235
:106FF000DCD31D4B01221A60D8E7002421E00CB13C
:10700000FFF766FD194B1C6874B9174B1B68E3B199
:10701000174B4FF080521A60BFF34F8FBFF36F8F43
:1070200001240EE0013C07D0FFF732FF0028F9D021
:107030000D4B01221A60F5E70C4B00221A60E4E7C1
:107040000024FBF7B7FA204638BD0024F9E700BF5B
:107050001005001004050010500500101805001060
:10706000780400106C040010940500100C0500104A
:1070700004ED00E010B540B90A4B4FF080521A60A1
:10708000BFF34F8FBFF36F8F10BD0446FFF7F2FEC3
:1070900000212046FFF738FEFFF77AFF0028EBD0EB
:1070A000F2E700BF04ED00E0264B1B68002B33D154
:1070B00010B5254B00221A60244B1B681B6B1A6805
:1070C000B2F1A53F03D15A68B2F1A53F28D01F4BBA
:1070D00018681968343100F074FE1D4B1B68B3FA50
:1070E00083F3DBB2C3F11F031A489A00D418A1003E
:1070F00001444C6864684C601A44910008310844AB
:10710000844216D003EB83039A00124B13445B684E
:10711000DA680E4B1A6010BD0B4B01221A607047E3
:107120009A68B2F1A53FD2D1DB68B3F1A53FCED1C9
:10713000D3E7606803EB83029100064A0A4450607B
:10714000E0E700BF10050010940500106C0400106B
:10715000180500107804001010B50C46044B19688F
:107160001831FFF71CF901212046FFF7CDFD10BDB6
:107170006C04001010B51446064B1A6841F000412B
:10718000916119681831FFF7FEF801212046FFF7D9
:10719000BBFD10BD6C04001038B50D461446064BFF
:1071A00019681831FFF7EFF80CB14FF0FF352146A1
:1071B0002846FFF7A9FD38BD6C04001038B5C36838
:1071C000DC6804F118052846FFF703F9134B1B6828
:1071D000E3B9251D2846FFF7FCF8E36A01229A402F
:1071E0000F49086802430A6003EB83039A002946AB
:1071F0000C481044FFF7C7F8E26A0B4B1B68DB6AC8
:107200009A4208D90120094B186038BD2946084820
:10721000FFF7B9F8F0E70020F7E700BF100500100E
:1072200018050010780400106C040010940500107C
:107230005005001038B541F000410160C468FFF707
:10724000C8F8251D2846FFF7C4F8E36A01229A40D2
:107250000A49086802430A6003EB83039A0029463F
:1072600007481044FFF78FF8E26A064B1B68DB6A99
:107270009A4202D9044B01221A6038BD1805001049
:10728000780400106C0400109405001010B504463A
:10729000FBF780F9044B1B682360044B1B68636099
:1072A000FBF788F910BD00BF4C05001090050010D9
:1072B000034B1B680360034B1B684360704700BFB0
:1072C0004C05001090050010F8B504460D46FBF77C
:1072D00061F9114B1A686168501A2B68B3F1FF3FCE
:1072E00016D027680D4E3668B74201D0914211D9A9
:1072F000834206D800232B600124FBF75BF920466C
:10730000F8BD1B1A2B602046FFF7D2FF0024F4E7DC
:107310000024F2E70124F0E7900500104C0500106E
:10732000014B01221A60704794050010014B186848
:10733000704700BF6C040010054B1B6833B1054B50
:107340001B680BB100207047022070470120704776
:107350006405001010050010002850D038B5044610
:10736000C26A28490968C96A8A423ED281690029ED
:1073700005DB24490968C96AC1F1070181616069B7
:1073800002EB82029100204A0A44904205D01D4A35
:107390001268D26AE262012038BD251D2846FFF737
:1073A00018F868B9E36A03EB83018A0016498A5822
:1073B00032B901229A4015490B6823EA02030B6097
:1073C000104B1B68DB6AE362012404FA03F20F49E5
:1073D000086802430A6003EB83039A0029460A48BF
:1073E0001044FEF7D0FF2046D6E7826C054B1B68A1
:1073F000DB6A9A4201D20120CEE70020CCE70020D0
:10740000704700BF6C0400107804001018050010CD
:10741000002834D038B50446C26C013AC264C06A50
:10742000A16C88422DD00AB1002038BD251D284608
:10743000FEF7CFFF68B9E36A03EB83018A001249C4
:107440008A5832B901229A4010490B6823EA020394
:107450000B60A36CE362C3F10702A261012404FA8A
:1074600003F20A49086802430A6003EB83039A00A7
:10747000294605481044FEF786FF2046D5E7002040
:1074800070470020D1E700BF7804001018050010F5
:1074900000283ED038B50446826C8A4200D20A46A3
:1074A000E16A914202D0E06C012800D038BDE2626E
:1074B000A069002802DBC2F10702A261636901EB47
:1074C00081018800134A02449342EFD1251D2846CA
:1074D000FEF77FFF68B9E36A03EB83018A000D4979
:1074E0008A5832B901229A400B490B6823EA0203F9
:1074F0000B60E36A01229A400749086802430A6068
:1075000003EB83039A00294602481044FEF73BFF31
:10751000CCE770477804001018050010044A13687F
:1075200098691368DB6A1268C3F1070393617047B7
:107530006C040010054B1B6823B1044B1A68D36C14
:107540000133D364014B1868704700BF6C0400100E
:1075500038B505460C46FBF71DF8194B1B681B6D2B
:107560002BB9174B1B68012283F85420ACB9FBF7E9
:1075700021F8FBF70FF8124B1B681C6D24B1CDB935
:107580000F4B1B68621E1A650D4B1B68002283F8A7
:107590005420FBF70FF8204638BD11462046FFF770
:1075A000B3FB084B4FF080521A60BFF34F8FBFF30D
:1075B0006F8FDCE7024B1B6800221A65E4E700BF0F
:1075C0006C04001004ED00E0F8B5EFF311854FF006
:1075D000280383F31188BFF36F8FBFF34F8F90F8A9
:1075E0005430DBB2022280F85420026D0132026571
:1075F000012B02D085F31188F8BD0E460446154BC9
:107600001B68E3B9071D3846FEF7E3FEE36A012273
:107610009A401149086802430A6003EB83039A0009
:1076200039460E481044FEF7AEFEE26A0C4B1B686A
:10763000DB6A9A42DED946B101233360DAE700F112
:1076400018010848FEF79FFEEFE7074B01221A607A
:10765000D0E700BF100500101805001078040010D6
:107660006C0400105005001094050010064B1A68B9
:107670001368B3FA83F35B09036013B9D36818681E
:1076800070470020704700BF9805001008B54160A2
:10769000006191420CD8D21A83699A4201D3012029
:1076A00010E0011D094B1868FEF779FE002009E083
:1076B0009A4201D2994206D2011D054B1868FEF785
:1076C0006EFE002008BD0120FCE700BF9C050010F5
:1076D0009805001038B5FAF75DFF0F4B1B6813B122
:1076E000FAF768FF38BD0D4D2846FEF73EFE0C4CFC
:1076F0002046FEF73AFE0B4B1D600B4B1C60002230
:107700000C210520FEF76BFF034B18600028E7D023
:107710000649FFF781F9E3E7CC050010A00500104A
:10772000B4050010980500109C05001040110100E0
:1077300000B583B0FFF7CEFF094B1B686BB1094B57
:1077400001930623009300234FF4967206490748DD
:10775000FFF726FB03B05DF804FB0020FAE700BF4B
:10776000CC050010D005001048110100D1790000AF
:1077700030B585B0134C25680DB31C4601910292BB
:107780000390052913DCFFF7D7FD022807D000235B
:107790001A4601A90B480068FEF746FF0DE00023DA
:1077A000089A01A907480068FEF73EFF05E000239C
:1077B000224601A92846FEF7C3FF05B030BD0020D0
:1077C000FBE700BFCC05001070B582B0154B1B68FD
:1077D0001A6802B3DB681E68DC68251D2846FEF7C0
:1077E000F8FD636A20469847E369012BEED1A3694F
:1077F00033449E4207D2636024612946094B1868CE
:10780000FEF7CDFDE2E7002100910B46324620460F
:10781000FFF7AEFFDAE7044A106802490860136018
:1078200002B070BD980500109C05001038B50546E3
:10783000FFF728FB0446074B1B68834205D800234B
:107840002B60044B1C60204638BDFFF7BDFF0123B1
:107850002B60F6E7C805001070B582B005460E46ED
:107860000F4B1B68DB68DC68201DFEF7B2FDE36987
:10787000012B04D0636A2046984702B070BDA1690D
:107880002B46324629442046FFF700FF0028F1D05E
:10789000002100910B462A462046FFF769FFE9E7E1
:1078A0009805001070B582B006460C46FFF7E2FA64
:1078B00001A8FFF7BBFF019B1BBB05460CB9B042FB
:1078C00018D22CB1114B1B681C68B4FA84F46409FB
:1078D0002246711B0E4B1868FFF7D0F8FFF758FBD4
:1078E00088B90C4B4FF080521A60BFF34F8FBFF333
:1078F0006F8F08E0FFF74CFB29463046FFF7ACFFDF
:1079000001E0FFF745FB02B070BD00BF9C05001011
:10791000CC05001004ED00E030B587B0002203A9CB
:107920002A4B1868FEF744FF00284CD0039B002B1D
:10793000F4DB059C636913B1201DFEF74AFD02A824
:10794000FFF774FF039B092BE8D801A252F823F03C
:107950007979000079790000797900001D790000BB
:10796000AD790000BF7900007979000079790000D5
:107970001D790000AD7900000499A5690B46024607
:1079800029442046FFF782FE0028C7D0636A2046BC
:107990009847E369012BC1D1A269002100910B46F0
:1079A000049802442046FFF7E3FEB7E70499A1617B
:1079B0000346024601442046FFF768FEAEE7204634
:1079C000FAF730FDAAE707B030BD00BFCC050010C4
:1079D00000B583B001A8FFF749FE0199FFF762FFE8
:1079E000FFF79AFFF6E7F8B51746446B866A002062
:1079F00005460BE0192003F0A3F9002006E032460B
:107A000004F13C01206805F025FE0544BD420CDA76
:107A10000644226CA36CE16C5B1AD21A1F2AE9DDC2
:107A20007B1B9342EBDB1346E9E7D4E906235019AD
:107A300043EBE571C4E906010020F8BD08B501F08B
:107A400069FA124B5B6913F0200F1CD0002000F084
:107A50004BFF32210E4B1868FEF730FF0028F0D0A4
:107A600001F084F800231A46194609480068FEF719
:107A7000DBFD00F0C1FE022000F036FF4FF4FA708B
:107A8000FFF7F8FADDE70120E1E700BF00C00920B9
:107A9000D405001008B503F0DFFD03F06FFB01F023
:107AA0006BFA08BD70B506464FF0804005F038FE11
:107AB0004FF0804401252561002003F0B5FF8008C8
:107AC00006FB00F66660236843F0030323600C2185
:107AD000204605F034FE23682B432360AA23A360CD
:107AE0005523A360034BC3F880511D60024B1D70EA
:107AF00070BD00BF00E100E06C42001010B586B020
:107B00000A23039302248DF81140030A43EA002359
:107B1000ADF81230062201212046FCF70DF9B0F134
:107B2000FF3F15D00446082204A9FCF7B0F988B934
:107B300004212046FCF794FC70B90423009303ABA6
:107B4000002211462046FCF7EEFD204606B010BD8F
:107B50000024FAE70024F8E70024F6E770B50646AB
:107B60000D461446BCB10023224629463046FCF798
:107B7000EEFB002811DB10B1844201DC002070BD57
:107B80000544241A064B4FF080521A60BFF34F8F02
:107B9000BFF36F8FE6E72046F1E74FF0FF30EEE7E7
:107BA00004ED00E02DE9F04F83B000AF8146C2B094
:107BB000C7F804D0456BFFF765F93860E8464FF029
:107BC000000B5E4635E04FF0000A04E04FF0010A7A
:107BD00001E04FF0000ABAF1000F03D000247B68E7
:107BE0009C550AE0FFF74EF93B68C01AFF2EF5DC02
:107BF0000128F3D8A0441CE00134022C09DCA31DA9
:107C000059F823000028F7D032467968FFF7A6FF1D
:107C1000F2E7BAF1000F01D1FF2E29DD0BF1010BC4
:107C2000BBF1040F24DCFFF72DF93860D7F804808E
:107C30000026294651F8280BC6F58073424605F008
:107C400039FD0446D5E90423101843EBE471C5E976
:107C5000040136190CD00023A342BADA95F8582053
:107C6000012AB0D118F803200A2AAFD00133F3E774
:107C70000C37BD46BDE8F08F38B505460C460846C2
:107C800007F083FF024621462846FFF767FF38BD0D
:107C90002DE9F04188B006460C46456B8B1D50F827
:107CA000238002F007F8074690B904F1080305EBBA
:107CB00083035B6883B1083405EB84046268023295
:107CC0000849684605F0BCFD69464046FFF7D4FF09
:107CD000384608B0BDE8F08104F1080305EB8303E2
:107CE0005E60E8E71812010030B589B08B1D50F8CE
:107CF000235001F04DFA044610B1204609B030BDC2
:107D00000449684605F09CFD69462846FFF7B4FF24
:107D1000F3E700BF0C12010008B54FF4807212495E
:107D2000124805F033FD0123002204E00F49895C6D
:107D30000B44DBB201329B2AF8D90C4A92F8982006
:107D40009B1A5942DBB2C9B258BF4B42DBB292B266
:107D50009A4207D04FF480720021044805F01AFDC2
:107D6000012008BD0020FCE700FC07007806001099
:107D700010B50023104A82F89830012204E00E4921
:107D8000C95C0A44D2B201339B2BF8D90A4C84F85F
:107D900098201D21084600F007FB1D21084600F031
:107DA000E7FA1D21084600F0FFFA4FF480720349FC
:107DB000204600F009FB10BD7806001000FC07000B
:107DC000FEE7FEE7C8B930B583B00C4C0C4B01930D
:107DD000022500950B4B4FF496720B492046FEF797
:107DE000DFFF0A4B01930095094B4FF49672094946
:107DF0002046FEF7D5FF03B030BD70479D810000DF
:107E000064120010140700104012010068120010E4
:107E10007008001048120100FEE7FFFF2DE9F0474F
:107E200007460D464FF48070FAF796FA002870D096
:107E300080464FF48070FAF78FFA814600286AD0A6
:107E40004FF480720021404605F0A4FC4FF480728C
:107E50000021484605F09EFC2C220021384605F002
:107E600099FC2C220021284605F094FC38220021A0
:107E7000894805F08FFC38220021884805F08AFCEB
:107E800038220021864805F085FC382200218548EB
:107E900005F080FC60220021834805F07BFC602215
:107EA0000021824805F076FC30220021804805F050
:107EB00071FCFFF731FF80BB7E4C062221467E48D5
:107EC00005F064FCA11D7D4807F03EFE04F116019B
:107ED0007B4807F039FE04F126017A4807F034FEAA
:107EE00001246D4E4FF0000A304600F802AB76498F
:107EF00007F02AFE86F801A0744BF362C6F82880CA
:107F000037636B4B7363F4B16A4B5B8FDBB1B38444
:107F100020E0FFF781FFFFF77FFF664C06226649EE
:107F2000204605F033FC6549A01D07F00DFE6449AD
:107F300004F1160007F008FE624904F1260007F07C
:107F400003FE0024CDE742F21073534A9384594A4A
:107F500053870024504A537803F00F03554981F8A2
:107F60003830534B4D4E1E604D4959609A604D4A12
:107F7000DA6004221A624FF0010A304600F802ABC0
:107F8000534907F0E1FD86F801A0524BF362C6F8B1
:107F900028903563444B73632CB1464BB3F846309D
:107FA0000BB1B38407E042F211733C4A9384414A17
:107FB000A2F846300024394B5A7802F00F023D4BAC
:107FC00083F8442003F14C02996C374802F06CFEB0
:107FD000334E3046022300F8023B3F4907F0B4FD20
:107FE000012373703B4BF362C6F8289035632F4B27
:107FF000736334B32F4BB3F85220B284284B5A78B2
:1080000002F00F022B4B83F8502003F15802596DF8
:10801000264802F06FFE234E3046032300F8023B51
:108020002E4907F091FD022373702D4BF362C6F8C1
:10803000288037636CB11F4BB3F85E304BB1B3840B
:108040000FE042F21273164A93841A4AA2F8523091
:10805000D4E742F21373134A9384164AA2F85E30AF
:108060000024104B5B7803F00F03124A82F85C3057
:108070007CB102233B62084A3A600A4A7A600122D4
:1080800085F824202B62054B2B60054B6B60BDE807
:10809000F087FFF76DFEECE71006001040070010B8
:1080A000D8070010D805001078070010100800103D
:1080B00048060010780600108C0000106C000010BC
:1080C0005C0000107C00001020120100917C000078
:1080D00028120100E7790000301201003812010077
:1080E000E97C000000B58DB006AC214D0FCD0FC46A
:1080F00095E8030084E8030006A8FAF7BFF9FFF744
:10810000C9FC1C491C48FFF789FE032200210120FD
:10811000FEF765FA194B186020B100231A4619467C
:10812000FEF782FA1648FBF77BFF05901548FBF730
:1081300077FF04901448FBF773FF039000240CAB07
:1081400043F8284D114A009203AA04A905A8FBF799
:10815000F1F80F4B01930223009323464FF49672DC
:108160000C490D48FEF71CFEFEF74CFEFEE700BF73
:10817000501101007008001014070010D405001001
:108180006C0000107C0000105C0000108C000010DF
:1081900060120010381201003D7A00002DE9F04312
:1081A00097B006460A23029390F8243033B94FF073
:1081B0000A08FBF70CFEB06200240DE04FF0000847
:1081C000F7E756F82450A88CFFF798FC6861052261
:1081D000B16AFBF711FE0134336AA342F1DCA9E076
:1081E00056F82400FFF7DEFC0134336AA342F7DCC3
:1081F000A5E00024F9E75948FFF70EFE04F106094F
:1082000055F8290002F0CCFD0522B16A55F8290085
:10821000FBF703FE002345F829300134022C26DC4D
:10822000A31D55F823000028F7D0B16AFBF703FE21
:108230000028F2D0A01D00234FF48072A96A55F8DF
:108240002000FBF7DDFF021ED8DDEB6A2146284641
:1082500098470028D2DB6B78012BDED0404B4FF0E3
:1082600080521A60BFF34F8FBFF36F8FD5E76869F5
:1082700018B1B16AFBF7DFFD38B90137336ABB4289
:1082800055DD56F827500024C8E716AA082342F8FF
:108290000C3D14A96869FBF728FF8146042300936D
:1082A00002AB00221146FCF73EFA0024022C0DDC42
:1082B000A31D55F823300BB10134F7E70522B16A4D
:1082C0004846FBF799FDA31D45F82390022C13DCCB
:1082D000FAF7CEF8B0F5005F16D36B78012B1BD1FF
:1082E0006B78012BC9D01E4B4FF080521A60BFF340
:1082F0004F8FBFF36F8FC0E71A494846FFF7BCFCAA
:10830000484602F04DFDB8E717494846FFF7B4FC70
:10831000484602F045FDB0E7AA1C1346134903A8DE
:1083200005F08EFA03A94846FFF7A6FCD8E796F8B1
:1083300024307BB196F82430002B7FF45AAF4146AD
:10834000B06AFBF781FD0028FFF655AF0028F1D099
:10835000002793E7322002F0F3FCEBE768110100FD
:1083600004ED00E0701101009C110100E811010012
:1083700000B58BB03423059306900791074B1B681B
:10838000074AA2FB03239B09089301A905A8054BF3
:10839000984701980BB05DF804FB00BF9463001090
:1083A000D34D6210F11FFF1F00B58BB03223059330
:1083B0000690079101A905A8024B984701980BB0B8
:1083C0005DF804FBF11FFF1F00B58BB0332305934D
:1083D000069107900892074B1B68074AA2FB0323EC
:1083E0009B09099301A905A8044B984701980BB074
:1083F0005DF804FB94630010D34D6210F11FFF1F62
:1084000010B5044604F040FA18B9204604F084FA86
:1084100010BD204604F050FAFAE7FFFF30B583B0F4
:1084200004460D4600238DF80730B1F1FF3F2CD0F4
:1084300001238B40DBB28DF80630154B1968A14241
:108440000CD04900E03101230DF10702C1F34701CF
:10845000002004F093F9012002F07CFC0C4B1C601E
:108460000C4B1C600C4B1D606100E03101230DF1D1
:108470000602C1F34701002004F080F904460220FF
:1084800002F068FC204603B030BD0023D3E700BFF4
:1084900094000010E04C0010DC4C001010B50446B5
:1084A000A9B9012303FA00F215490B6823EA020374
:1084B0000B60144904F0F0F83CB10B225109012380
:1084C0009340114A42F8213010BD0A22F6E70146D6
:1084D0000E4805F09BF9012303FA04F208490B68E2
:1084E00013430B6054B90A2201239340064AC2F891
:1084F00080300749204604F0CFF8E5E70B22F3E788
:10850000F44C001051C5000000E100E058120100D9
:108510009DC5000008B50020FFF772FF08BDFFFFF2
:1085200038B5084C4FF48075E561322002F008FC44
:10853000A561322002F004FCE561322002F000FC6B
:1085400038BD00BF00C0092008B52E2800DD02306C
:10855000282800DD0730024600280ADB434200F0ED
:10856000070103F0070358BF5942D010FFF756FF29
:1085700008BDC21DF2E7FFFF2DE9F04383B081463D
:10858000884616461D469DF82870012400E00134F7
:10859000052C14DC0095334642464946002004F081
:1085A00019F9854219D0002FF1D1114A136801330E
:1085B000136004EB8403580002F0CCFBE7E70020D3
:1085C0006FB998B90B4A1368013313600023AB42AB
:1085D0000ADA0022F2540133F9E70120F0E780F0D3
:1085E000010003B0BDE8F0830120FAE70020F8E7BE
:1085F000FC4C0010044D0010564B03EB40131B7F46
:10860000032B04D0534B03EB40135B7F03B970473C
:1086100070B588B00E460446FFF796FF18B94E4A6B
:108620001368013313604B4B03EB44135B7F022B46
:1086300077D1484B03EB44131B7F032B04D02B2330
:108640008DF81C3001250DE0142002F083FBF6E7C5
:10865000414A13680133136005EB8503580002F0AB
:1086600079FB0135052D53DC97238DF81D3011233F
:108670008DF81E30032307AA0B21002004F07EF89A
:108680000328E5D1012002F065FB2EB307238DF806
:108690001D3000208DF81E00032307AA0B2104F0D3
:1086A0006DF803281AD10023009302230DF10A026A
:1086B0002B210B20FFF760FFD0B9BDF80A304FF631
:1086C000FF7293421ED01EB103F00302032A19D198
:1086D0002EBBBBB901231CE03346D8E71E4A136802
:1086E0000133136005EB8503580002F033FBB8E754
:1086F000194A13680133136005EB8503580002F033
:1087000029FBAEE72246154903A805F099F8A8E72A
:108710000023CBB9124A13680133136014E001231C
:10872000F7E73F238DF81C3000208DF81D008DF8F1
:108730001E60032307AA0B2104F020F8032803D0AE
:10874000054A136801331360024800EB44100677B2
:1087500008B070BD78420010FC4C00107812010087
:10876000044D001038B50546002404E02946204693
:10877000FFF742FF0134362CF8DD38BD014B186895
:10878000704700BFFC4C0010014B1868704700BFD9
:10879000044D0010014B1888704700BF5849001065
:1087A000014B1868704700BFE84C0010014B188857
:1087B000704700BFE44C001000487047084D00109F
:1087C000034B1B7813B1034B187870470020704798
:1087D0007442001070420010014B1870704700BFC7
:1087E000CC4C0010024B1A68024B1A60704700BF55
:1087F000F84C0010D04C001008B50D4B1B781BB185
:108800000C4B1B78022B00D008BD0B4B1B680B4A8E
:1088100012689B1A782BF7D9094B2022DA61402283
:10882000DA610020FFF79EFF024B01221A70EBE78E
:10883000CC4C001075420010F84C0010D04C0010C9
:1088400000C009202DE9F041FFF7BAFF804600275C
:1088500000263C4600E00134444512DA1D4B03EB90
:1088600044139D8A284608F0A2FB1B4908F044FAED
:108870000146304608F00CFB0646002DEBD00137D0
:10888000E9E7384608F08AFB0146304608F034FA3A
:1088900008F092FB0022114B07F06EFF0022104BF4
:1088A00007F04CFE00220F4B07F0CEFE08F0C2F896
:1088B0000446094908F09CFB00B1074C0021204602
:1088C00008F096FB20B1204608F03AFBBDE8F081A5
:1088D0000020FBE77842001000007A4400003C4092
:1088E00000408F4000001440014B1870704700BFDB
:1088F000F04C001010B5484802680132474B83FB2A
:1089000002139918D317C3EB611303EB8301C3EB75
:10891000C103D31A0360424A1278012A03D0FAB184
:10892000022A5BD010BD3F4A1278012A0AD13E4983
:1089300081FB0321DA17C2EBA10202EB8202510094
:108940008B42EFD1FFF77EFF00220146C0F57A701F
:1089500002F088FB0123334A1370344A1370E1E7B5
:10896000304B1B7813B12C4B00221A60FFF76AFFC3
:10897000294B1B6803BB2E4B10221A60C0F57A737B
:108980002B4A116801FB03F300FB01F0294A82FB2B
:1089900000140444C11782FB03201844DB17002293
:1089A000C1EBE401C3EBE00002F05CFB00231D4AD5
:1089B00013701E4A1370B5E7042B06DD132B04DC7D
:1089C0001B4A1368013B1360D8E7152BD6DD242B17
:1089D000D4DC174A136801331360CFE7114B1B78BF
:1089E000022B02D00C4B00221A600B4B1B68042B8D
:1089F00007D9094B00221A600C4B1A78084B1A70E1
:108A000090E74FF47A720021084602F02BFB054BE9
:108A100002221A7086E700BFD84C0010D3200DD276
:108A2000F04C00109200001067666666930000101C
:108A3000EC4C00108988888808B50D4A936843F08B
:108A4000010393600B48026801320B4981FB02313C
:108A5000D317C3EBE10303EB83039900531A0360BD
:108A60001BB9064A136801331360FFF743FF08BDC3
:108A700000000B40D44C001067666666F84C00108E
:108A800010B582B0002405E01B4B03EB4413022217
:108A90001A770134FFF794FEA0422BDD164B03EB4F
:108AA00044135B7F022BF4D12046FFF74DFD0020DD
:108AB0008DF8040010238DF805308DF8060003238F
:108AC00001AA0B2103F05AFE032803D00B4A1368B6
:108AD00001331360192002F033F9032301AA0B219B
:108AE000002003F04BFE0328CED0044A1368013364
:108AF0001360C9E702B010BD78420010FC4C0010B2
:108B0000F0B583B0B0F1FF3F03D0064601273546EC
:108B100017E0FFF755FE07460026F8E7114A02EB7B
:108B20000512C4F13F0100230093022302EB44022B
:108B3000C9B20B20FFF720FD0134E4B2072CEDD9B8
:108B40000135F319AB420ADD074B03EB45131B7FDD
:108B5000032BF5D02846FFF7F7FC0024EEE7014889
:108B600003B0F0BD5C490010784200102DE9F04FD1
:108B700089B04FF6FF7B4FF0000947F6FF7AA94B0B
:108B80000293CDF80C904C46D7E0A74B03EB44136F
:108B90005A884FF6FF739A421ED16B1CDBB2042D2C
:108BA0001AD81D46A04A02EB441201230093022367
:108BB0001A4416210B20FFF7DFFC0028E5D09A4B62
:108BC00003EB441300225A80032119779A82DA8238
:108BD0005A831A830126D8E7002E40F0AD80934BCC
:108BE0001B782BB1904B03EB44139B8A002B3BD19A
:108BF0000025009502230DF1160203210B20FFF73B
:108C0000BBFCBDF8162042F4C042ADF81620032389
:108C10008DF81C308DF81D20120A8DF81E2007AA31
:108C20000B21284603F0AAFD009502237E4A02EBA1
:108C300044121C210B20FFF79FFC0095022305AA7C
:108C400018210B20FFF798FC50B9BDF8142040F60E
:108C500048539A427ED0744B03EB441301225A7757
:108C600000212046FFF7C8FC6F4D4FEA441808F179
:108C700010062E44002700970223321D09210B20E5
:108C8000FFF77AFC00970223B21D0F210B20FFF79C
:108C900073FC08F118062E4400970223F2181721DE
:108CA0000B20FFF769FC0097022332460A210B20B4
:108CB000FFF762FC4544B5F91820029B9A4200DD9B
:108CC0000292594B03EB44139B8A4B4500D99946BA
:108CD000524500DA92465B4500D29B46524B03EB6D
:108CE00044131B7F33B9504B03EB44139B7F13F0AA
:108CF000010F35D14E4B1B7813B94E4A1268DAB9C1
:108D000033B9494B03EB44135B8813F4006F06D16E
:108D1000454B03EB44139B7F13F0020F2ED0002131
:108D20002046FFF769FC404B03EB441300221A77FF
:108D30009A7F22F003029A770134362C23DC2046F6
:108D4000FFF702FC18B93C4A136801331360002690
:108D5000354627E7344B03EB441302225A777FE76B
:108D600001212046FFF748FC2F4B03EB441301225F
:108D70001A779A7F22F001029A77BBE7039B0133AF
:108D8000DBB20393D8E7039B192B0BD8284B1B7836
:108D900043B9284B1B6843B9284B1B683C33254A11
:108DA000136002E0234B00221A60224B1B681BB1A8
:108DB000224A12689A4214D801210520FFF72EFB9F
:108DC000F8B91D4A13680133136007210520FFF726
:108DD00025FB00283AD1184A136801331360002597
:108DE0006CE00399164804F011FD164B2022DA615D
:108DF0004022DA610020FFF7B5FC0D4B01221A700A
:108E0000DAE7114D0021009102232A464820FFF79E
:108E1000B3FB2A88130A43EA0223C3F30B132B8004
:108E2000D3E700BF0080FFFF7842001074420010BB
:108E300075420010004D0010FC4C0010F84C001062
:108E40008812010000C00920584900102B4D012351
:108E50002A462721002003F091FC322001F070FF08
:108E600004232A462721002003F0E3FC042803D032
:108E7000234A13680133136020490A6890B2030A39
:108E800043EA00231F480380130C1B029BB243EAF2
:108E900012639B080B60A2E7022306AA4821002068
:108EA00003F0C7FC022816D19DF818209DF8193050
:108EB00043EA0223144A22F815300135042D14DC4C
:108EC000A91C0520FFF7AAFA0028E5D10C4A13686F
:108ED00001331360F1E70A4A1368013313600A4B48
:108EE00042F20F7223F81520E7E7084B01221A70AF
:108EF000074B1C6009B0BDE8F08F00BFE84C0010C4
:108F0000FC4C0010E44C0010084D0010744200109E
:108F10007042001010B5FFF703FB4FF4DC62002134
:108F2000114804F037FC002406E04FF0FF312046E2
:108F3000FFF774FA0134E4B2072CF6D90B4C204643
:108F400004F097F83221204604F0ACF8084B4FF0BB
:108F500000521A600120FFF73FFCFFF743FC054B6E
:108F600000221A6010BD00BF7842001000000B40C4
:108F700000E100E0F84C001008B51B4B1A6842F005
:108F800010021A601A6842F020021A601A6842F051
:108F900040021A601A6842F080021A601A6842F4AD
:108FA00080721A601A6842F400721A601022DA6144
:108FB0002022DA614022DA618022DA614FF4007205
:108FC000DA610A4B01221A70002002F0E9F8002051
:108FD00003F014FB0649002003F02AFB0021084699
:108FE000FFF75CFA08BD00BF00C009207542001001
:108FF0008038010010B404460346002001E060B14F
:1090000001331A1B8A4206DA1A78202AF7D8002878
:10901000F6D000221A7010BC70471846F0E730B442
:1090200003460024254602E09DB1012401331A1AAB
:109030008A4209DA1A78202A01D9002CF6D0202A8F
:10904000F2D825B100221A70284630BC704701249E
:10905000ECE71D460124E9E770B505460E461446C7
:1090600006F093FDA04201D2002070BD284606F014
:109070008CFD0446304606F088FD844201D900206C
:10908000F3E7284606F081FD02462946304606F001
:10909000A1FDB0FA80F04009E7E7FFFF2DE9F04FAE
:1090A00083B0074689460023019306F06EFD06282B
:1090B0005ED90023C9F800303C469B461E469A46BE
:1090C00098461EE0C9F800404FF0010829E003224D
:1090D0002D4901A806F07EFD002839D04FF0FF3061
:1090E00040E00BF1010B0322002101A804F052FB28
:1090F0004FF0FF3603E002AA324402F8043C013488
:109100000136E51B384606F040FD854226D223781D
:10911000202B02D8B8F1000FF1D0D9F80030002B85
:10912000D0D02378202B03D8002323704FF0010ADE
:10913000032E20DC23782E2B02D0BAF1000FDAD0D8
:10914000002E1BDD01A806F0B1FC05460028BED0AC
:10915000B5F5807F15D8BAF1000FC2D0BBF1030F6F
:1091600003D1002003B0BDE8F08F4FF0FF30F9E7E6
:109170004FF0FF30F6E74FF0FF30F3E74FF0FF30EE
:10918000F0E74FF0FF30EDE72C120100FFFFFFFF8B
:109190002DE9F04F9FB0063150F82150866A002328
:1091A000B354012A02DD3378FF2B0CD0002A03DDF3
:1091B0003378FF2B00F06085072A0AD00024204670
:1091C0001FB0BDE8F08F7378EC2BEFD14FF0FF3478
:1091D000F5E70522B349304606F0FCFC0446C8B169
:1091E000B14B1B78002B67D00522B049304606F002
:1091F000F1FC0446002840F081804FF47A71AC4BBA
:109200001868FDF75BFB00285CD1AA492846FEF7E9
:1092100033FDD4E7A84FA949384604F011FB3E18A6
:10922000A749304604F00CFB0644A649304604F03A
:1092300007FB0644A449304604F002FB0644A34958
:10924000304604F0FDFA0644A149304604F0F8FA2D
:109250000644A049304604F0F3FA06449E493046DD
:1092600004F0EEFA06449D49304604F0E9FA06445B
:109270009B49304604F0E4FA06449A49304604F02B
:10928000DFFA06449849304604F0DAFA0644974972
:10929000304604F0D5FA06449549304604F0D0FA39
:1092A00006449449304604F0CBFA3218D21B3946B2
:1092B0002846FEF753FC82E78F492846FEF7DCFC80
:1092C00000247CE78D492846FEF7D6FC8C4B2022F3
:1092D000DA614022DA614FF40072DA618022DA61E9
:1092E000FFF7CEFB00231A46194671480068FDF7C8
:1092F0009BF984492846FEF7BFFC60E705228249B6
:10930000304606F067FC044650B305227F493046DC
:1093100006F060FC044650B305227D49304606F055
:1093200059FC044650B305227A49304606F052FCF7
:109330000446002846D178492846FEF79DFC704B2C
:109340002022DA614022DA614FF47A71584B1868B2
:10935000FDF7B4FAE0B957492846FEF78DFC2EE731
:10936000FFF740FA6D492846FEF786FC27E7FFF72E
:1093700033FA6B492846FEF77FFC20E70120FFF710
:109380002BFAFFF72FFA67492846FEF775FC16E718
:109390000120FFF7E7F900231A4619464448006800
:1093A000FDF742F9FA2001F0CBFC554B20229A61DF
:1093B0005D4B02221A70FFF715FA52492846FEF754
:1093C0005BFCFCE605225949304606F003FC0446E6
:1093D00060BB57492846FEF74FFC494B2022DA6113
:1093E0004022DA614FF47A71314B1868FDF766FA62
:1093F00020B930492846FEF73FFCE0E60120FFF7A0
:10940000B1F900231A46194629480068FDF70CF9FE
:10941000FA2001F095FC3A4B40229A61424B00221F
:109420001A7038492846FEF727FCC8E6052241494C
:10943000304606F0CFFB0446D8B105223E493046FF
:1094400006F0C8FB044600B305223C49304606F04E
:10945000C1FB0446002879D139492846FEF70CFCA7
:10946000274B4FF400729A6126492846FEF704FC08
:10947000A5E634492846FEF7FFFB214B80229A617E
:1094800020492846FEF7F8FB99E62F492846FEF7C3
:10949000F3FB1B4B8022DA611A492846FEF7ECFBEE
:1094A0008DE600BFB8120100744200107C15010067
:1094B000D4050010841501009C080010C0120100A2
:1094C000F81201001C1301004C1301007C13010071
:1094D000AC130100DC13010010140100381401006A
:1094E0006014010080140100C0140100F014010098
:1094F000181501004015010060150100A4150100B8
:1095000000C00920BC150100C4150100E8150100C8
:109510000C160100341601003C160100CC150100A8
:10952000F015010014160100754200105C160100D0
:109530006416010088160100A4160100C01601007F
:10954000C816010090160100AC160100052253490F
:10955000304606F03FFB044660B951492846FEF705
:109560008BFB504B4FF40072DA614F492846FEF7EF
:1095700083FB24E605224D49304606F02BFB0446CA
:1095800030BB4B492846FEF777FB464B2022DA6179
:109590004022DA614FF47A71464B1868FDF78EF974
:1095A00020B945492846FEF767FB08E60020FFF78B
:1095B000D9F800231A4619463E480068FDF734F8EA
:1095C0003E4B01221A7038492846FEF755FBF6E556
:1095D000F71C02223A49384606F0FCFA0446F0B974
:1095E00014AA3849304606F003FAFFF7E9F8149A4E
:1095F000904201DD002A04DA33492846FEF73CFB9D
:10960000DDE5324B03EB421302219977304915A86F
:1096100004F016F915A92846FEF72EFBCFE5022225
:109620002C49384606F0D6FA0446F0B914AA2A495D
:10963000304606F0DDF9FFF7C3F8149A904201DDD9
:10964000002A04DA20492846FEF716FBB7E51F4B2F
:1096500003EB421301219977204915A804F0F0F893
:1096600015A92846FEF708FBA9E505221C49304646
:1096700006F0B0FA0446002840F06F8119492846E8
:10968000FEF7FAFA4FF416710A4B1868FDF716F94F
:1096900060BB15492846FEF7EFFA90E5DC1601009D
:1096A000E416010000C00920BC150100F8160100F5
:1096B00000170100D4050010841501007542001048
:1096C000241701002017010028170100784200101C
:1096D000401701005C1701005817010060170100D6
:1096E000741701007C1701009C17010000238DF8FE
:1096F00075308DF87430A046BB4EFFF761F84045D9
:1097000000F3F48000231A461946B8480068FCF7B5
:109710008BFFFFF73FF807F04AFC4FF0765107F058
:1097200093FA8146FFF73CF807F041FCB04907F097
:109730008BFAB04907F03CFB8046FFF737F807F09B
:1097400036FCAD4907F080FA8246FFF735F8074648
:10975000484607F031FC0022A84B06F0EFFECDE9A9
:109760000E01404607F028FC0022A44B06F0E6FE5E
:1097700080468946504607F01FFC00229F4B06F0AA
:10978000DDFE82468B464046494607F07DF980461D
:10979000DDE90E0107F078F981465046594607F099
:1097A00073F9009043464A469549304604F048F81C
:1097B00006443A887B88B988F888B7F808C0CDF89D
:1097C00008C0019000918F49304604F039F80644F2
:1097D000388807F09CF97EA3D3E9002306F0AEFE9B
:1097E000CDE90E01788807F092F979A3D3E9002337
:1097F00006F0A4FE80468946B88807F088F976A36B
:10980000D3E9002306F09AFE82468B46F88807F0DB
:109810007EF971A3D3E9002306F090FECDE9100193
:10982000388907F074F96EA3D3E9002306F086FEA9
:10983000CDE912014046494607F026F98046DDE9A8
:109840000E0107F021F98146DDE9120107F01CF94C
:109850000290DDE9100107F017F9019050465946D2
:1098600007F012F9009043464A466749304603F034
:10987000E7FF06449DF875309DF874206349304633
:1098800003F0DEFF0644624F7A69C2F34012614979
:10989000304603F0D5FF06447A69C2F380125E4970
:1098A000304603F0CDFF06447A69C2F3C0125B492B
:1098B000304603F0C5FF06447A69C2F34022584996
:1098C000304603F0BDFF0644FEF758FF0746FEF79B
:1098D0005BFF03463A465349304603F0B1FF321866
:1098E0004149521A2846FEF739F968E44E4B1B6885
:1098F00015934E494FEA48128F183B7F06F1010934
:109900001EA8034413F8243C33708B5AB7F918206F
:10991000B98AF88A7E8BB7F802C0CDF810C00396DA
:1099200002900191009242464149484603F088FF67
:1099300009EB00067B7F012B07D19DF874300133C2
:109940008DF8743008F10108D7E6022BFAD19DF8A2
:10995000753001338DF87530F4E702223549384609
:1099600006F038F90446002840F0AF8015AA3249C5
:10997000304606F03DF8159B632B12D14FF0FF33B4
:109980001593FEF71DFF8046FEF71AFF159B9842C0
:1099900002DDB3F1FF3F07DA28492846FEF76CF9EC
:1099A0000DE44FF00108EFE725492846FEF764F97A
:1099B0004FF416710D4B1868FCF780FF002843D157
:1099C00020492846FEF758F9FFF7F9BBAFF30080AE
:1099D00049F59D5F94A0B73F8B8862F20698B93F26
:1099E00030B8E68EFE97C93F9C080010D4050010E1
:1099F0000805253C000020421004C83B000024401C
:109A0000E4170100FC170100201801003C180100B8
:109A100000C009205C1801006818010074180100DA
:109A2000801801008C180100B41201007842001067
:109A3000BC170100B4180100B0180100281701007C
:109A4000B81801009C1701001598FFF759F88146D6
:109A5000159BB3F1FF3F01D100231593159E894F4C
:109A6000159B4344B3420DDC00231A461946864831
:109A70000068FCF7D9FD83497A1A2846FEF76EF88C
:109A8000FFF79DBB330109EB030239F8033051881E
:109A90009088B2F806C0B2F808E0B2F80AA0B2F8AE
:109AA0000CB0D2890692CDF814B0CDF810A0CDF844
:109AB0000CE0CDF808C00190009132467349384659
:109AC00003F0BEFE07440136CAE70522704930465E
:109AD00006F080F80446002840F0D1804FF416715B
:109AE000694B1868FCF7EAFE002840F0B980694924
:109AF0002846FEF7C1F8FFF762BB674B03EB46133E
:109B0000988A584500D283460E9B984200D90E9001
:109B1000B8B1824407F04BFA12905F4B03EB461347
:109B2000B3F9180007F03AFA129907F08DF85B497B
:109B300007F0E2F80146109807F0AAF9109009F131
:109B40000109554B03EB4613DB8A03B19844524B92
:109B500003EB4613B3F918301F440136FEF730FE0D
:109B6000B042CADC00231A46194647480068FCF791
:109B70005BFD584607F01BFA494907F0BDF8064659
:109B80000E9807F014FA464907F0B6F80E905046C2
:109B900007F004FA8246484607F000FA814601467B
:109BA000504607F0A9F83E4907F0A6F8834640461C
:109BB00007F0F4F9494607F09FF8394907F09CF897
:109BC0008046384607F0EAF9354907F095F8074628
:109BD000FEF7E6FD07F0EBF9324907F035F83249B8
:109BE00007F0E6F88146FEF7E1FD07F0E0F92F49BE
:109BF00007F02AF88246304607F0DEF9CDE9120177
:109C0000204E504607F0D8F9CDE90C01484607F040
:109C1000D3F9CDE90A01109807F0CEF9CDE9080192
:109C2000384607F0C9F9CDE90601404607F0C4F906
:109C3000CDE90401584607F0BFF9CDE902010E98BD
:109C400007F0BAF9CDE90001DDE9122318493046E1
:109C500003F0F6FD31462846FEF70EF8FFF7AFBADF
:109C6000A046A2462746A14626460023109300237D
:109C70000E934FF6FF7B71E70124FFF7A0BA002493
:109C8000FFF79DBA9C080010D4050010E0180100F1
:109C9000101901009C17010078420010002474493B
:109CA00000007A440805253C000020421004C83B0F
:109CB000181901002DE9F04F95B0466B01F108032A
:109CC00006EB83035D688B1D50F82340836A012AED
:109CD00002DD1F78FF2F41D0002A03DD1F78FF2F00
:109CE00000F0EF8503EB020900279F54002D3CD0C4
:109CF0008B460690083106EB8101496891F8018096
:109D000011461846FFF776F90746002800F0DB8574
:109D100005F03BFF07EB000AA9EB0A090022B54951
:109D20003846FFF799F938BBB8F1000F00F097807B
:109D3000B8F1000F00F0F680B8F1000F40F0A481F8
:109D40000022AD493846FFF787F9002800F09C81D2
:109D5000AA4B00271F709846A1463EE15F78EC2F82
:109D6000BAD14FF0FF3300F0AFBD01F1080506EBAB
:109D7000850568600546BBE7A04EAA1CA049304691
:109D800003F05EFD3518B8F1010F48D0B8F1020FAD
:109D90005FD09C49284603F053FD05449A49284664
:109DA00003F04EFD05449949284603F049FD05445A
:109DB0009749284603F044FD05449649284603F098
:109DC0003FFD05449449284603F03AFD0544934974
:109DD000284603F035FD05449149284603F030FD3F
:109DE00005449049284603F02BFD05448E4928463A
:109DF00003F026FD05448D49284603F021FD054466
:109E00008B49284603F01CFD8A49284403F018FDBD
:109E10007A492046FDF730FF002300F055BD864902
:109E2000284603F00DFD05448449284603F008FD4B
:109E300005448349284603F003FD0544814928462B
:109E400003F0FEFC05448049284603F0F9FC054474
:109E5000D1E77E49284603F0F3FC0544CBE7002216
:109E60007B493846FFF7F8F800283FF461AF4946D0
:109E70005046FFF7D4F8074668B10025336AAB4275
:109E800043DD56F825100231384605F03BFE034607
:109E900090B30135F2E7594D6E49284603F0D0FCE6
:109EA0000544002714E056F827305B78012B19D0C1
:109EB000022B1CD068490EA805F046FE56F8272054
:109EC0000EAB02326549284603F0BAFC054401375F
:109ED000336ABB42E7DC49492046FDF7CDFE00234B
:109EE00000F0F2BC5E490EA805F02EFEE6E75D49E3
:109EF0000EA805F029FEE1E756F825100BF108023F
:109F000006EB8206716000F0DFBC3C4D3A465649D4
:109F1000284603F095FC29462046FDF7ADFE0023B8
:109F200000F0D2BC002251493846FFF795F80028CE
:109F30003FF402AF4E492046FDF79EFEFA2000F0A6
:109F4000FFFE204600F02CFF4A4B1B7843B14FF038
:109F5000804301225A60AA229A6055229A60FEE745
:109F60000020FDF79FFDFAE743490BA805F0ECFD43
:109F70000BAB00930EAB52464049404603F060FCE9
:109F800080440135022D27DC7B1C03EB83035A0040
:109F900002EB050A56F82730AA1D53F82240002C80
:109FA000EFD009A92046FAF778FB0A9A130E01931D
:109FB000C2F307430093C2F30723D2B230490EA87D
:109FC00003F03EFCA145CFD056F8272002322D49A0
:109FD0000BA803F035FCCBE70137336ABB4201DD48
:109FE0000025CFE705494846FDF746FE002300F06F
:109FF0006BBC00BFDC190100981D01009C0800101B
:10A00000E4190100241B0100401B0100681B010032
:10A01000A01B0100D81B0100141C01004C1C0100F6
:10A02000741C0100A01C0100C01C0100E01C010008
:10A03000181D010098170100F8190100281A0100E5
:10A040006C1A0100901A0100D01A0100F81A0100E0
:10A05000381D01003C1D010020120100541D0100AB
:10A060004C1D010038120100601D01007C1D010023
:10A07000841D01006C420010AC1D0100BC1D0100DC
:10A08000A01D0100B41D01000022C1493846FEF7A1
:10A09000E3FF079000284AD1B8F1000F00F0CF800D
:10A0A000B8F1000F00F0FC80B8F1000F00F029813A
:10A0B000B8F1000F00F05681B8F1000F00F0CE812A
:10A0C000B8F1000F07D10022B2493846FEF7C4FFAD
:10A0D000002840F04F82B8F1010F00F06B82B8F118
:10A0E000010F00F07982B8F1010F00F0B682B8F1EB
:10A0F000010F00F03A83B8F1010F00F08783B8F147
:10A10000020F00F0C1830022A3493846FEF7A4FFE6
:10A11000002800F0D0830BF1080306EB8306002330
:10A120007360069B9D4200F0C3830023CCE3494645
:10A130005046FEF774FF804628B998492046FDF73F
:10A140009BFD0023C0E305F0B1FC0746421E4FF61D
:10A15000FE739A420DD8AB8C834216D00022336A2C
:10A1600093422BDD56F82230998CB94219D0013236
:10A17000F5E78B4D42468B49284603F061FB2946A3
:10A180002046FDF779FD00239EE3854D0246864972
:10A19000284603F055FB29462046FDF76DFD0023B8
:10A1A00092E37F4D02333A468049284603F048FB4C
:10A1B00029462046FDF760FD002385E3784E3A46A8
:10A1C0007B49304603F03CFB31462046FDF754FD09
:10A1D0000024022C12DCA31D55F8230060B100F00E
:10A1E000DFFD2B6BA61D0522996A55F82600F9F7AD
:10A1F00014FE002345F826300134EAE7642000F01D
:10A200009FFD686900F0CCFD2B6B0522996A686997
:10A21000F9F703FEBFB2AF843846FDF76FFC686103
:10A220002B6B0522996AF9F7E7FD2B78614A0C211F
:10A2300001FB03235F87FDF79BFD002344E300221E
:10A240005D493846FEF708FF00283FF429AF002398
:10A250000E9349465046FEF7E2FE28B94F49204684
:10A26000FDF70AFD00232FE30EA9FEF717FFB0F15B
:10A27000FF3F04D151492046FDF7FEFCF2E70E995D
:10A280004F4805F061FCFDF773FD454D0E9A4D49B1
:10A29000284603F0D5FA29462046FDF7EDFCE1E714
:10A2A000002249493846FEF7D7FE00283FF4FCAEAD
:10A2B00000230E9349465046FEF7B1FE28B93749B0
:10A2C0002046FDF7D9FC0023FEE20EA9FEF7E6FECC
:10A2D000B0F1FF3F04D139492046FDF7CDFCF2E74C
:10A2E0000E993A4805F030FCFDF742FD2C4D0E9AD0
:10A2F0003749284603F0A4FA29462046FDF7BCFC5E
:10A30000E1E7002233493846FEF7A6FE00283FF475
:10A31000CFAE00230E9349465046FEF780FE28B983
:10A320001E492046FDF7A8FC0023CDE20EA9FEF74A
:10A33000B5FEB0F1FF3F04D127492046FDF79CFC54
:10A34000F2E70E99254805F0FFFBFDF711FD144DCE
:10A350000E9A2349284603F073FA29462046FDF752
:10A360008BFCE1E700221F493846FEF775FE059099
:10A3700000283FF4A1AE49465046FEF750FE06467F
:10A3800090BB06492046FDF777FC00239CE200BF06
:10A39000CC1D01006020010064220100D41D0100D9
:10A3A0009C080010EC1D0100041E0100281E010085
:10A3B000501E010078060010841E0100881E010056
:10A3C0007E060010A41E0100D01E01008E060010A3
:10A3D000D41E0100041F0100081F01009E0600108A
:10A3E000201F0100481F010005F0CFFB112804D0F9
:10A3F000A4492046FDF740FCC7E70025052D17DCE2
:10A4000005EB4500831CF25C042D03DC2D2A01D0F2
:10A410003A2A0FD10021F1541022304405F008FBF4
:10A42000FF2807D814AB2B4403F8180C0135E5E7D7
:10A43000079B0593059B002BDAD106220EA99248B3
:10A4400003F0A4F9FDF794FC904D9149284603F0E0
:10A45000F7F929462046FDF70FFC96E700228D49C3
:10A460003846FEF7F9FD00283FF42AAE874EAA8C45
:10A470008949304603F0E4F93518884E3246884958
:10A48000284603F0DDF905443146864805F03AFBDD
:10A49000002858D0834A8449284603F0D1F905445E
:10A4A000824E32468249284603F0CAF905443146B5
:10A4B000804805F027FB00284BD07E4A7A49284681
:10A4C00003F0BEF905447C4E32467C49284603F031
:10A4D000B7F9054431467A4805F014FB00283ED010
:10A4E000774A7149284603F0ABF90544754E327836
:10A4F0007378B178F078377996F805C0CDF80CC04C
:10A500000297019000917049284603F099F905449B
:10A51000062231465C4803F0BDFE30B35A490A7842
:10A520004B788878CE780F79497903910297019614
:10A5300000906649284603F083F954492046FDF708
:10A540009BFB0023C0E16249284603F079F90544EA
:10A55000A6E75F49284603F073F90544B3E75C4971
:10A56000284603F06DF90544C0E75949284603F031
:10A5700067F9E2E7454D574A5749284603F060F925
:10A58000054404225549564B186805F023FB60B971
:10A59000534B1A6804325349284603F051F93B499A
:10A5A0002046FDF769FB00238EE14F49284603F062
:10A5B00047F9F4E702224D493846FEF74DFD0028E1
:10A5C0003FF48DAD6D6B4A492046FDF755FB287968
:10A5D00000F02AFA002377E1022246493846FEF7C6
:10A5E0003BFD00283FF47FAD49465046FEF717FD7E
:10A5F000074628B940492046FDF73EFB002363E1AA
:10A6000005F054FA061E0ADC3A463C491F4803F09E
:10A6100017F91E492046FDF72FFB002354E1686B14
:10A6200000220092194B314600F032FA0028F0D196
:10A6300032463349154803F003F92B7812490C22AE
:10A6400002FB0312D26BB242E3D00A460C2101FB9B
:10A650000323DE63FDF78CFBDBE700222949384644
:10A66000FEF7FAFC00283FF442AD49465046FEF79B
:10A67000D6FC0646002847D11F492046FDF7FCFAC4
:10A68000002321E14C1F0100780600109C080010F7
:10A69000841F0100B01F0100B81F01006C000010F2
:10A6A000CC1F01007E060010E01F01007C0000109E
:10A6B000E81F01009E0600105C000010FC1F010056
:10A6C0008E0600108C000010102001003C200100BC
:10A6D0009817010050120100682001007C20010041
:10A6E000980000108420010098200100AC20010097
:10A6F000B4200100C8200100D41D0100D0200100B9
:10A700000821010024210100686B00230093704B95
:10A7100032464FF0FF3100F0BBF900BB327873785E
:10A72000B17800916B496A4803F08AF82A780C23C3
:10A7300003FB02F34033032231466748184405F017
:10A7400049FA60B12A780C2303FB02F34033032259
:10A7500031466148184405F068FAFDF709FB5C4989
:10A760002046FDF789FA0023AEE000225B49384617
:10A77000FEF772FC00283FF4BEAC6E6B49465046B3
:10A78000FEF74DFC074628B955492046FDF774FAF7
:10A79000002399E005F0F9F9012805D83A78A2F1EB
:10A7A0003003DBB2012B0AD93A464E49484803F040
:10A7B00047F847492046FDF75FFA002384E04A49FD
:10A7C000434803F03DF83B78302B10D12B78424AB8
:10A7D0000C2101FB032393F8382022F0100283F8A8
:10A7E0003820002386F85830FDF7C2FAE1E72B78CD
:10A7F000394A0C2101FB032393F8382042F0100260
:10A8000083F83820012386F85830EDE700223749D5
:10A810003846FEF721FC00283FF471AC6F6B2C4EDC
:10A82000AA8C3349304603F00BF8351807F10C03B6
:10A83000BA683049284603F003F8054497F85830C1
:10A84000E3B92D49284602F0FBFF0544D7E906236A
:10A850002A49284602F0F4FF0544D7E90423284991
:10A86000284602F0EDFF3A6A2649284402F0E8FF44
:10A8700017492046FDF700FA002325E02249284623
:10A8800002F0DEFF0544E1E7002218493846FEF7F2
:10A89000E3FB00283FF437AC0D4EAA8C1B49304631
:10A8A00002F0CEFF31462046FDF7E6F900230BE02B
:10A8B0004FF0FF3308E016492046FDF7DDF900238D
:10A8C00002E0012300E00023184615B0BDE8F08F38
:10A8D0009C0800102C21010078060010482101007E
:10A8E000D41D0100502101007C210100B01F010096
:10A8F0009C210100B4210100D021010004220100AB
:10A900001C22010034220100E82101004C22010038
:10A910006C22010008B5034A034B1A6000F0CDFC1D
:10A9200008BD00BF0020000008ED00E010B504469F
:10A93000006802F0CDFD236881229A60206802F051
:10A9400003FE4FF400630122216D04F1280002F0A0
:10A95000D8F94FF400730122616D04F13C0002F05C
:10A96000D0F92368C7229A602268536843F0050330
:10A97000536094F90530002B11DB03F1604303F5BC
:10A980006143082283F8002394F9053003F01F0186
:10A990005B0901228A40054941F8232010BD03F0DC
:10A9A0000F03034A1A4408231376EDE700E100E0A1
:10A9B000FCEC00E030B585B00446C36A426B816BA5
:10A9C000521A9B1A03EB83035A0002F2FF7240F6FD
:10A9D000FE739A420ED8056ACC3508E0102269460B
:10A9E00004F1280002F097FA236A18442062236ACF
:10A9F000AB42F3D304F13C0204F12801206802F0D9
:10AA00006AFE05B030BDFFFF08B50248FFF7D2FF70
:10AA100008BD00BF7807001008B50248FFF7CAFF5D
:10AA200008BD00BF100800102DE9F04383B018B135
:10AA3000032826D1192600E00226DFF850800025E1
:10AA40000095082332462946404601F0FCFF0E4C93
:10AA500023684FF0010909FA06F73B432360E369D5
:10AA60003B43E36140F2DC5000F06AF9A3693B43E9
:10AA7000A361CDF80090082332462946404601F0F4
:10AA8000E2FF03B0BDE8F08300C0092000C002402F
:10AA90002DE9F04782B0074615469A469DF8288072
:10AAA0000023ADF8063038238DF804304E238DF89E
:10AAB000053031238DF806300E1E19DDB6F5965F90
:10AAC00025D01BDDB6F5964F21D037DDB6F5614FA9
:10AAD0001DD0B6F5E13F1AD0B6F5164F17D0B8F134
:10AAE000000F32D04FF41653BB604FF0000911E055
:10AAF000B8F1000FE2D14FF000090BE0B6F5167F78
:10AB000005D014DC6E2E02D0B6F5967FE7D1BE607C
:10AB10004FF0000925B30024284605F036F8A0427E
:10AB200025D92A192B5D202B1FD90134F4E7B6F55E
:10AB3000966FECD0B6F5166FD1D1E8E7B6F5165F93
:10AB4000E5D0B6F5615FCAD1E1E75249504602F05F
:10AB500077FE504605F019F882444FF00109D9E715
:10AB6000B8F1000F33D100245CE0002313702846B5
:10AB700005F00BF8022803D8B8F1000F29D001AD79
:10AB80002A78A2F13004E4B2A2F13503DBB2032B40
:10AB900026D83A73053C6B78453B2A2B5FD8DFE813
:10ABA00003F0545E5E5E5E5E5E5E5E2F595E5E5ECC
:10ABB0005E5E5E5E5E5E5E5E5E5E5E5E5E5E5E5EB5
:10ABC0005E5E545E5E5E5E5E5E5E5E2F59000024D9
:10ABD000A2E73149504602F033FE4FF0010930E060
:10ABE000B8F1000F03D038233B730324D3E72B497C
:10ABF000504602F025FE824400244FF00109CAE7C6
:10AC00004E237B73AA78A2F13103DBB2012B34D936
:10AC1000B8F1000F33D03123BB73BB7B322B01D192
:10AC200044F00404B9F1000F0BD1002E02DCB8F19E
:10AC3000000F03D0B968386802F09EFC35B33B685A
:10AC4000DC60484602B0BDE8F08745237B7344F0E2
:10AC50001804D7E74F237B7344F00804D2E7B8F118
:10AC6000000F02D04E237B73CCE70D49504602F013
:10AC7000E7FD82444FF00109C4E7BA73CDE7094903
:10AC8000504602F0DDFD4FF00109C6E7B8F1000FB4
:10AC9000D5D1D6E778220100F02201001823010067
:10ACA0005023010080230100F0B583B004460E4616
:10ACB00017466022002102F06DFD052363710A4BE7
:10ACC000236000252571094B2365094B63652046E8
:10ACD000FFF72CFE012300932B463A4631462046CF
:10ACE000FFF7D6FE03B0F0BD00C00040144D0010C9
:10ACF000145D001070B582B004460D461646602201
:10AD0000002102F047FD082363710A4B23600323EF
:10AD10002371094B2365094B63652046FFF706FE47
:10AD2000012300930023324629462046FFF7B0FE58
:10AD300002B070BD00C0094014550010145F00102F
:10AD400008B5034BA3FB0030C008FCF793F908BD1E
:10AD5000CDCCCCCC82B04FF47A7303FB00F00090E2
:10AD60000D4B1A680D4BA3FB0232D20C009B4BB962
:10AD7000009B0133009305E0019B01330193019B8C
:10AD80009A42F9D8009B013B009313B10023019331
:10AD9000F5E702B0704700BF94630010819F5E1614
:10ADA00030B591B005460221F9F7A6FB0024002337
:10ADB000402269462846F9F723FA002808DB0220DA
:10ADC000FCF758F9631CDBB2182C01D81C46EEE7DF
:10ADD0002846F9F7CFF811B030BD80B582B000AF8A
:10ADE00078600F2000F02CFD00BF0837BD4680BD05
:10ADF00080B483B000AF78600B46FB701346BB7025
:10AE0000FA787B681A3253F82210BB78012202FAD2
:10AE100003F3FA7819437B681A3243F8221000BF13
:10AE20000C37BD4680BC704780B483B000AF7860FB
:10AE30000B46FB70FA787B68DA6700BF0C37BD46BB
:10AE400080BC704780B582B000AF78600F2000F002
:10AE5000F7FC00BF0837BD4680BD80B483B000AFAB
:10AE600078600B46FB70FA787B681A6000BF0C377D
:10AE7000BD4680BC704780B483B000AF78607B680B
:10AE80001B68DBB218460C37BD4680BC704780B4E7
:10AE900083B000AF786039607B683A68DA6000BFE1
:10AEA0000C37BD4680BC704780B483B000AF78607B
:10AEB0007B685B6918460C37BD4680BC704780B420
:10AEC00083B000AF78607B685B6843F001027B6809
:10AED0005A607B685B6843F008027B685A6000BF79
:10AEE0000C37BD4680BC704780B485B000AFF860B9
:10AEF0000B467A60FB7297F90B30062B2CD801A217
:10AF000052F823F021AF000029AF000031AF00005C
:10AF100039AF000041AF000049AF000051AF000061
:10AF2000FB687A689A6118E0FB687A68DA6114E075
:10AF3000FB687A681A6210E0FB687A685A620CE073
:10AF4000FB687A681A6408E0FB687A685A6404E06F
:10AF5000FB687A689A6400E000BF00BF1437BD4602
:10AF600080BC704780B586B000AFF860B9607A6089
:10AF700000237B6109E0BA687B6913441B7818469B
:10AF800000F0CCF87B6901337B617B687A699A4277
:10AF9000F1D37B6818461837BD4680BD80B582B0B6
:10AFA00000AF00F0D5F80346FB71FB79184608376F
:10AFB000BD4680BD80B582B002AF012300930C2353
:10AFC00002220221254801F03EFD012300930C23BB
:10AFD00003220221214801F036FD012300930C23B6
:10AFE000042202211D4801F02EFD1D4801F0B0FD94
:10AFF0001B4801F0BCFD012300220521184801F087
:10B00000D1FD012300220321154801F0CBFD0123CE
:10B0100000220421124801F0C5FD4FF47A7200218C
:10B020000F48FFF761FF002205210D48FFF75CFF85
:10B03000002203210A48FFF757FF00220421084895
:10B04000FFF752FF01220021054801F0F0FD0448FE
:10B05000FFF735FF00BFBD4680BD00BF00C0024006
:10B060000080014080B584B000AFF860B9607A60BC
:10B07000BA681346DB009B1A154A82FB0312921032
:10B08000DB17D31ABB60FB681A4605211148FFF78E
:10B090002BFFBB681A4603210E48FFF725FF7B688C
:10B0A0001A4604210B48FFF71FFF0122052109481A
:10B0B00001F0BDFD01220321064801F0B8FD012287
:10B0C0000421044801F0B3FD00BF1037BD4680BD28
:10B0D000676666660080014080B483B000AF786028
:10B0E00000BF0C37BD4680BC7047FFFF80B500AF86
:10B0F0000948FFF7F1FF084802F0EAF94FF4E1319F
:10B10000054802F039FA03210348FFF7C0FE024860
:10B1100002F01AFA00BF80BD00C0094080B582B0BD
:10B1200000AF0346FB7100BF0848FFF7BDFE0346B2
:10B1300003F02003002BF7D0FB7919460348FFF7F3
:10B140008CFE00BF0837BD4680BD00BF00C009406F
:10B1500080B500AF0848FFF7A7FE034603F00103E0
:10B16000002B04D00448FFF786FE034601E04FF0B1
:10B17000FF33184680BD00BF00C0094080B500AF56
:10B18000FFF7B4FF0448FFF75DFE0448FFF725FE14
:10B19000FFF710FF00BF80BD00C0092000C00240C3
:10B1A00080B584B002AF0346FB71FB79012B19D047
:10B1B000022B32D0002B00D04AE001230093082359
:10B1C0001B220021244801F03EFC012300930823A8
:10B1D0001C220021204801F036FC00211E48FFF708
:10B1E00023FE35E0022300930823132200211A488E
:10B1F00001F029FC022300930823142200211648A1
:10B2000001F021FC132200211348FFF7F1FD142265
:10B2100000211148FFF7ECFD1AE0022300930823F8
:10B220000A2200210C4801F00EFC0223009308239F
:10B230000B220021084801F006FC0A2200210648E2
:10B24000FFF7D6FD0B2200210348FFF7D1FD00BF19
:10B2500000BF0837BD4680BD00C0024080B485B045
:10B2600000AF0346FB71084B1B68C3F30B03FB6085
:10B27000FB791B031946044AFB680B43136000BFAC
:10B280001437BD4680BC704700C00F4080B500AF8A
:10B2900011220349034801F020FC00BF80BD00BF1C
:10B2A000C023010000C0024080B500AF01F082FF62
:10B2B0000420FFF7D3FF00BF80BD80B500AFFFF7CC
:10B2C000E5FFFFF7F1FF00BF80BD80B483B000AFA2
:10B2D00078607B685B6B03F00103002B14BF0123D4
:10B2E0000023DBB218460C37BD4680BC7047FFFF19
:10B2F00080B584B000AF03460A46FB711346BB809D
:10B300000023FB73FA23BB60BA88FB7919464FF020
:10B31000A04000F059FC12E04FF0A040FFF7D5FF2D
:10B320000346002B07D0BB68013BBB60084B1B6882
:10B330000120984703E00023BB600123FB73BB6837
:10B34000002BE9DCFB7B18461037BD4680BD00BFF3
:10B350002061001080B584B000AF03463960FB71F6
:10B360000023FB73FA23BB60FB7919464FF0A04022
:10B3700000F048FC1DE04FF0A040FFF7A6FF034699
:10B3800083F00103DBB2002B0CD00023BB604FF035
:10B39000A04000F04FFC03461A463B681A80012388
:10B3A000FB7306E0BB68013BBB60064B1B680120DA
:10B3B0009847BB68002BDEDCFB7B18461037BD4688
:10B3C00080BD00BF2061001080B483B000AF034691
:10B3D0000A46FB801346BB80FB8803F00403002B66
:10B3E00006D0314B1B6843F008032F4A136005E079
:10B3F0002D4B1B6823F008032B4A1360BB8803F016
:10B400001C03082B1DD0142B0ED0042B26D0264B4A
:10B410001B6843F01003244A1360234B1B6843F05E
:10B420002003214A136026E01F4B1B6823F0100302
:10B430001D4A13601C4B1B6843F020031A4A13601B
:10B4400019E0194B1B6843F01003174A1360164BA1
:10B450001B6823F02003144A13600CE0124B1B6896
:10B4600023F01003104A13600F4B1B6823F02003D6
:10B470000D4A136000BF0C4B1A680C4B1B685340FD
:10B4800003F03803002B09D0074B1B68074A1360F1
:10B49000054B1B6843F00403034A136000BF0C37DD
:10B4A000BD4680BC704700BF1461001018610010D9
:10B4B00080B586B000AFB9607A603B600346FB732D
:10B4C00000237B822E4ABB6813602E4B00221A6039
:10B4D0002D4B00221A602C4B1B682C4A13604FF432
:10B4E00000410020FFF704FF0346012B01D0002399
:10B4F00041E04FF4C8737B611AE0214B1B680120C7
:10B50000984707F1100319460020FFF723FF034671
:10B51000012B01D000232EE03B8A03F40843002BCB
:10B5200003D14FF0FF337B6102E07B69013B7B611C
:10B530007B69002BE1DC7B69002B01D100231AE041
:10B540007B68642B03D17B8A43F400537B827B6846
:10B55000002B03D17B8A43F490537B823B68002B02
:10B5600003D07B8A43F480737B827B8A1946002058
:10B57000FFF7BEFE012318461837BD4680BD00BF49
:10B58000206100101C61001014610010186100108F
:10B5900098B500AF2D4B1B68012B16D0022B2FD076
:10B5A00001214FF0A04000F02DFB294B1B6823F038
:10B5B0000403274A1360264B1B6843F00203244A06
:10B5C0001360224B01221A603CE04FF0A040FFF7CD
:10B5D0007CFE034683F00103DBB2002B2FD04FF03B
:10B5E000A04000F027FB03461A461A4B1A801F2181
:10B5F0004FF0A04000F006FB144B02221A601EE040
:10B600004FF0A040FFF761FE034683F00103DBB279
:10B61000002B16D00E4B1B6823F002030C4A13605C
:10B620000C4B1C884FF0A04000F004FB0346194669
:10B630002046FFF7C9FE054B00221A6001E000BF5B
:10B6400000E000BF024B1B68184698BD1C6100104B
:10B65000146100102461001080B500AF00F0D8F92B
:10B660000246024B1A6000BF80BD00BF9463001009
:10B6700080B400AF064BD3F8883003F08073002B02
:10B6800014BF01230023DBB21846BD4680BC7047BF
:10B6900000C00F4080B400AF064BD3F8883003F0F1
:10B6A0000073002B14BF01230023DBB21846BD46F4
:10B6B00080BC704700C00F4080B483B000AF034629
:10B6C000FB71094AFB795B0113448C33AA221A608F
:10B6D000054AFB795B0113448C3355221A6000BF85
:10B6E0000C37BD4680BC704700C00F4080B400AF2F
:10B6F000054BD3F80C31DBB203F00303DBB2184681
:10B70000BD4680BC704700BF00C00F4080B400AF92
:10B71000024B1B681846BD4680BC7047B823010029
:10B7200080B400AF024B1846BD4680BC704700BFD6
:10B7300000093D0080B400AF024B1B681846BD46AF
:10B7400080BC7047BC23010080B500AF00F008F951
:10B750000346184680BDFFFF80B584B000AF0346A6
:10B760003960FB710C4AFB7904335B0113441B689D
:10B77000FB60FA683B681343FB60074AFB790433BC
:10B780005B011344FA681A60FB791846FFF794FFCF
:10B7900000BF1037BD4680BD00C00F4080B584B0EB
:10B7A00000AF03463960FB710D4AFB7904335B013E
:10B7B00013441B68FB603B68DB43FA681340FB6083
:10B7C000074AFB7904335B011344FA681A60FB797A
:10B7D0001846FFF771FF00BF1037BD4680BD00BFA0
:10B7E00000C00F4080B586B000AF0346B9607A60F4
:10B7F000FB73FB7B002B05D17B681B04BA681343EA
:10B800007B6104E07B685B01BA6813437B610B4A90
:10B81000FB7B04335B01134404337A691A60074AE3
:10B82000FB7B04335B01134401221A60FB7B184647
:10B83000FFF742FF00BF1837BD4680BD00C00F4074
:10B8400080B485B000AF0346FB71FB79FB60084B09
:10B85000D3F8C4300121FA6801FA02F21146044A11
:10B860000B43C2F8C43000BF1437BD4680BC7047DC
:10B8700000C00F4080B582B000AFFFF70BFF03465A
:10B88000002B02D00123FB7101E00023FB71FB7947
:10B8900018460837BD4680BD80B483B000AF7860DD
:10B8A000044A7B68C2F8043100BF0C37BD4680BC37
:10B8B000704700BF00C00F4080B400AF044BD3F806
:10B8C0000431DBB201331846BD4680BC704700BF6F
:10B8D00000C00F4080B487B000AF0346FB71012366
:10B8E0007B61FB795B003B613B6903F01F03FB60FD
:10B8F0003B695B093B61194A3B696A3352F8233063
:10B900007B617A69FB6822FA03F303F003037B612E
:10B910007B69002B02D104237B6119E07B69012B39
:10B9200002D101237B6113E07B69022B02D1022348
:10B930007B610DE0FB790D2B05D0FB790E2B02D03E
:10B94000FB790F2B02D106237B6101E008237B6189
:10B950007B6918461C37BD4680BC704700C00F404D
:10B9600080B500AFFFF7C2FE0346012B07D0022BC4
:10B9700009D0002B0BD1FFF7D3FE034608E0FFF7F9
:10B98000C5FE034604E0FFF7D5FE034600E00023B2
:10B99000184680BD80B584B000AF0023FB60FFF780
:10B9A00067FE0346002B18D00E4BD3F88430C3F348
:10B9B0000E030133BB600B4BD3F884301B0CDBB29E
:10B9C00001337B60FFF7C0FE0246BB6803FB02F356
:10B9D0005A007B68B2FBF3F3FB60FB681846103734
:10B9E000BD4680BD00C00F4080B500AFFFF742FFED
:10B9F0000346002B05D0012B07D1FFF7CBFF0346F1
:10BA000004E0FFF7ADFF034600E00023184680BDC9
:10BA100098B500AFFFF7E8FF0446FFF74DFF034678
:10BA2000B4FBF3F3184698BD90B583B000AF03465E
:10BA3000FB71FFF7EDFF0446FB791846FFF74AFF5D
:10BA40000346B4FBF3F318460C37BD4690BD80B5F2
:10BA500000AFFFF7DDFF0346184680BD80B483B01A
:10BA600000AF78607B684FF44F421A607B687822A1
:10BA7000C3F8002100BF0C37BD4680BC704780B5BD
:10BA800084B000AF78607868FFF7E8FF0023FB60C0
:10BA900002E0FB680133FB60FB68632BF9D900BF50
:10BAA0001037BD4680BD80B582B000AF78600B46D0
:10BAB000FB701E20FFF7C4FE7868FFF7E0FF7B688D
:10BAC00002221A607B6831225A60FB78002B05D075
:10BAD0007B684FF4C862C3F8002104E07B684FF430
:10BAE0008862C3F800217B6815229A607B68122265
:10BAF000DA607B684FF480729A617B684FF4C062B1
:10BB00005A617B6843F20F721A617B68D3F8003187
:10BB100043F080027B68C3F800217B684FF6FF7218
:10BB2000C3F8E82F7B680022C3F8E42F00BF083772
:10BB3000BD4680BD80B485B000AFF860B9601346E3
:10BB4000FB71FB791B0203F4F8530A4A1360BB68CC
:10BB50009B0003F03C0343F40042FB681A62FB685D
:10BB60001B6A23F40042FB681A6200BF1437BD460B
:10BB700080BC70472861001080B584B000AF786049
:10BB800039600023FB60FFF762FF02463B68B2FBAF
:10BB9000F3F3BB600023FB600CE00A4AFB6813442C
:10BBA0001B781A46BB68934201D8FB6806E0FB6825
:10BBB0000133FB60FB680E2BEFD90E2318461037BC
:10BBC000BD4680BD0424010080B483B000AF78601E
:10BBD0000B46FB7013463B807B6800225A62FB7861
:10BBE00003F01F02064B1B681A437B689A623A886F
:10BBF0007B68DA6200BF0C37BD4680BC704700BF6F
:10BC00002861001080B483B000AF78600B46FB70F1
:10BC1000FB7803F01F02064B1B681A437B689A628D
:10BC20007B6801225A6200BF0C37BD4680BC70475A
:10BC30002861001080B483B000AF78607B68002278
:10BC40005A627B681B6B9BB218460C37BD4680BCA2
:10BC5000704780B483B000AF78607B685B6843F066
:10BC600001027B685A607B68D3F8003143F480623C
:10BC70007B68C3F800217B6815229A6000BF0C37EF
:10BC8000BD4680BC704780B483B000AF78607B68ED
:10BC90005B6823F001027B685A607B68D3F800314F
:10BCA00023F480627B68C3F800217B6812229A60CB
:10BCB00000BF0C37BD4680BC704780B485B000AF74
:10BCC000F860B9607A603B60BA68FB68C3F81C2111
:10BCD0003B685A1EFB68C3F824217A68FB68C3F8E6
:10BCE0002021FB680022C3F8282100BF1437BD467D
:10BCF00080BC704780B485B000AFF860B9607A60EE
:10BD00003B60BA68FB68C3F808213B685A1EFB68B1
:10BD1000C3F810217A68FB68C3F80C21FB68002285
:10BD2000C3F8182100BF1437BD4680BC704780B4EB
:10BD300085B000AFF860084611461A4603467B817D
:10BD40000B463B811346FB803A897B899A4201D19D
:10BD5000002311E03B89002B06D17A89FB88013B47
:10BD60009A4201D1022307E03A897B8901339A4242
:10BD700001D1022300E0012318461437BD4680BCE0
:10BD8000704780B485B000AF78607B68D3F8283105
:10BD9000FB60FB680133FB607B68D3F82431FA68F1
:10BDA0009A4201D90023FB607B68FA68C3F8282116
:10BDB000FB689BB218461437BD4680BC704780B400
:10BDC00085B000AF78607B68D3F81831FB60FB6802
:10BDD0000133FB607B68D3F81031FA689A4201D9CD
:10BDE0000023FB607B68FA68C3F81821FB689BB2EC
:10BDF00018461437BD4680BC7047FFFF80B582B03F
:10BE000000AF0346FB71FA7907491346DB009B1A22
:10BE10009B000B4404331B781846FFF711FD00BF4D
:10BE20000837BD4680BD00BF9C00001080B582B0C1
:10BE300000AF0346FB71FB79044AD35C1846FFF759
:10BE4000F3FD034618460837BD4680BD14240100A3
:10BE500080B483B000AF78607B683C229A617B68D5
:10BE600060221A6000BF0C37BD4680BC704780B4AA
:10BE700083B000AF78607B6838229A617B68442287
:10BE80001A6000BF0C37BD4680BC704780B483B0D9
:10BE900000AF78607B681B6803F01003002B0CBFB9
:10BEA00001230023DBB218460C37BD4680BC704727
:10BEB00080B483B000AF78607B685B6803F0F80300
:10BEC00018460C37BD4680BC704780B582B000AFC5
:10BED00078607868FFF7ECFF03465F2BD4BF01233F
:10BEE0000023DBB218460837BD4680BD80B483B05E
:10BEF00000AF0346FB710B46BB7113467B717B7928
:10BF000043F001037B71FA79BB795340DBB21A46E7
:10BF10007B79DB431340002B0CBF01230023DBB2F2
:10BF200018460C37BD4680BC704780B582B000AF64
:10BF300078600B46FB70FB785B08DBB2002B01D10D
:10BF400000233CE07B68DB68D8B27B681B6BDAB20D
:10BF5000FB781946FFF7CAFF0346002B01D00123E7
:10BF60002DE07B681B6AD8B27B685B6BDAB2FB782A
:10BF70001946FFF7BBFF0346002B01D002231EE04A
:10BF80007B685B6AD8B27B689B6BDAB2FB78194638
:10BF9000FFF7ACFF0346002B01D003230FE07B68C3
:10BFA0009B6AD8B27B68DB6BDAB2FB781946FFF785
:10BFB0009DFF0346002B01D0042300E00023184618
:10BFC0000837BD4680BDFFFF80B584B000AF786004
:10BFD00039603C23FB607868FFF76AFF0346582B03
:10BFE00000F2158101A252F823F000BFFDC100004C
:10BFF0000FC200000FC200000FC200000FC20000FD
:10C000000FC200000FC200000FC2000051C10000AB
:10C010000FC200000FC200000FC200000FC20000DC
:10C020000FC200000FC200000FC2000051C100008B
:10C030000FC200000FC200000FC200000FC20000BC
:10C040000FC200000FC200000FC200006FC100004D
:10C050000FC200000FC200000FC200000FC200009C
:10C060000FC200000FC200000FC20000E5C10000B7
:10C070000FC200000FC200000FC200000FC200007C
:10C080000FC200000FC200000FC200006FC100000D
:10C090000FC200000FC200000FC200000FC200005C
:10C0A0000FC200000FC200000FC20000E5C1000077
:10C0B0000FC200000FC200000FC200000FC200003C
:10C0C0000FC200000FC200000FC20000F5C1000047
:10C0D0000FC200000FC200000FC200000FC200001C
:10C0E0000FC200000FC200000FC20000D3C1000049
:10C0F0000FC200000FC200000FC200000FC20000FC
:10C100000FC200000FC200000FC20000E5C1000016
:10C110000FC200000FC200000FC200000FC20000DB
:10C120000FC200000FC200000FC20000B7C1000024
:10C130000FC200000FC200000FC200000FC20000BB
:10C140000FC200000FC200000FC20000AFC100000C
:10C150003B681B785B003A689268002A0CBF01229A
:10C160000022D2B213431A467B689A604FE03B68C4
:10C170009B68002B0CD13B681B69002B02D06FF031
:10C18000200301E06FF01003FA681340FB603EE00B
:10C190003B685B68591C3A6851601B781A467B689B
:10C1A0009A603B689B685A1E3B689A602FE0FB6868
:10C1B00023F01003FB607B6898683B68DB68591CC0
:10C1C0003A68D160C2B21A703B681B695A1E3B685C
:10C1D0001A613B681B69012B18DDFB6823F004031F
:10C1E000FB6013E03B6801221A75FB6823F0100323
:10C1F000FB600CE03B6802221A7508E03B680322F2
:10C200001A75FB6823F01003FB6000E000BFFB68B9
:10C2100083F03C027B681A607B68FA689A61FB686D
:10C2200003F01003002B03D03B681B7D022B08D1C9
:10C230003B681B7D042B02D13B6800221A7500234A
:10C2400000E0012318461037BD4680BD80B582B09E
:10C2500000AF78607868FFF72BFE0346702B0CD098
:10C26000702B04DC602B08D0682B06D00EE0A82BC6
:10C2700003D0B02B01D0782B08D17B689B68DBB250
:10C2800019467868FFF751FE034600E00023184680
:10C290000837BD4680BDFFFF80B584B000AF786031
:10C2A00039603C23FB600023BB603B6804221A75A5
:10C2B0007868FFF7FDFD0346603B682B00F23A818A
:10C2C00001A252F823F000BF9FC4000035C5000052
:10C2D00035C5000035C5000035C5000035C5000076
:10C2E00035C5000035C500009FC4000035C50000FD
:10C2F00035C5000035C5000035C5000035C5000056
:10C3000035C5000035C500009FC4000035C50000DC
:10C3100035C5000035C5000035C5000035C5000035
:10C3200035C5000035C500009FC4000035C50000BC
:10C3300035C5000035C5000035C5000035C5000015
:10C3400035C5000035C500006DC4000035C50000CE
:10C3500035C5000035C5000035C5000035C50000F5
:10C3600035C5000035C5000003C5000035C5000017
:10C3700035C5000035C5000035C5000035C50000D5
:10C3800035C5000035C500006DC4000035C500008E
:10C3900035C5000035C5000035C5000035C50000B5
:10C3A00035C5000035C5000003C5000035C50000D7
:10C3B00035C5000035C5000035C5000035C5000095
:10C3C00035C5000035C5000003C5000035C50000B7
:10C3D00035C5000035C5000035C5000035C5000075
:10C3E00035C5000035C50000C1C4000035C50000DA
:10C3F00035C5000035C5000035C5000035C5000055
:10C4000035C5000035C50000C1C4000035C50000B9
:10C4100035C5000035C5000035C5000035C5000034
:10C4200035C5000035C50000D1C4000035C5000089
:10C4300035C5000035C5000035C5000035C5000014
:10C4400035C5000035C5000003C5000035C5000036
:10C4500035C5000035C5000035C5000035C50000F4
:10C4600035C5000035C5000003C500007B6898682D
:10C470003B68DB68591C3A68D160C2B21A703B68ED
:10C480001B695A1E3B681A610523BB603B681B6928
:10C49000012B4ADDFB6823F00403FB6045E07B6869
:10C4A0009B68DBB223F00103DAB23B681A703B6889
:10C4B0001B69012B3BDDFB6823F00403FB6036E0C6
:10C4C0007B689B68DBB223F00103DAB23B681A7029
:10C4D0003B685B68591C3A6851601B781A467B6858
:10C4E0009A603B689B685A1E3B689A603B689B68F1
:10C4F000002B03DDFB6823F00403FB600623BB6015
:10C5000018E00223BB60FB6823F00403FB603B6878
:10C5100000221A753B681B7803F00103002B08D03A
:10C52000FB6823F02003FB6003E000BF02E000BFD4
:10C5300000E000BFFB6883F03C027B681A607B6808
:10C54000FA689A61BB6818461037BD4680BD00BFC7
:10C5500080B485B000AF03460A46FB711346BB7139
:10C56000FA791346DB009B1A9B000B4A1344FB60CD
:10C57000BB79012B0AD1FB681B691433BB6000BF78
:10C58000BB681B78DBB2042BFAD000E000BF143785
:10C59000BD4680BC704700BF9C00001080B584B0D1
:10C5A00000AF03460A46FB711346BB71FA79134686
:10C5B000DB009B1A9B00104A1344FB60BB79012BE4
:10C5C00015D1FB681B691433BB600AE0FB79184680
:10C5D00000F002FA0346002B03D0FB79184600F066
:10C5E0006BF9BB681B78DBB2042BEFD000E000BF17
:10C5F0001037BD4680BD00BF9C00001080B582B0E2
:10C6000000AF0346FB71FB791846FFF7F7FBFA7999
:10C6100006491346DB009B1A9B000B441B686C22E7
:10C620009A6100BF0837BD4680BD00BF9C00001066
:10C6300080B584B000AF03463960FB71FB791846C2
:10C64000FFF7F4FB02463B68B2FBF3F3FB60FA79B9
:10C6500010491346DB009B1A9B000B441B68FA68C9
:10C6600052081A61FA790B491346DB009B1A9B00AA
:10C670000B441B681969FA7906481346DB009B1ABC
:10C680009B0003441B68FA68521A5A6100BF1037B6
:10C69000BD4680BD9C00001080B485B000AF03464D
:10C6A0003960FB71FA791346DB009B1A9B000B4A39
:10C6B0001344FB60FB681B69002B02D1FB683A68DE
:10C6C0009A60FB689B683A689A420CBF012300237A
:10C6D000DBB218461437BD4680BC70479C00001082
:10C6E00080B584B000AF03463960FB71FA79134618
:10C6F000DB009B1A9B00204A1344FB60FB689B688D
:10C70000FA790321104698473B6804221A75FB68A2
:10C710003A681A61FB685B69002B04D1FB681B68EF
:10C720001846FFF795FBFB689B68FA7901211046D4
:10C730009847FB6800221A6100BFFB681B68184617
:10C74000FFF7A4FB0346002BF7D0FB689B6903F4BB
:10C750007F43002B04D0FB681B681846FFF787FB5C
:10C76000FB689B68FA790421104698473B681B7D5B
:10C7700018461037BD4680BD9C00001080B588B0BB
:10C7800000AF3A601A460346FB710B46BB71134675
:10C790007B7107F1080300221A605A609A60DA6020
:10C7A0001A615A61BB793B723B68FB607B793B61E4
:10C7B00000BF07F10802FB7911461846FFF790FF0A
:10C7C0000346022BF5D07A793B69D31A18462037F5
:10C7D000BD4680BD80B588B000AF3B600346FB71AD
:10C7E0000B46BB7113467B7107F1080300221A60E8
:10C7F0005A609A60DA601A615A61BB793B727B1D9C
:10C80000FB6001233B613B687B61BB6ABB6100BF8E
:10C8100007F10802FB7911461846FFF761FF03464E
:10C82000022BF5D0BB69BA6AD31A18462037BD4629
:10C8300080BD80B58AB000AFBA607B600346FB73F1
:10C840000B46BB7307F1100300221A605A609A600E
:10C85000DA601A615A61BB7B3B74BB68FB617B6821
:10C860003B6200BF07F11002FB7B11461846FFF741
:10C8700037FF0346022BF5D03B6A7A68D31A184675
:10C880002837BD4680BDFFFF80B582B000AF0346AC
:10C89000FB71FA7907491346DB009B1A9B000B4496
:10C8A0001B681846FFF711FB034618460837BD46BC
:10C8B00080BD00BF9C00001080B582B000AF034671
:10C8C000FB71FA7913491346DB009B1A9B000B445A
:10C8D0001868FA790F491346DB009B1A9B000B443A
:10C8E00010331B681946FFF76FFB0346002B0CD172
:10C8F000FA7908491346DB009B1A9B000B44083366
:10C900001B68FA7902211046984700BF0837BD46D8
:10C9100080BD00BF9C00001080B586B000AF03460C
:10C92000FB71FA791346DB009B1A9B00284A1344DB
:10C930007B617B695B69002B18D17B691B6818469A
:10C94000FFF784FC0346FB74FA79F97C13469B00DD
:10C9500013440B44DB001F4A1344FB60FB681A6856
:10C960007B695A61FB685A687B69DA607B695B693D
:10C970001B785AB27B691B69002B14BF012300236B
:10C98000DBB25BB213435AB27B695B69D2B21A70F5
:10C990007B691A687B695B6919461046FFF77CFC66
:10C9A000B860BB68002B0ED07B695B691B7D002BD8
:10C9B00002D17B6900225A617B69DB68BA68D1B217
:10C9C000FA791046984700BF1837BD4680BD00BFB2
:10C9D0009C0000102C61001080B483B000AF0346AF
:10C9E000FB71FA7909491346DB009B1A9B000B4443
:10C9F0001B681B6803F00803002B14BF01230023EE
:10CA0000DBB218460C37BD4680BC70479C00001056
:10CA100080B586B002AFF8607B600B46FB721346B0
:10CA2000BB727B6898087B68DBB203F00303DBB260
:10CA3000BA7AF97A00930346F86800F004F800BF68
:10CA40001037BD4680BD80B487B000AFF8607B6012
:10CA50000B46FB721346BB72BB7A03F00F03DBB2CB
:10CA60005B00FB75FB7A5B00DAB2BB7A1B09DBB2B9
:10CA70001344BB75BA7DFB6853F82220FB7D03216C
:10CA800001FA03F3DB4313403B6197F82020FB7D61
:10CA900002FA03F31946BA7D3B691943FB6843F870
:10CAA0002210BA7DFB68103253F82220FB7D03214F
:10CAB00001FA03F3DB4313403B61FB7D7A6802FA22
:10CAC00003F1BA7D3B691943FB68103243F8221029
:10CAD00000BF1C37BD4680BC704780B586B000AF34
:10CAE000F860B9607A6000237B611FE07B699B007E
:10CAF000BA6813441B78C3F30203DBB219467B699F
:10CB00009B00BA6813441B78C3F3C403DBB2184616
:10CB10007B699B00BA6813441B68C3F31723024662
:10CB2000F868FFF775FF7B6901337B617A697B6881
:10CB30009A42DBD300BF1837BD4680BD80B483B0B6
:10CB400000AF7860062318460C37BD4680BC70479E
:10CB500080B582B000AF78607868FFF7EFFF0346DA
:10CB60001846FEF76DFE00BF0837BD4680BD80B495
:10CB700085B000AF78607B685B68FB607B680022F3
:10CB80005A607B6801229A607B685B6843F0080208
:10CB90007B685A607B68FA685A6000BF1437BD46EC
:10CBA00080BC704780B483B000AF786008461146FF
:10CBB0001A460346FB700B46BB7013467B70FB782E
:10CBC000002B2FD07B78002B0AD07B68DB6CFA78A7
:10CBD0000832012101FA02F21A437B68DA640AE0A2
:10CBE0007B68DB6CFA780832012101FA02F2D24349
:10CBF0001A407B68DA64BB78012B09D17B68DB6C57
:10CC0000FA78012101FA02F21A437B68DA6409E03A
:10CC10007B68DB6CFA78012101FA02F2D2431A40F8
:10CC20007B68DA6400BF0C37BD4680BC704780B4B7
:10CC300083B000AF78600B46FB701346BB70BB78C7
:10CC4000002B09D07B681B6DFA78012101FA02F2F2
:10CC50001A437B681A6509E07B681B6DFA7801212D
:10CC600001FA02F2D2431A407B681A6500BF0C3702
:10CC7000BD4680BC704780B483B000AF78607B68ED
:10CC80000C331A687B6810331B68D31A18460C37AC
:10CC9000BD4680BC704790B583B000AF78607B68BC
:10CCA0005C687868FFF7E7FF0346E31A18460C371D
:10CCB000BD4690BD80B582B000AF78607868FFF760
:10CCC000DAFF02467B685B689A42ACBF012300230F
:10CCD000DBB218460837BD4680BD80B483B000AFD4
:10CCE00078607B680C331A687B6810331B689A4243
:10CCF0000CBF01230023DBB218460C37BD4680BCB5
:10CD0000704780B485B000AFF860B9607A603B606E
:10CD1000FB68BA681A60FB683A685A60FB687A6810
:10CD20009A60FB6800221A61FB681A69FB68DA6086
:10CD3000012318461437BD4680BC704780B584B0C7
:10CD400000AF786039607B681B68FB607868FFF72C
:10CD5000B1FF0346002B01D0002319E07B68DB689C
:10CD60007A685268013A13407A68926802FB03F3CA
:10CD7000FA681344FB607B689B681A463968F86858
:10CD800000F004FD7B68DB685A1C7B68DA600123D5
:10CD900018461037BD4680BD80B588B000AFF8603A
:10CDA000B9607A60FB681B68BB61F868FFF782FFB7
:10CDB0000346002B01D000237BE0F868FFF76BFFF0
:10CDC00078617B69FB61FB68DB68FA685268013A4D
:10CDD0001A40FB691344FA68526893420AD3FB680D
:10CDE0005B681946FB68DB68FA685268013A1340D1
:10CDF000CB1AFB617A69FB69D31A7B61FA697B689C
:10CE00009342A8BF1346FB617A68FB69D31A7B6023
:10CE10007A697B689342A8BF13467B617A687B6915
:10CE2000D31A7B60FB68DB68FA685268013A1340EA
:10CE3000FA68926802FB03F3BA691344BB61FB68AA
:10CE40009B68FA6902FB03F31A46B968B86900F0F7
:10CE50009DFCFB68DA68FB691A44FB68DA60FB68D2
:10CE60001A68FB68DB68F968496801390B40F968A2
:10CE7000896801FB03F31344BB61FB689B68FA6993
:10CE800002FB03F31A46BB681344BB60FB689B6854
:10CE90007A6902FB03F31A46B968B86900F076FCB8
:10CEA000FB68DA687B691A44FB68DA60FA697B69B7
:10CEB000134418462037BD4680BD80B584B000AF0E
:10CEC000786039607B681B68FB607868FFF705FF56
:10CED0000346002B01D0002319E07B681B697A68A8
:10CEE0005268013A13407A68926802FB03F3FA68C9
:10CEF0001344FB607B689B681A46F968386800F049
:10CF000045FC7B681B695A1C7B681A610123184623
:10CF10001037BD4680BD80B588B000AFF860B960FD
:10CF20007A60FB681B68BB61F868FFF7D6FE0346B2
:10CF3000002B01D000237BE0F868FFF79CFE7861AE
:10CF40007B69FB61FB681B69FA685268013A1A4009
:10CF5000FB691344FA68526893420AD3FB685B6822
:10CF60001946FB681B69FA685268013A1340CB1AEC
:10CF7000FB617A69FB69D31A7B61FA697B6893422A
:10CF8000A8BF1346FB617A68FB69D31A7B607A6994
:10CF90007B689342A8BF13467B617A687B69D31A8A
:10CFA0007B60FB681B69FA685268013A1340FA68B3
:10CFB000926802FB03F3BA691344BB61FB689B6888
:10CFC000FA6902FB03F31A46B969B86800F0DEFBA0
:10CFD000FB681A69FB691A44FB681A61FB681A68E6
:10CFE000FB681B69F968496801390B40F968896871
:10CFF00001FB03F31344BB61FB689B68FA6902FB06
:10D0000003F31A46BB681344BB60FB689B687A69EC
:10D0100002FB03F31A46B969B86800F0B7FBFB6876
:10D020001A697B691A44FB681A61FA697B691344BF
:10D0300018462037BD4680BD80B483B000AF78600D
:10D0400039607B683A681A6000BF0C37BD4680BC07
:10D05000704780B483B000AF786039607B689A68AD
:10D060003B681A437B689A6000BF0C37BD4680BCA2
:10D07000704780B582B000AF78601020FEF7E0FB0B
:10D080007B684FF0FF321A607B6800225A607B6831
:10D090000C229A607B680022DA6000BF0837BD4628
:10D0A00080BDFFFF80B584B000AF786039601D207F
:10D0B000FEF7BAFC02460A4BA3FB02239A093B681F
:10D0C00002FB03F3FB60F9687868FFF7B5FF022104
:10D0D0007868FFF7BEFF00BF1037BD4680BD00BFB8
:10D0E000D34D621080B400AF064BD3F8883003F004
:10D0F0008073002B14BF01230023DBB21846BD460A
:10D1000080BC704700C00F4080B400AF064BD3F81E
:10D11000883003F08063002B14BF01230023DBB2AF
:10D120001846BD4680BC704700C00F4080B400AFB9
:10D13000064BD3F8883003F00073002B14BF012393
:10D140000023DBB21846BD4680BC704700C00F40CC
:10D1500080B400AF054BD3F8A031044A43F020035C
:10D16000C2F8A03100BFBD4680BC704700C00F4070
:10D1700080B400AF064BD3F8A03103F04003002B7E
:10D1800014BF01230023DBB21846BD4680BC7047A4
:10D1900000C00F4080B483B000AF0346FB71044A67
:10D1A000FB79C2F80C3100BF0C37BD4680BC70471C
:10D1B00000C00F4080B500AFFFF7B8FF0346002B5B
:10D1C00003D002210020FEF7E9FAFFF78BFF0346A8
:10D1D000002B03D001210020FEF7E0FAFFF7C8FF83
:10D1E000034683F00103DBB2002B01D0FFF7B0FF51
:10D1F00000BFFFF7BDFF034683F00103DBB2002B46
:10D20000F7D10020FEF748FB0120FFF7C3FF002203
:10D210000F210020FEF7E6FA01210020FEF79CFA1C
:10D220000320FEF739FB00BFFFF76EFF034683F0D4
:10D230000103DBB2002BF7D102210020FEF78CFAAC
:10D2400000BF80BD80B483B000AF78607B680C33D2
:10D250001A687B6810331B689A420CBF01230023B5
:10D26000DBB218460C37BD4680BC704780B483B033
:10D2700000AF78600B46FB70FA787B681A6000BFDD
:10D280000C37BD4680BC704780B483B000AF786077
:10D290007B681B68DBB218460C37BD4680BC704704
:10D2A00080B483B000AF786039607B685A683B68AF
:10D2B0001A437B685A6000BF0C37BD4680BC70477C
:10D2C00080B483B000AF786039607B685A683B688F
:10D2D000DB431A407B685A6000BF0C37BD4680BCF8
:10D2E000704780B483B000AF78607B689B68184655
:10D2F0000C37BD4680BC704780B483B000AF786007
:10D3000039607B683A689A6000BF0C37BD4680BCC4
:10D31000704780B483B000AF786039607B683A684A
:10D32000DA6000BF0C37BD4680BC704780B483B064
:10D3300000AF78607B68DB6843F080027B68DA606E
:10D3400000BF0C37BD4680BC704780B483B000AFCF
:10D3500078607B68DB6823F080027B68DA6000BF5E
:10D360000C37BD4680BC704780B483B000AF786096
:10D370000B46FB701346BB70FA787B681A60BA786C
:10D380007B685A6000BF0C37BD4680BC704780B4D4
:10D3900083B000AF78607B685B6918460C37BD4688
:10D3A00080BC704780B483B000AF786039607B6820
:10D3B0001A6A3B681A437B681A6200BF0C37BD4685
:10D3C00080BC704780B485B000AF78607B680E4A3F
:10D3D000934202D10423FB730FE07B680B4A934214
:10D3E00002D11823FB7308E07B68094A934202D1FB
:10D3F0001923FB7301E00323FB73FB7B18461437EF
:10D40000BD4680BC704700BF00000140008009405D
:10D4100000C0094080B582B000AF78607868FFF73F
:10D4200060FF034603F48073002B11D04FF480712A
:10D430007868FFF7B7FF4FF480717868FFF740FF17
:10D440000E4B1B78DBB2002B02D10C4B01221A7061
:10D450007868FFF746FF034603F40073002B09D0FA
:10D460004FF400717868FFF79DFF4FF40071786802
:10D47000FFF726FF00BF0837BD4680BDA46100103E
:10D4800080B485B000AF78607B680E4A934202D1C9
:10D490000423FB730FE07B680B4A934202D11823ED
:10D4A000FB7308E07B68094A934202D11923FB739E
:10D4B00001E00323FB73FB7B18461437BD4680BC99
:10D4C000704700BF000001400080094000C00940D3
:10D4D00080B584B000AF78607868FFF773FF0346CB
:10D4E0001846FEF7ADF907217868FFF705FF786861
:10D4F00000F036F87B6800225A607B680022DA6010
:10D500007B6800221A627B680022DA647B68002252
:10D510005A657B6800221A657B680A4A934205D1E6
:10D520007B6800221A617B689B69FB600321786835
:10D53000FFF7EFFE7B6810229A6200BF1037BD46EE
:10D5400080BD00BF0000014080B483B000AF7860B0
:10D550007B6880221A6300BF0C37BD4680BC7047D1
:10D5600080B483B000AF78607B6800221A6300BF8C
:10D570000C37BD4680BC704780B586B000AF786080
:10D5800039607868FFF77CFF03461846FEF74CFACF
:10D5900078613B681B017A69B2FBF3F33B613B693D
:10D5A0001B0AFB60FB681B023A69D31ABB607868F0
:10D5B000FFF7BCFEBB68DBB2FA68D2B219467868E6
:10D5C000FFF7D2FE7868FFF7C0FE7A693B69B2FBCD
:10D5D000F3F318461837BD4680BD80B584B000AF60
:10D5E000786039600AE07868FFF74EFE0346FB7307
:10D5F00007F10F0319463868FFF7A0FB7868FFF7BB
:10D60000C6FE034603F00103002BECD100BF103728
:10D61000BD4680BD80B584B000AF7860396004E05D
:10D62000FB7B19467868FFF721FE7868FFF7AFFEAD
:10D63000034603F02003002B08D007F10F0319461F
:10D640003868FFF73AFC0346002BE9D100BF1037DA
:10D65000BD4680BD80B586B000AFF860B9607A6025
:10D660003B607B687B610221F868FFF729FE3A681E
:10D670007969B868FFF790FB03463B61B968F868C1
:10D68000FFF7C8FF7A693B69D1183A683B69D31A3A
:10D690001A46B868FFF780FB03461A463B691344F5
:10D6A0003B610221F868FFF7FBFD3B69184618371C
:10D6B000BD4680BD80B584B000AFF860B9607A60C7
:10D6C0003B603A687968B868FFF725FC034618465E
:10D6D0001037BD4680BD80B584B000AFF860B9603A
:10D6E0007A60FB685B6803F00203002B0DD0796859
:10D6F000F868FFF78FFF7868FFF7A4FD0346002B5B
:10D7000003D00221F868FFF7DBFDB968F868FFF77E
:10D7100064FFF868FFF77EFE00BF1037BD4680BD8E
:10D7200080B483B000AF78607B6800221A607B68A9
:10D73000FF225A6000BF0C37BD4680BC704780B4E2
:10D7400083B000AF786039603B6803F00403002BBE
:10D7500005D07B681B6803F01B027B681A603B687E
:10D7600003F00803002B05D07B681B6843F0080218
:10D770007B681A6000BF0C37BD4680BC704708B597
:10D7800000F04CFDBDE80840FAF7ACBC03F04DBC1E
:10D7900003F065BC03F071BC10B5425C4318342A39
:10D7A00001DC002010BD352A06D1194611F8012FE1
:10D7B000302AFBD0002AF4D01A46302412F8011D7A
:10D7C000392901D11470F9E7013111700278302A3A
:10D7D000E7D01A1A002A01DA0120E3E713F8012939
:10D7E0009A70F6E730B50A258C1FA14200D130BDF2
:10D7F00090FBF5F3C3EB4312C3EB8202303000EB36
:10D80000420001F801091846EFE7FFFF0FB47FB5AA
:10D8100008AB53F8042B08490593CDE90131009278
:10D820006FF000434FF0FF32044800F055FD07B0A1
:10D830005DF804EB04B07047B1D80000F06100104F
:10D840000EB430B594B017AB53F8044B05463C22E8
:10D85000002105A80493FFF79DFF0A2308936FF0AA
:10D8600000430793104B4FF0FF320293049B05A82F
:10D87000CDE900436FF00043059500F02DFD079BB7
:10D880000446013B002B079308DB0022059B1A701E
:10D89000204614B0BDE8304003B0704705A9002011
:10D8A00002F0F8FAF4E700BFB1D80000FFFFFFFF75
:10D8B0002DE9F04F9DB004930B68144606934B6816
:10D8C00081460593079347F6F073059ADDF89CA00F
:10D8D00033EA12432AD10023E370C2F31303069AFA
:10D8E00013434FF06E031BD1637066236922A3704C
:10D8F000059B2270002B07DAAB4B0325269A136099
:10D9000028461DB0BDE8F08F049B980706D4A74AAF
:10D9100013F0040FA64B18BF1346EEE7A54BECE738
:10D9200061222370A3706270A14BE6E720F0200310
:10D93000412B00F0A982DDE906010022002303F05B
:10D9400005F9069E00283FD0079B03F100450123FF
:10D950000C93002200233046294603F0E1F800280A
:10D9600040F08C8240F22D1B0FAA3046294602F06F
:10D970008EFB4FF47A730F9ACDE910010BFB02FB7B
:10D98000ABF5AB5BABF11C0B9BFBF3FB0020ABEBF4
:10D990000202894902F0A6FBBBF1000FCDE91A0192
:10D9A00015DA7BA3D3E90023CDE91623CBF10005DB
:10D9B000E90714D4DDE91601DDE9162302F0BEFD06
:10D9C0006D10CDE91601F3E7059D0C90C1E74FF00E
:10D9D00000027A4BCDE916230BD05D46E8E7DDE97E
:10D9E0001601DDE91A2302F0A9FD012DCDE91A0186
:10D9F000E0D1DDE91001DDE91A2302F025FE002661
:10DA0000CDE912016E4FDDE9120163A3D3E90023D2
:10DA100003F09CF8002840F095800026684FDDE96F
:10DA200012015FA3D3E9002303F0E4F8002840F0DB
:10DA30009C80DDE9120103F027F805468BEAEB73C1
:10DA4000A3EBEB730D930F9A2846ABEB020603F0A2
:10DA50005EF8324602F046FB00220023BBF1000FC5
:10DA6000CDE91201CDE9142380F2AC8048A3D3E9BB
:10DA70000023CDE9162300220023CDE91823DDE998
:10DA80001667DDE916010026DDE91823CDE9082334
:10DA900032463B4602F070FEDDE9082302F044FF07
:10DAA000CDE91801CDE91667DDE916010022434BE7
:10DAB00002F044FD02460B4600203F4902F05CFEA6
:10DAC00000223E4B02F0C0FDCDE91801DDF83480A4
:10DAD00018F0010F40F08D80DDE91623DDE9180113
:10DAE000DDE91867CDE908011046194602F01CFF70
:10DAF000DDE9082302F018FF32463B4602F01EFD26
:10DB0000CDE91801DDE91601DDE9162302F016FD65
:10DB1000CDE91601DDE91667DDE916010026DDE92C
:10DB20001823CDE9082332463B4602F025FEDDE905
:10DB3000082302F0F9FE4FEA6808CDE91801CDE9A3
:10DB40001667C5E7DDE9120132463B4602F0F6FCF6
:10DB5000CDE91201DDE91A0132463B4602F074FDBF
:10DB60000BF1FF3BCDE91A014DE7DDE91201324629
:10DB70003B4602F069FDCDE91201DDE91A013246AA
:10DB80003B4602F0DBFC0BF1010BCDE91A0146E745
:10DB90009A9999999999C93F00000000006AF84044
:10DBA0000000000080842E41492401001924010056
:10DBB0009F240100172401000000F03F00001440E2
:10DBC000000024404FF00002B94BCDE916234FF07E
:10DBD00000024FF00003CDE918237FF477AFDDE9B1
:10DBE0001201DDE9102302F0DBFF002847D1013DDF
:10DBF00029E7DDE91223CDE90823DDE91823DDE972
:10DC00001601CDE90A23DDE91823DDE9146702F0E6
:10DC10008BFE32463B4602F091FCDDE90A230646C4
:10DC20000F46DDE9080102F089FC02460B4630464A
:10DC3000394602F079FECDE91401DDE91601DDE98E
:10DC4000122302F07BFCCDE91201DDE91267DDE968
:10DC500012010026DDE91423CDE9082332463B46B4
:10DC600002F08AFDDDE9082302F05EFEB8F1010F43
:10DC7000CDE91401CDE912677FF42EAFAFE7DDE9FE
:10DC80001223DDE9100102F077FDCDE91001DDE995
:10DC90001423DDE9100102F06FFDCDE91001DDE98B
:10DCA0001A23DDE9100102F0CFFC7FA3D3E90023A2
:10DCB000CDE91001DDE9100102F040FCCDE91001D1
:10DCC000DDE9100102F0E0FEDDE91067804602F0B8
:10DCD0001EFF02460B463046394602F04DFD72A348
:10DCE000D3E9002302F02AFCCDE91001DDE910019F
:10DCF00002F0CAFE0646002EC0F28C806D4B9E429A
:10DD000000F38F80B8F1000FC0F29280694B984504
:10DD100000F39480684A954200F39680674B0A218D
:10DD200098FBF3F296FBF3F3654801FB052500FB36
:10DD3000028800FB036601FB08384E430BF1FF3BF2
:10DD400021463027284601F8067BFFF74BFD04F1FA
:10DD50000C014046FFF746FD04F112013046FFF783
:10DD600041FD002323750C9B0BF1050BE77443EA7F
:10DD70008B0B1BF0010F00F08A80524B269A2BF080
:10DD8000010B13600423B9F1610F9BFBF3FBDAF87D
:10DD900000500DD000F3A480B9F1450F00F0AC8025
:10DDA000B9F1470F00F0E781B9F1410F40F0E1818F
:10DDB000059B0027C3F31301069B00201E461A464D
:10DDC000059B0F43C3F30A510643002900F00A8163
:10DDD000A1F2FF30002D40F00B81049B1B0700F1E6
:10DDE0000781002903463849384814BF31223022C0
:10DDF000B9F1610F18BF01462046FFF721FD314AF6
:10DE0000079B3349054612EA230338BF0B46269A7F
:10DE1000136075E506F5742606F5107608F1FF38EF
:10DE200069E7A6F57426A6F5107608F1010866E7FD
:10DE300008F5742808F51078013D63E7A8F5742803
:10DE4000A8F51078013562E79D427FF779AF0A2285
:10DE50006FF0090395FBF2F103FB01551D480BF12F
:10DE6000010B00FB058595FBF2F803FB085300FB53
:10DE70000366053696FBF2F60D4661E700266FF065
:10DE8000040BB04635465BE74FF0000B71E7049B8F
:10DE90009A0706D4104A13F0040F0D4B18BF13460F
:10DEA0006CE70E4B6AE700BF0000000080842E4143
:10DEB000000014403F420F009F860100A086010031
:10DEC0006079FEFF492401001B2401002324010086
:10DED0009F24010040420F00192401001724010073
:10DEE000B9F1660F00F06681B9F1670F00F0438168
:10DEF000B9F1650F40F03D81DAF80030112B05DDF6
:10DF0000299A113B13601123CAF80030049BDAF8F8
:10DF1000005013F4006605F1020504D1294620469D
:10DF2000FFF73AFC834463782370DAF8003023B9B2
:10DF300040F60803049A1A426CD02E236370299B82
:10DF40001B68002BC2BF3E236355013576B1049B8D
:10DF500019070BD46219151B12F8013D302BFAD0AA
:10DF60003E2BF8D02E2B08BF05F1FF35BBF1000F7B
:10DF7000B6BF2D212B21CBF1000B6A1CBBF57A7F9C
:10DF800004F8059005F10203A1540ADB4FF47A72FC
:10DF90009BFBF2F202F13001E1549C4B03FB02BB0C
:10DFA000EB1CBBF1630F0ADD64229BFBF2F202F172
:10DFB0003001E1546FF0630101FB02BB01330A221F
:10DFC0009BFBF2F2D2B202F13001E1549D1C1C44E1
:10DFD000C2EB4213C2EB83020BF1300B0BEB42029C
:10DFE00062708DE456EA0703894808BF0020F1E615
:10DFF000002902908749884814BF31223022CDE998
:10E000000067B9F1610F18BF01462B462046FFF7A4
:10E0100017FCF4E6012592E75B449D1C122DC1BF5D
:10E02000299A113B1360132576B929462046FFF73C
:10E03000B3FB48B17FEA0B0705F1010504D1637812
:10E0400023702E236370CDE0012F04EB05030CD168
:10E050001A1B002A02DC01353023F1E713F80129ED
:10E060009A70F5E713F80129DA701A1B002AF9DC17
:10E07000302323702E2363703C23A370289B013F21
:10E0800002351F60AEE00BEB0307BD1C122D51DD06
:10E090008EBB13212046FFF77FFB60B314250BF1E5
:10E0A000010B6A1E5A45234627DD5A7803F8012BD7
:10E0B0001A1B9345F9DA2E2204EB0B035A70DAF897
:10E0C0000030299A5B44113B1360002B40F08F8095
:10E0D000002E44D0049B1A073FF512AC6219151BA1
:10E0E00012F8013D302BFAD03E2BF8D02E2B7FF4C6
:10E0F00007AC013D04E41325D3E7597803F8011B6D
:10E10000191B8A42F9DC3C22631903F8012CABEBA2
:10E11000050B289A0BF1020313602E226255DAF8E0
:10E1200000206B1C002A6CD0299902350A603E221F
:10E13000E254CDE73EB929462046FFF72DFB10B14A
:10E140000BF1010BFD1C23465A7803F8012B1A1B17
:10E150009345F9DA2E23A3448BF80130B8E7DAF8B7
:10E160000030002B7FF4CCAB049B1B073FF5C8AB02
:10E17000BFE74FF06709049B002D43F4006304934D
:10E18000DCBF0123CAF80030DAF80010204611295C
:10E19000A8BF11210131FFF7FFFADAF800308344FC
:10E1A0005B4528DD1BF1040F25DB0BF101029B1AF7
:10E1B000CAF80030049ABBF1000FDAF8003002F41C
:10E1C0000066BFF660AFCBF100075A1CBA42BFF63B
:10E1D00023AF302323702E2302256370DAF800303A
:10E1E000299A1360299B1B68002B7FF771AF3E2390
:10E1F000635501356CE7013BCAF80030A9F102090B
:10E200007AE61D46002E7FF465AFADE718FCFFFFF0
:10E2100001FCFFFF2B2401003A24010010B5174A2E
:10E220001749002001F0D6FE4FF480734FF480624E
:10E230000021124801F046FC124A1349012001F066
:10E24000C9FE4FF480734FF4806200210D4801F045
:10E2500039FC0E4B1B68022B0EDD0D4A0A490220C9
:10E2600001F0B8FEBDE810404FF480734FF48062B7
:10E270000021074801F026BC10BD00BFB4610010AA
:10E280004B240100F06100104D2401002026010004
:10E290002C62001040EA01039B0770B50CD10446C4
:10E2A0000B46032A1946204606D906680D68043431
:10E2B000AE4203F1040304D00A44914203D100208A
:10E2C00008E0043AEDE710F8013B11F8014BA342D6
:10E2D000F3D0181B70BDFFFF2DE9F04F9FB0CDE9C3
:10E2E0000A23DDE92839002205460592187803F152
:10E2F000010818B905981FB0BDE8F08F252819D07E
:10E30000DDE90A67059B1946DA175C1C1346B14222
:10E31000BB4108DAAB68013B002BAB6006DB2B6826
:10E320005A1C2A60187005944346DFE7294601F01D
:10E33000B1FDF8E7002409E02D2F04D0302F0FD1D4
:10E3400044F4007401E044F00104B046464616F877
:10E35000017B2B2F12D0EFD8202F12D0232F13D0D8
:10E360002A2F14D000230A21A7F13002D0B20928A5
:10E370001BD801FB032316F8017BF5E744F00204E8
:10E38000E3E744F00404E0E744F00804DDE709F1C2
:10E390000402D9F800309146002B98F80170BCBFF8
:10E3A0005B4284F0010408F1020623EAE3732E2F96
:10E3B0000D9334D137782A2F0FD000230A2201364B
:10E3C0000693A7F13003D9B209290DD8069916F89A
:10E3D000017B02FB01330693F3E7D9F8003077782D
:10E3E000069309F104090236069B002B17DB44F063
:10E3F00010046C2F0AD137786C2F03BF777844F064
:10E4000060040236013618BF44F020044C2F01D0BE
:10E41000712F07D1377844F0600401360FE00023F4
:10E420000693E6E7682F1FD13778682F03BF777808
:10E4300044F480740236013618BF44F08004672F1C
:10E440006DDC652F80F2AF82472F00F0AC8216DCC6
:10E45000412F00F0A282452F00F0A582002F00F08E
:10E460003881CDF83090C4E06A2F03D144F04004E5
:10E470003778D2E77A2FFBD0742FE0D1F8E7612FFD
:10E4800000F08B8220DC582FEBD1610640F1A28195
:10E4900009F1070929F0070909F108030C93D9E9E3
:10E4A00000AB220640F19F811FFA8AFA4FF0000B61
:10E4B000B64B14F0080FB64A18BF1A46E00601D54D
:10E4C00024F40074B34BC9E1632F00F08D80642FF6
:10E4D000C7D1630640F1498209F1070929F007090C
:10E4E00009F108030C93D9E900AB200640F14682FC
:10E4F0000FFA8AFA4FEAEA7BBAF1000F7BF10003C8
:10E5000080F24282DAF1000AA34A6BEB4B0B14F063
:10E51000100300F0A38124F4007400239EE1702F07
:10E5200000F0928106DC6E2F00F0DB8000F3D081DA
:10E53000692FCDE7752F00F0F181782F00F0598118
:10E54000732F8ED109F104030C93D9F800A0934BDB
:10E55000BAF1000F08BF9A46504601F016FB8346F9
:10E56000E00603D5069B9B45A8BF9B460D9BA3EBEE
:10E570000B0714F00103069313D1059A14F4007FDE
:10E580000CBF2023302390463C464FEAE279013C01
:10E5900040F1C080059A27EAE7731A44013F0592CB
:10E5A000FF1A059B002498464FEAE379AAEB030A79
:10E5B0005C45C0F2CA80059BBBF1000FA8BF5B445D
:10E5C0000593069B002B00F08780059B3C469846F0
:10E5D0004FF0200A4FEAE379013C40F1E180059BCE
:10E5E000002FA8BFDB1939E009F10403D9F8007046
:10E5F0000C930D9B14F0010903F1FF3849D1059BE1
:10E6000014F4007F0CBF202430249A464FEAE37BA9
:10E61000B8F10108524623D5DDE90A01531C0593E0
:10E6200082424FEAE2738B4108DAAB68013B002B70
:10E63000AB6030DB2B685A1C2A601F70B9F1000FE9
:10E640004AD0059B44469A4620274FEAE37B013C8B
:10E6500026D5059BB8F1000FA8BF434405933BE0C6
:10E66000DDE90A2392457BEB030308DAAB68013B43
:10E67000002BAB6008DB2B685A1C2A601C701AF157
:10E68000010A4BF1000BC3E72946204601F002FCCA
:10E69000F5E7059AC0E72946384601F0FBFBCDE7D0
:10E6A000DDE90A2392457BEB030308DAAB68013B03
:10E6B000002BAB6008DB2B685A1C2A601F701AF114
:10E6C000010A4BF1000BC2E72946202001F0E2FBD2
:10E6D000F5E7013ECDF83090DDF83090059CB0466E
:10E6E00021E609F104030C936006D9F80030059A7D
:10E6F00004D51046D117C3E90001EDE7A10601D505
:10E700001A60E9E7E70501D51A70E5E72406F7D5B1
:10E710001A80E1E7DDE90A12884579EB020208DA9E
:10E72000AA68013A002AAA6008DB2A68511C2960FD
:10E73000137018F1010849F1000928E71846294625
:10E74000089301F0A7FB089BF3E7DDE90A23904556
:10E7500079EB03030BDAAB68013B002BAB600DDBFD
:10E760002B685A1C2A600AEB080212781A7018F1FA
:10E77000010804F1010449F1000919E70AEB080353
:10E780002946187801F086FBF1E700BF5624010006
:10E790009F2401005E240100492401004F24010050
:10E7A000DDE90A23904579EB030309DAAB68013B05
:10E7B000002BAB6009DB2B685A1C2A6083F800A091
:10E7C00018F1010849F1000906E72946202001F067
:10E7D00061FBF5E709F104030C93D9F800304FF021
:10E7E000000B9A465DE6E3057FF562AE0AF0FF0A8C
:10E7F0005CE661061AD509F1070929F0070909F154
:10E8000008030C93D9E900AB220618D51FFA8AFA3F
:10E810004FF0000B7E4B14F0080F7E4A18BF1A46CB
:10E82000E00601D524F400747B4B17E009F10403E2
:10E830000C93D9F800304FF0000B9A46E4E7E3055B
:10E84000E8D50AF0FF0AE3E74FF0000B09F10403F3
:10E850000C93D9F800306E4A9A466F4B0599DDE962
:10E860000A89B8EB010869EBE1790699CDE90889D5
:10E87000CDE910124FF0FF325521CDE912220022CE
:10E8800016A881540132202AFAD114F4826F04BFF1
:10E8900001221092672F00F3AA80652F08DA472F14
:10E8A00006D000F39A80412F02D0452F40F0A88077
:10E8B00013AB039312AB029310AB019311AB009314
:10E8C0003846234616AA14A92A9FB8470690BDE0E9
:10E8D000610615D509F1070929F0070909F10803AF
:10E8E0000C93D9E900AB220613D51FFA8AFA4FF030
:10E8F000000B484A494B14F0080F18BF1A4606E6A9
:10E9000009F104030C93D9F800304FF0000B9A463C
:10E91000E9E7E305EDD50AF0FF0AE8E7600616D55A
:10E9200009F1070929F0070909F108030C93D9E94E
:10E9300000AB210614D51FFA8AFA4FF0000B14F031
:10E94000100302D0002324F40074324A86E709F150
:10E9500004030C93D9F800304FF0000B9A46E8E717
:10E96000E205ECD50AF0FF0AE7E709F104030C938E
:10E97000D9F800309A464FEAE37BB6E5E1057FF52A
:10E98000BBAD4FFA8AFAB5E5A20704D414F0040F20
:10E99000204A234BB1E7234AB9E5E3065EBF0D23C6
:10E9A00044F01004069314F0100F069B08BF0623D2
:10E9B00009F1070929F00709069309F108030C93E7
:10E9C000D9E90023CDE91423002344F480644FF0F7
:10E9D000000A4FF0000B1A4640E7612F3FF468AF82
:10E9E000642F00F00981582F0AD100222AE0702FED
:10E9F000FBD008DC692F00F0FF806F2F00F09A80B9
:10EA00000023069322E0752F00F0F680782FEBE7C5
:10EA1000592401009F2401006F2401005C2401009F
:10EA200019240100172401000AF00F01595C16A8EF
:10EA300081544FEA1A1141EA0B714FEA1B108A46C2
:10EA4000834601325AEA0B010692EDD114F4806339
:10EA50000E9300F0D58000231093129B002BC4BFAF
:10EA600003F1FF331093139B002B03DD109A013B3E
:10EA700013441093069B109F11981F4401F085F8D2
:10EA80000D9B4FF00008DF1B04F001030D9340F2D3
:10EA900001231C42A7EB000700F0DB80C2464FEACF
:10EAA000E87B119B5A1C119293F80090B9F1000F6A
:10EAB00040F0D6800D9B83B914F4007F0CBF202357
:10EAC0003023C2463C464FEAE87B013C40F1E480FB
:10EAD00027EAE7737A1ED71A98440E9B002B00F0A2
:10EAE000F6803024069B4B4500F306810D9B5BB1FD
:10EAF000C2463C464FF020094FEAE87B013C40F11A
:10EB00009681002FA8BFB844059B4344A6E50AF0B0
:10EB10000702303216A9CA544FEADA0242EA4B72AF
:10EB20004FEADB0192468B4601335AEA0B02069309
:10EB3000EDD18BE70023F8E75FEA5B014FEA3A008B
:10EB40004FEA9A0242EA8B7210EB02084FEA9B03EB
:10EB500041EB03094FEA181242EA097218EB02006E
:10EB60004FEA191349EB030189464946020A42EA72
:10EB7000096280184FEA112349EB03014FEA10485C
:10EB800048EA014818EB00024FEA114949EB01033A
:10EB9000002112EB030843EB01094FEAD80848EAC9
:10EBA0004978A8FB0C014FEAD9090CFB09111AF1AD
:10EBB00006024BF10003121A63EB0103CDE90623B1
:10EBC000069B0AF1300A1809079B40EA037010EB14
:10EBD00008024FEA131141EB090302EB8201AAEB91
:10EBE000410A16A901F807A09B46924601375AEA46
:10EBF0000B030697A0D129E700274FF00A0CF6E790
:10EC0000069A109B9B1A0E9A48BF134631E7DDE91E
:10EC10000823904579EB030309DAAB68013B002B2D
:10EC2000AB6011DB2B685A1C2A6083F800B018F126
:10EC3000010849F10009AAEB0803002BE7DA27EAEB
:10EC4000E778AAEB080729E72946202001F022F9F6
:10EC5000EDE74FF0000907F1FF3A4FF0200BEAE72C
:10EC6000DDE9082392457BEB030308F1010809DA8B
:10EC7000AB68013B002BAB6009DB2B685A1C2A6098
:10EC800083F800901AF1010A4BF1000B09E72946BD
:10EC9000484601F0FFF8F5E7DDE908128A457BEB0D
:10ECA000020208DAAA68013A002AAA6008DB2A6888
:10ECB000511C296013701AF1010A4BF1000B04E793
:10ECC000184629460F9301F0E5F80F9BF3E7C2467B
:10ECD00030244FEAE87B109B013B002B10936DDA48
:10ECE000C246069C4FEAE87B002C00F38280069B1C
:10ECF000002BA8BF9844F9E616AB13F80900C246EA
:10ED00003C284FEAE87B31D03E2841D1139B013BA0
:10ED1000002B13932FDBDDE9082392457BEB0303E4
:10ED200008F1010808DAAB68013B002BAB602ADB75
:10ED30002B685A1C2A601C701AF1010A4BF1000B57
:10ED4000E4E7DDE9082392457BEB030308F10108C2
:10ED500008DAAB68013B002BAB600FDB2B685A1C59
:10ED60002A601C701AF1010A4BF1000B129B013B47
:10ED7000002B1293E5DA09F10109B3E629463020A8
:10ED800001F088F8EEE72946302001F083F8D3E758
:10ED9000DDE9082392457BEB030308F10108EADA79
:10EDA000AB68013B002BAB6004DB2B685A1C2A606C
:10EDB0001870E0E7294601F06DF8DCE7DDE908238B
:10EDC00092457BEB030308F1010808DAAB68013BCD
:10EDD000002BAB6008DB2B685A1C2A601C701AF1F0
:10EDE000010A4BF1000B76E72946302001F052F87A
:10EDF000F5E7DDE9082392457BEB03030CDAAB680A
:10EE000016AA013B2244002BAB6012F8010C0ADB6E
:10EE10002B685A1C2A6018701AF1010A04F1FF3499
:10EE20004BF1000B60E7294601F034F8F4E7DDE927
:10EE3000082392457BEB030309DAAB68013B002B07
:10EE4000AB6009DB2B685A1C2A6083F800901AF12A
:10EE5000010A4BF1000B51E62946202001F01AF877
:10EE6000F5E700BF0A4B034493F880309A0605D5B6
:10EE700030388842A8BF4FF0FF3070471A0701D5DD
:10EE80005738F6E7DB064CBF37384FF0FF30F0E776
:10EE9000A02401002DE9F84F804615460346894617
:10EEA00027491E4616F8010B80B30A1892F88020F5
:10EEB000D20724D4302829D158789E1C00F0DF02D4
:10EEC000582A1ED135F0100724D110259878DE1C61
:10EED0000024A246A3462946FFF7C4FF00281DDAF6
:10EEE0000FB106F1FF38C9F80080BBF1000F24D044
:10EEF00022224FF0FF30134B1A60BDE8F88F3346E3
:10EF0000CFE70127002DE3D10825E1E725B92F46FA
:10EF10000A25DDE70127DBE70027D9E704FB050425
:10EF2000230C0AFB053ABAF5803FA4B228BF4FF084
:10EF3000010B16F8010B0127CDE744EA0A40DCE794
:10EF4000A0240100A86100102DE9F74F0446914666
:10EF500098464FF0FF35DDF830A0654F00916168AD
:10EF60006A1C01390029616057DB2168481C206058
:10EF70000E78B91991F88010C8074CD4711C00F0B4
:10EF8000B280BAF1000F66DD19F0200F14D02B2EDD
:10EF900003D02D2E10D149F4007962680235013A70
:10EFA000002A626040DB2268511C21601678BAF1A9
:10EFB000010B52D02A46DA46302E4CD1616849F412
:10EFC0008077013900290AF1FF3B02F101056160F8
:10EFD0002FDB2168481C20600E78BBF1000F34D075
:10EFE00026F02001582930D138F010030FD1636882
:10EFF000AAF1020B013B002B02F1020563601FDB4B
:10F0000023685A1C22601E784F464FF010084FF0BC
:10F010000009AB4437E01546A1E72046019200F015
:10F020005DFE019A0646A4E7204600F057FE06461C
:10F03000BDE72046019200F051FE019A0646CCE75A
:10F04000204600F04BFE0646DEE7B8F1000F08BF91
:10F050004FF00808DBE71546D346B8F1000F4F46DE
:10F0600008BF4FF00A08D2E7636847F48077013B96
:10F07000002B09FB080905F1010563602BDB236800
:10F080005A1C22601E78ABEB0503002B05DD4146C0
:10F090003046FFF7E7FE0028E6DA2146304600F06A
:10F0A000F2FDFB0521D5FE0711D4009BBC061B68B1
:10F0B00007F0040203F1040103D5B80548BFC9F104
:10F0C0000009009801601B6852B1A3F8009028461F
:10F0D00003B0BDE8F08F204600F000FE0646D2E700
:10F0E000C3F80090F3E73546F1E76FF00105EEE76E
:10F0F000A0240100FFFFFFFF00232DE9F04F04468D
:10F100009BB0CDE902330F920D7801F1010B002D78
:10F1100000F08880252DDFF8A09347D009EB050289
:10F1200092F880206368D60703F1FF3325D55A464D
:10F1300012F8013B4B4493F88030D80713D463682E
:10F14000013B002B636014DB23685A1C2260187893
:10F1500009EB000393F88030D90706D4214600F06C
:10F1600092FD5946D0E79346E1E7029B01330293B3
:10F17000E5E7204600F0B2FDEAE7002B636009DB1B
:10F1800023685A1C22601E78AE4208D1029B0133CC
:10F190000293E6E7204600F0A1FD0646F4E730467C
:10F1A000214600F070FD01363CD171E14B7800271B
:10F1B0002A2B06BF01F1020B4FF0010A4FF0000AA3
:10F1C0005B460A20BB491BF8018B09EB080292F849
:10F1D000802092062AD41AF0080F08BF6FF000476B
:10F1E000B8F16C0F2DD19BF800804AF0020A03F1B0
:10F1F000020BB8F1670F00F3AB80B8F1650F80F236
:10F200005D81B8F1580F00F0CB832ADCB8F1450FCF
:10F2100000F05481B8F1470F00F05081B8F1250F8C
:10F2200000F0EF8003981BB0BDE8F08F8F42F9DC4F
:10F2300000FB0788B8F13007F4D44AF0080A5B46AF
:10F24000C1E7B8F14C0F04D19BF800804AF0120AD4
:10F25000CDE7B8F1680FCCD19BF800804AF0040AE2
:10F26000C5E7B8F1630F00F0E38000F31981B8F14E
:10F270005B0FD7D19BF8005000235E2D14BF0021F7
:10F2800001214FF00100CDE91233CDE91433CDE96E
:10F290001633CDE918330ABF9BF801500BF1010B6F
:10F2A0000BF1020B002DBDD06A111AAB03EB8202E9
:10F2B00005F01F0300FA03F552F8203C2B431BF81E
:10F2C000015B42F8203C5D2DECD149B1002312A92D
:10F2D00051F82320D24341F823200133082BF7D1E2
:10F2E0001AF0010609BF0F9B4FF000081A1D0F927C
:10F2F00008BFD3F800806368013B002B6360C0F255
:10F30000528323685A1C2260187800254FF0200988
:10F31000AF4214D0421C12D090FBF9F21AAB41421A
:10F3200003EB820201F01F0152F8202C00F01F03B2
:10F3300058BF4B4242FA03F3DB0700F13B832146FF
:10F3400000F0A1FC002E40F0A28288F800609EE24E
:10F35000B8F1700F00F003830CDCB8F16E0F00F011
:10F36000EF8200F3F982B8F1690F7FF45BAF009789
:10F37000002397E0B8F1750F00F00E83B8F1780F15
:10F3800000F00E83B8F1730F7FF44CAF4FF0FF35F0
:10F3900063680135013B002B6360C0F2E58223689E
:10F3A0005A1C2260187809EB000393F8806016F06D
:10F3B0000106EDD1411C6BD01AF0010808BF0F9B6C
:10F3C0002F4402BF1A1D0F921E68BD4208D0421C76
:10F3D00006D009EB000393F88030DB0740F1C882C8
:10F3E000214600F050FCB8F1000F01D186F80080F2
:10F3F0001AF0010F02BF039B01330393029B2B44BE
:10F40000C6E66368013B002B63600CDB23685A1C73
:10F4100022601D78252D3FF4B9AE2146284600F024
:10F4200032FC0135C0E6204600F058FC0546F1E705
:10F430001AF0080F08BF01271AF0010609BF0F9B39
:10F4400000251A1D0F9208BF1D68002F3FF4EAAE79
:10F45000029B1F44029B013302936368013B002B14
:10F46000636010DB23685A1C226018780EB928707C
:10F470000135029BBB42EDD1002E7FF472AE039B9F
:10F48000013303936DE6204600F028FC431CEDD1C8
:10F49000039B002B7FF4C6AE4FF0FF330393C1E60E
:10F4A0000A2300974AF020020FA92046FFF74CFDDF
:10F4B0000546ECE1CCCCCC0CA02401004FF0FF3889
:10F4C000636808F10105013B002B6360C0F2D28044
:10F4D00023685A1C2260187809EB000393F88030E7
:10F4E000DE0700F1C580411CD2D0002F00F0CC8097
:10F4F0002B2800F0C3802D2840F0C6804AF4007607
:10F50000636808F10205013B002B6360C0F2B8801C
:10F5100023685A1C22601878013FB3A3D3E9002363
:10F52000CDE9062300230022CDE908230023B846B5
:10F530001F460493B8F1000F40F0A880214600F068
:10F54000A2FBDDE908010A2303227B4393FBF2F3CC
:10F55000A7EB030842460E9300F0C4FDCDE90A0173
:10F56000049801F0D4FA424600F0BCFD002FCDE92A
:10F57000060180F252810FF27829D9E90089002230
:10F580009D4B4046494600F0D9FF02460B460020FD
:10F590009A4901F0F1F80022974B01F055F8CDE9B6
:10F5A00004017F4200220023CDE90823FA0738D561
:10F5B000DDE904234046494601F0B6F902460B4610
:10F5C000CDE90C01DDE90A0100F0B8FFDDE908230F
:10F5D000CDE90A01DDE90C0100F0B0FFDDE9062309
:10F5E000CDE90801DDE9040100F0A8FFDDE9082309
:10F5F00001F09AF9DDE90623CDE9080140464946C4
:10F6000000F09CFF00220B46CDE9062301F0B4F880
:10F61000DDE9082301F088F9012FCDE9080100F0A8
:10F62000038142464B464046494601F07DF9DDE9FB
:10F63000042301F079F902460B46DDE9040100F0EC
:10F640007DFF4246CDE904014B464046494600F065
:10F6500075FF4FF000080B464246894601F08CF8D2
:10F66000DDE9042301F060F97F10CDE904019DE795
:10F67000A84625E7204600F031FB2DE756463FE738
:10F68000204600F02BFB47E7564646E72E2811D1CF
:10F6900072060FD446F0400963680135013B002B28
:10F6A00063603ADB23685A1C2260187808F1FF383F
:10F6B0004E463FE7524B034493F880309B0630D5CB
:10F6C000049B46F480791A464E4B06F040069A4257
:10F6D000A0F1300007DC0A2303FB02030493002E91
:10F6E000DAD0013FD8E701F012FADDE9062300F095
:10F6F00025FF02460B46DDE9080101F015F900225D
:10F70000CDE90801DDE906013F4B00F09DFFCDE9A1
:10F710000601002EC0D10137BEE7204600F0DEFA18
:10F72000C4E720F02002452A06F480737FF406AF78
:10F73000002B3FF403AF636826F4C076013B002B37
:10F7400063601EDB23685A1C226018782B281ED0A9
:10F750002D281AD008F1FF3801354FF000090A2290
:10F76000274BA844A8EB0501002904DD191891F8DE
:10F77000801089061CD431064CBFA7EB09074F4403
:10F78000DCE6204600F0AAFAE0E746F0800663686F
:10F790000235013B002B636006DB23685A1C2260A4
:10F7A0001878A8F10208D8E7204600F097FAF8E7A1
:10F7B000616830380139002946F4807602FB090976
:10F7C00005F10105616004DB2168481C20600878B0
:10F7D000C8E720460A92069300F080FA0A9A069B30
:10F7E000C0E700BFAFF300809A9999999999B93F02
:10F7F000000000009999C93F000014400000F03F4C
:10F80000A02401009F86010000002440CDE90423CC
:10F810004FF00008DFF8D491C4E64FF000024FF03B
:10F820000003F3D1CDE90823DDE90823DDE90A016E
:10F8300001F07AF8DDE9062301F076F811AA00F06C
:10F8400026FC119F0E9B80463B44B3F5806F894692
:10F850001F4611931FDD2222604BD3E90078B305C8
:10F860005F4B48BF08F100481A60F3057FF5DAAC3A
:10F87000B00706F001092DD5B9F1000F07D10F9B94
:10F880001A1D0F9219683A464346C1E90023002D1C
:10F89000FFF6C7ADACE56FF47F739F420ADA002232
:10F8A000002301F03DF928B922224D4B07461A608A
:10F8B0008046DAE73A46B7054046494605D500F0A6
:10F8C00011FC074601F10048CFE700F00BFC0746AA
:10F8D0008846CAE712AA3846414600F0D8FB129B78
:10F8E0007E33002B129313DC00220023384641465E
:10F8F00001F016F9F8B922220020394B1A60B9F14B
:10F90000000FC4D10F9B1A1D0F921B681860BEE731
:10F91000FE2B10DD002200233846414601F06AF933
:10F92000304B314A002814BF1846104622222C4B77
:10F9300000681A60E3E73846414601F07BF8DEE7ED
:10F940000F9B1AF0040F03F104020F921B68029A36
:10F9500014BF1A801A6004E400970823A2E50097F8
:10F9600010232AF006029FE5204600F0B7F91AE5B9
:10F97000B8F1000F01D13070013663680135013BE9
:10F98000002B636004DB23685A1C226018781CE596
:10F99000204600F0A3F918E500970A23524683E5B4
:10F9A000009710237EE5204600F098F9411C7FF473
:10F9B000ACAC6DE51EB988F8000008F10108636879
:10F9C0000135013B002B636004DB23685A1C226075
:10F9D00018789DE4204600F081F999E48024010024
:10F9E000A8610010F4000010F000001000001440A6
:10F9F0000EB430B590B013AB53F8045B04463C2210
:10FA0000002101A80093FDF7C5FE09232046CDE99A
:10FA10000434019400F0B9F8009A0290294601A834
:10FA2000FFF76AFB10B0BDE8304003B07047FFFF3E
:10FA3000F7B507460E4601461A480D4615F8014B24
:10FA40001CB3031993F8803013F001031BD12B2C46
:10FA500002D02D2C1BD00D461C4601A92846FFF7CD
:10FA600019FA26B1019BAB4208BF3B4633608CB10B
:10FA70000028BDBF22224FF000400B4B4042B8BFD0
:10FA80001A6003B0F0BD2946D7E70D46E5E74FF40D
:10FA90000074E2E70028BFBF2222034B6FF0004052
:10FAA0001A60EEE7A0240100A861001038B5044CEC
:10FAB0000A2225680021FFF7BBFF256038BD00BF83
:10FAC000A861001070B5C468A5070CD0B2F5007F1E
:10FAD00005D0B2F5806F08D0B2F5807F03D1084D14
:10FAE0005E1EAE4204D9012008E0012300F124018A
:10FAF000144301610160C361C460002070BD00BF98
:10FB0000FEFFFF0040EA01039B0730B510D1054618
:10FB10000C4628462146036854F8042B04359A42C3
:10FB200006D1A2F1013323EA020313F0803FF0D0A3
:10FB300010F8013B11F8012B934201D0981A30BD07
:10FB4000002BF5D11846FAE740EA01039B0710B5F0
:10FB500013D10246043951F8043FA3F1013424EAD9
:10FB6000030414F0803F05D0D9B202F8011B59B14B
:10FB70001B12F9E742F8043BEDE7421E11F8013B86
:10FB800002F8013F002BF9D110BD10B5421C8307CC
:10FB900016D1034650F8041BA1F1013424EA0104F4
:10FBA00014F0803FF5D011F0FF0F11D011F47F4F0A
:10FBB0000CD011F47F0F14BF03460333981A04E0EE
:10FBC00010F8013B002BE2D1801A10BD0233F5E79B
:10FBD0000133F3E740EA01039B0770B512D10546F4
:10FBE0000E46032A314628460CD956F8044B0368C2
:10FBF00004359C4206D1A4F1013323EA040313F037
:10FC0000803F04D00A44914203D1002008E0043A26
:10FC1000E7E710F8013B11F8014BA34201D0181B94
:10FC200070BD002BEFD11846FAE740EA010370B52A
:10FC30009D0724D10E460346032A314608D956F8BB
:10FC4000045BA5F1013424EA050414F0803F0FD0D1
:10FC5000013A0139013B541C09D011F8014F9D1C98
:10FC6000561E03F8014F64B92A44954204D170BD71
:10FC700043F8045B043ADFE705F8014BF5E7034678
:10FC8000E6E73246E7E7431C15D0CB6813F40222BF
:10FC90000FD123F4012323F0400343F40123CB606D
:10FCA0008B6881F825008B634B68C1E901224B63A7
:10FCB00070474FF0FF30704738B50D46044608B91D
:10FCC000012A05D029462046BDE8384001F0F8B9A0
:10FCD000FBF764F92870204638BDFFFFF8B5C3680C
:10FCE00004461E0309D5426B23F400234260826B55
:10FCF000C360826090F82500F8BD9D0601D500F034
:10FD0000A9F846F2C902E3681A40012A0FD000227E
:10FD1000626044F24002134276D023F4A04323F001
:10FD2000400343F04003E3604FF0FF30E4E7474A0D
:10FD300013420CD14FF4807000F0ACFA4FF4807392
:10FD4000E361E368206143F400632060E36062687C
:10FD5000E368501C0DDA43F48053C2F1FF22E360E4
:10FD600002F57F022368FE3262605A1C2260187816
:10FD7000C2E7D906676904D5DA033ED5204600F00C
:10FD80005DF9E268E56942F48053E360D3032669D4
:10FD900021684CD5E36A99422CBFC6EB0106C6EB3D
:10FDA0000306AD1B33D1204600F048F9E569E6694A
:10FDB0002169761B0E44E3682A4623F01003E360B2
:10FDC00031463846FFF778FF0028BEBFE36820F0D1
:10FDD000004043F48043A5EB0005B8BFE36073190E
:10FDE000E362E3692363E36835BB23F4805343F0A4
:10FDF0004003E360C4E9006596E7A169384601F075
:10FE000064F90028BDDAE36843F080038BE7104B08
:10FE10001340002BCBD1A1693846314401F055F98C
:10FE20000028E368F0DB43F40033E360BFE7A36935
:10FE3000891B1944A161BEE7013D721C43F40033E4
:10FE400065602260E360307856E700BF000F010074
:10FE500010000200C36810B523F02003C36082695C
:10FE6000836A04469A420ED000F0E8F8E36823F46F
:10FE7000405323F0100343F01003E360A36AA3612F
:10FE80002369E3622360E36823F4804323F04003A3
:10FE9000E36010BDCB6870B523F400220C46CA6045
:10FEA0009906054602D52046FFF7D4FFD4E902366D
:10FEB0005A1C10DAB0050ED4C3F1FF2303F57F03FB
:10FEC000FE33A360236846F490365A1CE660226035
:10FED0001D70E8B270BD41F28A023240022A07D09A
:10FEE000002346F08006A360E6604FF0FF30F1E7A4
:10FEF0004AF210033340B3F5004F0AD100212046E7
:10FF000000F026FAE368990602D52046FFF7A2FF23
:10FF1000E66846F4903316F4706FE3600ED16069C2
:10FF200001F0CBF800B372051ED504F12403236160
:10FF300023600123E36146F49233E36013F4106F0E
:10FF40002168266926D0E36A99422CBFC6EB0101DD
:10FF5000C6EB0301B9B9731CE3622360E3695A1E5F
:10FF6000A26023633570B4E74FF4807000F092F91B
:10FF70004FF48073E268E36146F494331A432061DE
:10FF80002060E260DAE72246304600F0D1F800282F
:10FF9000E1D0AAE74A1CEDB222600D70E26A216846
:10FFA00091422CBFC6EB0101C6EB0201E2695B0581
:10FFB000226303D40A2D01D08A4209DC0023E662C1
:10FFC0002660A3602246304600F0B2F800288CD1AB
:10FFD00028467FE770B50D4606461046144600F0E9
:10FFE00069F92B78722B1AD0772B05D0612B23D18E
:10FFF000082348F2020201E00423022215F8011F3F
:020000021000EC
:100000002B290FD0622912D01B07E260666104D54C
:1000100002220021204600F09BF9204670BD0023FB
:100020000122EBE742F0030243F00203E6E742F06D
:10003000040243F00103E1E70024EEE738B504468B
:1000400005690168C36AC06820F40022E26000F01C
:100050008202022A02D04FF0FF3038BD10F4803007
:10006000FBD0994238BF19468D4208D10020E36881
:10007000E56223F480332560A060E360EDE722466B
:10008000491B284600F054F80028EFD0E3E7F8B504
:1000900016460023002204460D4600F041FD20B123
:1000A0000023002000213360F8BDC5F30A53204629
:1000B0002946A3F2FE327BB9C5F31303E70F03F41D
:1000C000002547EA4303C3F3130364000DB9013A63
:1000D000F4E7204663F3130140F2FE33326063F32A
:1000E0001E51E1E770B500231646002204460D4676
:1000F00000F016FD10B10020002170BD40F2FE732B
:10010000C5F30A5232449A422046294606DD22228D
:10011000054B1A60054BD3E90001EEE7002AEADD42
:1001200062F31E51E9E700BFA861001080240100BE
:100130002DE9F041D5688046EB020E46144657691A
:1001400005D5384600F0B6FF45F01005A061124B0A
:100150002B408BB1A169384600F0B7FF002806DAC2
:10016000E3684FF0FF3043F08003E36011E025F4D3
:10017000003525F01005E560324641463846FAF76D
:10018000F1FE20F00043F61AA3691E44A661002880
:10019000E6D1BDE8F08100BF10000200F8B5304F95
:1001A0003C68002851D10020F8BD2368B3F1805F7E
:1001B00039D1D4E9013151B10A68B2F1805F06D179
:1001C000DA1C4B681A448B686260A360F1E7AB42AB
:1001D00007DB9E4505DB20464FF0005340F80C3B03
:1001E000E2E7634511D920464FF00052656040F8C0
:1001F0000C2B00EB8502A2604FF080545B1B033B8D
:1002000040F82540C2E90131CEE761B9A0EB830097
:1002100000F04AF90130C6D04FF0005304F10C0051
:10022000C4E90035C0E72646A468002CBDD10C30D7
:1002300000F03AF9431CB6D04FF000538460C0E997
:10024000003556B938600C30AEE7C31C9D08002657
:1002500005F10A0C05F1030EE7E7B060F3E700BF14
:10026000B0610010A8B14FF0805340F80C3C50F83A
:10027000042C72B11368B3F1805F0AD150F8083CC6
:10028000516803330B4440F8083C936840F8043C41
:10029000EDE7704710B5FFF781FF044628B9172234
:1002A0000349FAF75FFE00F001FF204610BD00BFD2
:1002B00088240100F0B5C46889B0A107054622D0A2
:1002C000220718D4D0E9046700F020F8384600F07F
:1002D000EEFE230502D53046FFF7C4FFA40DA405AA
:1002E00014F1A54F07D12022296A684600F0F0FEDC
:1002F000684600F0CFF83C2200212846FDF74AFA74
:10030000002009B0F0BD4FF0FF30FAE7F7B5044622
:1003100098B103B0BDE8F04000F0E4B807FB04601A
:1003200000F0E0F8002818BF4FF0FF350134019BC2
:10033000A342F3DC284603B0F0BD034B05461B681F
:100340003C270193014EF2E720260100B461001022
:100350002DE9F843C6683D4B044633400D469046B0
:100360000BB9022747E0D0F81490484600F0A5FEEC
:1003700007460028F5D1B8F1010F2CD0B8F1020FD3
:100380002ED0B8F1000FECD1002DEADBB00404D57B
:100390002368E26A9A4238BFE362A169A9420EDC8F
:1003A0002368E26A934238BF134622695818801ABC
:1003B000A84204DB206B01EB000CAC4536DC0023CB
:1003C000C4E9013346F02006A56226F4032626F090
:1003D0004006E6600FE0204600F03AF80544D3E717
:1003E000484600F067FEB0F1000CE26806DA01272B
:1003F00042F08002E2603846BDE8F883E36A1846BE
:10040000A3691946236883422CBFC91809180B46F3
:1004100021699206A3EB010303D5A26A9342B8BFF8
:1004200013466345ACBFED186544ADE76D1AB107DF
:1004300044BF281AA060F10744BF9B1AEB1A154469
:1004400048BF6360256026F02006BEE70300100069
:10045000C3689A0705D121220D4B4FF0FF301A6077
:10046000704703F020021B0309D512B1806A0138DE
:1004700070470368826900691344181AF7E70AB1E4
:10048000806A70470368826900691344181A7047CC
:10049000A861001010B50446FFF777FB014620461F
:1004A000BDE8104000F00EBE70B50B4D2B680BB9C7
:1004B0000A4B2B60C41C2E6824F0030434442046ED
:1004C00000F030F810B92C60304670BD0C22044B9F
:1004D0004FF0FF361A60F7E7AC6100109863001028
:1004E000A8610010C36870B513F00306044611D06C
:1004F0009B0611D5856AFFF7ADFCE368204623F41F
:100500004053E360FFF79AFD002206462946204645
:10051000FFF71EFF304670BD836905681D440369FF
:10052000ED1AEAE7044B23B1984234BF00200120C2
:1005300070471846704700BF946B00102DE9F04FCC
:1005400081EA0306C1F30A5740F2FF7506F0004640
:10055000002F5AD0AF4258D0C3F30A54002C54D0C5
:10056000AC4252D04FEA525CC1F3130141F4801106
:100570004CEAC3234FEAC22843F0004CA1FB0823F6
:10058000A8FB0089924627444A461C4600230025C2
:10059000E0FB0C234FF0000B12EB0A008246ECFB51
:1005A000014543EB0B01601845F10001B1F5801FD7
:1005B0004AEA98021DD2041841EB01052946D30FDF
:1005C000A7F5806744EA03005200D30FC41841F135
:1005D0000005B2F1004F40F2FD72234608BF24F03F
:1005E0000103974208D818462E4306EB0751BDE891
:1005F000F08FA7F2FF37E8E7002F03DB46F0FF4656
:1006000046F4E00600203146F1E7490011F5001FED
:1006100012D25A0012F5001FF4D3094A5B0093422C
:100620000BD811424FF0000008D0134206D046F01C
:10063000FF4141F4E001DAE7EFD000200149D6E7BD
:100640000000E0FF0000F87F2DE9F043C1F30A57F6
:1006500040F2FF7E83EA0104002F58D0774556D040
:10066000C3F30A56002E52D0764550D09446BA1B9A
:10067000460D46EAC12141F000474FEA5C5141EA8C
:10068000C32343F00049C6024FEACC284F4508BFB8
:1006900046452CD202F2FD315FEA59094FEA38088B
:1006A000352200234F4508BF46454FEA430305D393
:1006B000B6EB080667EB090743F00103B6197F4163
:1006C000212A08BF1D46013AECD14F4508BF4645D7
:1006D00002D3013308BF013540F2FD70814204F0BE
:1006E00000420AD802EB0152511918460DE07F086A
:1006F0004FEA360602F2FE31CEE70029A4BF42F0EF
:10070000FF4242F4E00200201146BDE8F083184A9F
:100710004800904202D85D00954202D90020154958
:10072000F3E70B4312EA430301D11249DDE704F07A
:10073000004310EA020402D119462046E5E72A40A8
:1007400005D143F0FF4141F4E0011046DDE715F526
:10075000001F05D043F0FF41002041F4E001D4E741
:1007600010F5001F4FF00000D9D01946CDE700BFAB
:100770000000E0FF0000F87F944693EA0102F0B425
:1007800005460E4606D503F100452B46F0BC6246F1
:1007900000F0CAB88B4203D8844508D38B4206D1F7
:1007A00002F10042564053402A466546944640F2C4
:1007B000FF71370D27F400628A42A7EB135400F053
:1007C000A680944200F09F80C6F31302C3F3130384
:1007D0001F2C42F4801143F4801352D823FA04F200
:1007E000891A2CFA04F2C4F12004A34013439D4259
:1007F000A5EB03022CBF00230123154603B10139E9
:100800001CFA04F303D05B42551E02B9013911F4FE
:10081000C01F57D1EA0FDB0F42EA410243EA45030A
:1008200052EA030470D0BC1E510B24D0510C01BFFE
:10083000190F41EA02121B01043CD10C01BF990FB0
:1008400041EA82029B00023C110D02BFD90F41EA2E
:10085000420204F1FF344FEAD67108BF5B00B1EBEE
:10086000D42F4FF0000006BF184602EB045106F0EB
:100870000041F0BC7047190E41EA02221B02083CFD
:10088000D2E7352C1ED8203C23FA04F29542A5EB82
:1008900002002CBF00220122054602B10139C4F139
:1008A000200293402CFA04F45FEA0C6243EA04034A
:1008B00006D043F0FF035B42451E18B9013901E041
:1008C000002BF8D1CA0209D4013F7A050FD0EA0FF4
:1008D00042EA4101DA0F42EA45055B00002B21F4B0
:1008E00080124FEA075405DB11192846C1E7390584
:1008F0001046BEE7013508BF0132B3F1004F08BF13
:1009000025F00105F0E75CB921462046B1E7330345
:100910004FF0000001D00349ABE70CB90149F4E7FF
:100920003146E2E70000F87F93EA010FF0B4054694
:100930000E4605D503F100452B46F0BCFFF71CBF62
:100940008B4288BF1E4640F2FF7488BF0B464FEAB9
:10095000165184BF1546024621F40060A0425ED0C5
:10096000A1EB1354844255D0C6F31307C3F313030A
:100970001F2C47F4801743F4801327D823FA04F080
:10098000074422FA04F0C4F12004A3400343ED1805
:1009900028BF013702FA04F3BA022BD5013508BF8C
:1009A00001370BB925F00205360D360506EB570663
:1009B000730013F5001F35BF31460020FF074B1CA5
:1009C00034BF47EA55001905F0BC7047352CE3D811
:1009D000203C23FA04F02D18C4F1200003FA00F3A0
:1009E00022FA04F428BF01372343120618BF43F04C
:1009F000FF03D1E7002B01F1FF3207DA013508BF11
:100A00000137B3F1004F08BF25F0010507EB025194
:100A10002846D9E74CB906F000412046D4E7330315
:100A20004FF0000001D00249CEE73146F0E700BFA9
:100A30000000F87F21F0004230B502F1474505F58E
:100A40007005B5F17E6F01F000440FD202F148430A
:100A5000420FC10042EAC30202EBD173B1F1004F71
:100A600008BF23F0010343EA040030BD002D01DA82
:100A70002046FAE7490011F5001F94BF44F0FF40FB
:100A80000048F2E70000C07FCB0243EA505040F23A
:100A90001E43A3EB115340F00040FF2B20FA03F05C
:100AA00011D913F4E06F01D14042704711F080403A
:100AB00009D04B0013F5001F04D86FF0004000EB85
:100AC000D17070470020704720B903460246104697
:100AD00019467047030C0CBF000401F18071030E2E
:100AE0000CBF000201F50001030F0CBF000101F56E
:100AF0008001830F0CBF800001F500110028ACBFFE
:100B0000400001F5801101EBE0234205DFE700F032
:100B10000041002801F18041B8BF4042FFF7D4BF37
:100B200010B54C0054EA000C02D152EA430C09D033
:100B3000994209D1904207D114F5001F8CBF0020C3
:100B4000012010BD0120FCE70020FAE730B5054682
:100B500051EA03000BD4580010F5001F1ED899422B
:100B60001AD31BD195422CBF0020012030BD480074
:100B700010F5001F12D85C0014F5001F0ED8284392
:100B800002D154EA0200F1D0994205D806D195422B
:100B900094BF00200120E9E70120E7E70020E5E716
:100BA00030B551EA03040BD45C0014F5001F1FD8C4
:100BB00099421BD31CD190428CBF0020012030BD34
:100BC0004D0015F5001F13D85C0014F5001F0FD859
:100BD00099420BD801D1904208D255EA000307D1BF
:100BE00054EA02030CBF01200020E8E70120E6E7F9
:100BF0000020E4E730B551EA03054FEA41040AD486
:100C000014F5001F1ED899421AD81BD1904234BF48
:100C10000020012030BD14F5001F13D85D0015F52C
:100C2000001F0FD899420BD301D1904208D950EA46
:100C3000040307D155EA02030CBF01200020E9E7B5
:100C40000120E7E70020E5E7C0F3C75230B581EAAD
:100C500000039AB3FF2A31D0C1F3C75474B3FF2CF9
:100C60002CD022440902040241F0004144F0004427
:100C7000A4FB01452946002DA8BF690003F00040F0
:100C800040EA11234FEA0161B4BF7F3A803AB1F1E3
:100C9000004F03EBC25304D0FD2A02D803EBD170FE
:100CA00030BD01330CB923F00103FD2A01D81846E9
:100CB000F6E7002AF4DB40F0FF40F1E74000B0F136
:100CC0007F4F06D24A00B2F17F4F03D203F00040BB
:100CD000E6E70CD14900B1F17F4F08D810F07F4F03
:100CE00005D011F07F4F02D003F00040E3E7014848
:100CF000D6E700BF0000C07F30B5C0F3C75581EA1A
:100D00000003CDB3FF2D37D0C1F3C752A2B3FF2AE2
:100D100032D00402090244F0004441F000418C4208
:100D2000A5EB020532BF7D357E356408FD2D1CD84C
:100D3000090AB4FBF1F201FB1244D80F240202EBC2
:100D4000C030B4FBF1F201FB12442402B4FBF1F316
:100D500001FB134402EB002003EB002000EBC55025
:100D6000A1EB440100EBD17030BD002D03F0004039
:100D7000FADB40F0FF40F7E74200B2F17F4F13D8B3
:100D80004C00B4F17F4F0FD80843400010F07F4F64
:100D90000AD012F07F4F03F00040E5D0B4F17F4F4E
:100DA000E7D1B2F17F4FDFD10048DDE70000C07F1F
:100DB00091EA000230B4034604D530BC01F1004191
:100DC00000F066B8814284BF02F1004253404FEA0E
:100DD000D35488BF5140E2B2FF2AA4EBD1554DD085
:100DE000954247D009021A0241F0004142F0004208
:100DF00021FA05F0121A13D502F100428032E00503
:100E000000EB1223120608D1C5F1200011FA00F2FE
:100E10000CBF23F0010303F1FF33184630BC7047C9
:100E20005200002A18DADB0D8032DB0503EB2223A7
:100E3000120604F0FE0401D0002CEED1C5F1200012
:100E400011FA00F20CBF23F0010303F1FF33002C71
:100E5000E3D103F00043E0E716D0B2FA82F1A01E1E
:100E6000401AC00593EA000FF3D402FA01F300EB35
:100E70001323D2E7002D08BF2B46CEE75A0201D13B
:100E8000002DCAD1014BC8E70023C6E70000C07F90
:100E900091EA000F30B4024604D530BC01F10041A4
:100EA000FFF786BF81429CBF0B4601464FEAD150F7
:100EB00098BF1A46C3B2FF2B3BD0A0EBD2549C4242
:100EC00032D012020B0242F0004243F0004322FAF9
:100ED00004F55B190AD203F100438033C00500EB2F
:100EE00013211B0618D030BC08467047013003F5AB
:100EF0008073C50505EB5321DB05C0B201D0FF2887
:100F0000F1D1C4F1200412FA04F308BF21F0010169
:100F1000FF2808BF2946E6E7C4F1200412FA04F3CB
:100F2000E1D121F00101DEE7002CDCD101F000412C
:100F3000D9E74B0218BF0149D5E700BF0000C07FC9
:100F4000C20D010241F00041C2F19E039D2A10B57D
:100F5000044621FA03F003D9D2B29D2A01D84042B7
:100F600010BDFF2A02D1B1F1004FF9D16FF000435B
:100F700003EBD470F4E778B1B0FA80F200FA02F330
:100F8000C2F11F00803301EBC05000EB23201B0691
:100F900003D120F0010070470020704700F00041AD
:100FA000002801F18041B8BF4042FFF7E4BF4FF095
:100FB0008041FFF7E0BFFFFFC31013F07F610AD04D
:100FC000B1F17F6F4FEA407243F0E04308D003F184
:100FD00048411046704703F000430020194670470F
:100FE00052EA0332014A18BF1346F6E70000F87FC1
:100FF00050EA01034FEA400207D4B2F17F4F12D802
:10100000884294BF002001207047B2F17F4F0AD878
:101010004A00B2F17F4F06D8884204D213F1004053
:1010200018BF012070470020704740EA0103DB072A
:1010300003460CD40346043A22BF51F804CB43F8CC
:1010400004CBB2F10402F7D2043208BF7047013A70
:1010500024BF11F801CB03F801CBF8D870478B18E7
:10106000814238BF9842BFF4E0AF81418018013A15
:101070000B5C00F8013DFAD87047034613F0030FEC
:101080000ED101F0FF0141EA012141EA0141043A98
:1010900024BF43F8041BB2F10402F9D202F10402A6
:1010A000013A24BF03F8011BFAE77047FEE74FF04F
:1010B000FF3070474FF0FF3070474FF0FF30704700
:1010C000104670474FF0FF3070474FF0FF307047C9
:1010D0004FF0FF307047FFFF454D414300FFFFFFDA
:1010E000000000004E657442756653656D00FFFF99
:1010F000FFFFFFFFFFFF00000000000008060001E7
:1011000008000604000100000000000000000000CC
:10111000000000000000FFFF4E657445766E74000D
:1011200049502D7461736B00FFFFFFFFFFFFFFFF4E
:10113000000000000000000049444C4500FFFFFF94
:10114000546D725100FFFFFF546D7220537663009F
:101150006C1200100030000000C00720008000006A
:10116000000000000000000073656C6563740000FF
:101170000D0A546F6F206D616E792061637469761A
:101180006520636F6E6E656374696F6E732C206388
:101190006C6F73696E67210D0A0A00000D0A5275A3
:1011A0006E6E696E67206C6F77206F6E206D656D57
:1011B0006F72792C20636C6F73696E67210D0A431F
:1011C0006F6E736964657220636C6F73696E6720FC
:1011D000756E7573656420636F6E6E656374696F99
:1011E0006E732E0D0A0A0000FFFD22FFFA22010194
:1011F000FFF00D0A0A436F6E6E65637465642074B8
:101200006F202573200D0A25733E200062617474DF
:101210006572793E2000FFFF25733E2000FFFFFF2F
:10122000636F6E74726F6C007561727430000000D1
:1012300075617274330000006261747465727900C4
:10124000636F6D6D00000000736572636F6D6D00FC
:10125000332E312E3500FFFF73657474696E67207D
:10126000493243256420746F20706F6C6C696E671F
:10127000206D6F64650A00FF62617425643A206620
:1012800065740D0A00FFFFFF7475726E696E67204A
:101290006F666620737461636B206265636175734A
:1012A00065206F6E20636F756E74206973202564EE
:1012B0000A00FFFF232A242E48494C46450000001F
:1012C00020403939414620202E2E2E202054757280
:1012D0006E206F6666207061636B732C2064697387
:1012E00061626C6520616C6C2073776974636865FA
:1012F0007320200D0A00000020403939414320208E
:101300002E2E2E2020456E61626C6520636861720E
:101310006765207377697463680D0A002040393966
:10132000414420202E2E2E2020456E61626C6520C7
:101330006469736368617267652073776974636851
:10134000204120286D61696E290D0A00204039393D
:10135000424420202E2E2E2020456E61626C652096
:101360006469736368617267652073776974636821
:1013700020422028415558290D0A000020403939C3
:10138000424620202E2E2E202044697361626C6517
:101390002064697363686172676520737769746339
:1013A0006820422028415558290D0A00204039392B
:1013B000434420202E2E2E2020456E61626C652035
:1013C00064697363686172676520737769746368C1
:1013D0002043202841555832290D0A002040393930
:1013E000434620202E2E2E202044697361626C65B6
:1013F00020646973636861726765207377697463D9
:10140000682043202841555832290D0A0000000069
:1014100020403F3F504620202E2E2E202054757213
:101420006E206F6666207061636B203F3F2028301E
:10143000302D3534290D0A0020403F3F504E2020EA
:101440002E2E2E20205475726E206F6E20706163D8
:101450006B203F3F202830302D3534290D0A000005
:1014600020403939525120202E2E2E2020526571D5
:1014700075657374207374617475730D0A000000D0
:1014800020403F3F435620202E2E2E2020476574BB
:101490002063656C6C20766F6C7461676573206681
:1014A0006F72207061636B203F3F2028332E3441E0
:1014B00068207061636B73206F6E6C79290D0A0070
:1014C00020403939534820202E2E2E20205075746C
:1014D000207061636B7320696E746F20736875741C
:1014E000646F776E206D6F6465200D0A0000000048
:1014F0002057444F464620202E2E2E20204469732C
:1015000061626C65206368617267652077617463EE
:1015100068646F670D0A000020574441435420203F
:101520002E2E2E2020456E61626C652063686172EC
:101530006765207761746368646F670D0A00000057
:1015400020574452535420202E2E2E2020526573B3
:101550006574207761746368646F670D0A0000002A
:10156000426174746572792064617461206E6F7475
:10157000207265616479210A000000004039395306
:101580004800000043616E27742074616B6520621F
:101590006174746572792073656D6170686F7265CE
:1015A000210D0A005368757474696E672070616359
:1015B0006B7320646F776E202E2E2E0020646F6E6A
:1015C000650D0A005744525354000000436861728D
:1015D0006765207761746368646F672072657365FF
:1015E000742E0D0A0000000057444F4646000000CC
:1015F000436861726765207761746368646F672010
:1016000064697361626C65642E0D0A00574441433E
:1016100054000000436861726765207761746368F5
:10162000646F67206163746976617465642E0D0A66
:1016300000000000403939414300000053657474D4
:10164000696E672062617474657269657320746F76
:1016500020636861726765202E2E2E004039394163
:101660004400000053657474696E6720626174748D
:10167000657269657320746F206469736368617251
:101680006765202E2E2E00004039394244000000AC
:10169000456E61626C696E6720415558202E2E2E72
:1016A000000000004039394246000000446973617F
:1016B000626C696E6720415558202E2E2E00000066
:1016C0004039394344000000456E61626C696E67C1
:1016D0002041555832202E2E2E000000403939432B
:1016E0004600000044697361626C696E6720415571
:1016F0005832202E2E2E000040393941460000007D
:101700005475726E696E6720616C6C2062617474CE
:101710006572696573206F6666202E2E2E000000AC
:101720004025326450460000696E76616C69642021
:101730007061636B206E756D6265720D0A0000004A
:101740007475726E696E67206F6666207061636B78
:101750002025640A0000000040253264504E00003D
:101760007475726E696E67206F6E207061636B2096
:1017700025640A00403939525100000071756572C4
:1017800079696E672062617474657279207374611F
:10179000747573202E2E2E200D0A00004E6F2061CE
:1017A000636365737320746F20626174746572790A
:1017B00020737461747573210D0A00002530326442
:1017C0003A253034642C253034642C253035642C93
:1017D000253034642C253033642C253034580D0AE0
:1017E00000000000456E763A253364432C253364AF
:1017F000432C253364252552480D0A004D6561733D
:10180000313A253034642C253034642C253034644E
:101810002C253034642C253034640D0A000000007F
:101820004D656173323A2533642C2533642C25339E
:10183000642C2533642C2533640D0A005061636BDE
:10184000747970653A2032393C253032643E2C334D
:10185000343C253032643E0D0A0000004348473ACC
:101860002025642C2000000044495343483A202599
:10187000642C20004155583A2025642C200000009B
:10188000415558323A2025640D0A0000534D425507
:10189000536572723A256C752028256C7520756E1B
:1018A0007265636F76657261626C65290D0A00006E
:1018B00040253264435600007175657279696E6720
:1018C00020626174746572792063656C6C20766F38
:1018D0006C7461676573202E2E2E200D0A000000A7
:1018E000253032643A253034642C253034642C257C
:1018F0003034642C253034642C253034642C25306D
:1019000034642C253034642C253034640D0A0000F6
:1019100053544154530000006D696E20766F6C740F
:101920006167653A2020202025362E3266560D0A42
:101930006D617820766F6C746167653A2020202095
:1019400025362E3266560D0A61766720766F6C74E6
:101950006167653A2020202025362E3266560D0A12
:101960006176672063617061636974793A20202031
:1019700025362E326641680D0A746F74616C2063DF
:10198000757272656E743A202025362E3266410DCE
:101990000A746F74616C20706F7765723A20202032
:1019A00025372E3266570D0A0A616D6269656E74BD
:1019B0002074656D703A20202025362E31662A432A
:1019C0000D0A68756D69646974793A2020202020B9
:1019D000202025362E316625250D0A0068656C709D
:1019E000000000000D0A2020257320636F6D6D61DB
:1019F0006E64733A0D0A0A0062617564203C766178
:101A00006C75653E202020207365742062617564CA
:101A1000207261746520746F203C76616C75653E40
:101A2000206270730D0A00006D6F6465203C766162
:101A30006C75653E20202020736574206D6F646591
:101A40003A203C776F72646C656E3E3C70617269DF
:101A500074793E3C73746F70626974733E202865BC
:101A60002E672E20384E31290D0A00006272656102
:101A70006B202020202020202020202073656E64F1
:101A800020627265616B207369676E616C0D0A007C
:101A90006361636865203C76616C75653E2020203B
:101AA000736574206361636865206D6F6465203CB5
:101AB00076616C75653E2028303A2074696D6564E6
:101AC0002C20313A206E65776C696E65290D0A000D
:101AD0007374617475732020202020202020202022
:101AE00073686F7720554152542061707020737471
:101AF000617475730D0A000073746174757320202E
:101B0000202020202020202073686F7720626174BD
:101B10007465727920617070207374617475730DCF
:101B20000A0000006170702020202020202020204A
:101B30002020202073686F7720617070730D0A0079
:101B4000617070203C76616C75653E2020202020FD
:101B50006D616E61676520617070203C76616C75A7
:101B6000653E0D0A000000006970203C76616C75CE
:101B7000653E20202020202073657420495020617C
:101B80006464726573732028726571756972657318
:101B9000204D4355207265736574290D0A000000BD
:101BA0006E6D203C76616C75653E202020202020E3
:101BB000736574204950206E65746D61736B2028C5
:101BC0007265717569726573204D43552072657336
:101BD0006574290D0A0000006777203C76616C75FA
:101BE000653E202020202020736574206761746585
:101BF00077617920616464726573732028726571FE
:101C00007569726573204D4355207265736574293B
:101C10000D0A00006D6163203C76616C75653E20A5
:101C200020202020736574204D414320616464723C
:101C300065737320287265717569726573204D43F1
:101C400055207265736574290D0A00007374617400
:101C500075732020202020202020202073686F779B
:101C6000206E6574776F726B207374617475730D79
:101C70000A000000636C69656E74732020202020C8
:101C80002020202073686F7720636F6E6E65637409
:101C9000656420636C69656E74730D0A0000000052
:101CA00072657365742020202020202020202020B1
:101CB000726573657420746865204D43550D0A0084
:101CC00076657273696F6E202020202020202020EE
:101CD00073686F772076657273696F6E0D0A000006
:101CE000706F7274203C76616C75653E20202020F8
:101CF0007365742054435020706F72742028646997
:101D000073636F6E6E6563747320636C69656E7464
:101D100073290D0A000000006578697420202020D6
:101D200020202020202020206C65617665206D65B4
:101D30006E750D0A00000000617070004170702027
:101D40002874797065290D0A0A00000073657269AC
:101D5000616C00002020257320282573290D0A00BE
:101D60004170702027257327206973206E6F7420BF
:101D7000646566696E6564210D0A000072657365AD
:101D800074000000726573657474696E67204D435A
:101D900055202E2E2E0D0A00636C69656E7473003B
:101DA00025752E25752E25752E25750028796F75BC
:101DB00029000000282573290000000020205B2551
:101DC000645D2025732025730D0A0000706F727406
:101DD00000000000417267756D656E742072657158
:101DE0007569726564210D0A00000000496E766114
:101DF0006C696420706F72742027257327210D0A87
:101E000000000000436F6E74696E75696E6720751F
:101E100073696E67206F6C6420706F727420272561
:101E200064270D0A00000000506F7274202725649B
:101E30002720697320616C72656164792074616B1D
:101E4000656E2062792027257327210D0A00000086
:101E500053657474696E6720706F727420746F209C
:101E600025642C20636C69656E74732077696C6CD3
:101E700020626520646973636F6E6E656374656468
:101E80002E0D0A00697000004E6F7420612076618B
:101E90006C69642049502061646472657373210D1C
:101EA0000A0000004E657720495020616464726525
:101EB0007373202725732720616374697665206119
:101EC00066746572207265736574210D0A000000E6
:101ED000677700004E65772047572049502061649E
:101EE0006472657373202725732720616374697694
:101EF00065206166746572207265736574210D0AD0
:101F0000000000006E6D00004E6F7420612076614D
:101F10006C6964206E65746D61736B210D0A00003D
:101F20004E6577206E65746D61736B20272573276E
:101F300020616374697665206166746572207265DC
:101F4000736574210D0A00006D6163004E6F74208B
:101F5000612076616C6964204D4143206164647244
:101F6000657373210D0A28666F726D61743A20588B
:101F7000583A58583A58583A58583A58583A585877
:101F8000290D0A004E6577204D414320616464723B
:101F90006573732069732061637469766520616677
:101FA000746572207265736574210D0A000000006B
:101FB0007374617475730000506F72743A2020203E
:101FC000202020202025640D0A00000049502061B7
:101FD0006464726573733A2020257320000000004A
:101FE000282573290D0A00006E65746D61736B3AC4
:101FF00020202020202573200000000067617465E8
:102000007761793A202020202025732000000000ED
:102010004D414320616464726573733A2025303208
:10202000783A253032783A253032783A253032788D
:102030003A253032783A253032782000282530325F
:10204000783A253032783A253032783A253032786D
:102050003A253032783A25303278290D0A000000CE
:1020600076657273696F6E004261744D616E3A20DD
:102070002020202025730D0A00000000424F4C4F05
:1020800000000000426F6F746C6F616465723A20EB
:1020900025730D0A00000000426F6F746C6F61645D
:1020A00065723A206E2F610D0A0000006272656150
:1020B0006B00000073656E64696E67206272656113
:1020C0006B202E2E2E0D0A00626175640000000048
:1020D000496E76616C696420626175642072617416
:1020E00065202725732721204D6F7374206265209A
:1020F0006120706F73697469766520696E746567B5
:1021000065722E0D0A0A000053657474696E6720AB
:1021100062617564207261746520746F2025642E7D
:102120000D0A0A006D6F6465000000005365747449
:10213000696E67206D6F646520746F202563256369
:1021400025632E0D0A0A00006361636865000000C4
:10215000496E76616C6964206361636865206D6FA8
:102160006465202725732721204D6F7374206265D5
:102170002030206F7220312E0D0A0A0053657474CE
:10218000696E67206361636865206D6F64652074A4
:102190006F2025632E0D0A0A000000000D0A506F03
:1021A00072743A2020202020202020202020256426
:1021B0000D0A0000554152542073657474696E67AE
:1021C000733A2020256C752025730D0A000000004D
:1021D0004361636865206D6F64653A20202020208C
:1021E00074696D65640D0A004361636865206D6FF5
:1021F00064653A20202020206E65776C696E650D3D
:102200000A000000545820746F74616C2062797465
:1022100065733A20256C6C750D0A000052582074C5
:102220006F74616C2062797465733A20256C6C75EB
:102230000D0A00005258206C6F7374206279746527
:10224000733A2020256C75200D0A0A000D0A506F84
:1022500072743A2020202020202020202020256475
:102260000D0A0A0065786974000000007361792026
:10227000776861743F0D0A00496E76616C6964206D
:10228000626175642072617465210D0A20206163AA
:102290006365707461626C652076616C7565733A14
:1022A000203131353230302C2035373630302C204B
:1022B00033383430302C2031393230302C20313426
:1022C0003430302C20393630302C20343830302C1B
:1022D00020323430302C20313230302C2036303027
:1022E0002C203330302C203131300D0A000000001A
:1022F000496E76616C6964206D6F64652076616CEF
:102300007565210D0A20206578616D706C653A2035
:10231000384E310D0A000000496E76616C69642008
:10232000776F7264206C656E677468210D0A2020D7
:1023300061636365707461626C652076616C75655C
:10234000733A20352C20362C20372C20380D0A00EB
:10235000496E76616C696420706172697479210DCF
:102360000A202061636365707461626C6520766128
:102370006C7565733A206E2C20652C206F0D0A0059
:10238000496E76616C696420616D6F756E74206F43
:10239000662073746F702062697473210D0A616323
:1023A0006365707461626C652076616C7565733A03
:1023B00020312C20320D0A00001BB70000800000E5
:1023C0001009000018090000B0080000B80900005A
:1023D000C80B0000D00B0000010900000909000033
:1023E00021090000410900004909000051090000CD
:1023F00071090000790900008109000089090000C5
:10240000D90900000406080A0E141C24282C3034B4
:10241000383C40FF07131A2B0020003078256370EA
:102420002564003058256350256400307825632EDC
:10243000252E2A6C6C7870256400305825632E2573
:102440002E2A6C6C58502564002D007200770028ED
:102450006E756C6C290030580030780030003031D7
:1024600032333435363738394142434445460030FB
:10247000313233343536373839616263646566002A
:10248000FFFFFFFFFFFFEF7F2A2A2A205F437379B8
:10249000735F616C6C6F63206661696C65640A00D0
:1024A000000000000000000000000000000000002C
:1024B000000000000000000000000000000000001C
:1024C000000000000000000000000000000000000C
:1024D00000000000000000000000000000000000FC
:1024E00000000000000000000000000000000000EC
:1024F00000000000000000000000000000000000DC
:1025000000000000000000000000000000000000CB
:1025100000000000000000000000000000000000BB
:1025200040404040404040404041414141414040A6
:10253000404040404040404040404040404040409B
:102540000502020202020202020202020202020268
:10255000202020202020202020200202020202022F
:102560000290909090909010101010101010101079
:1025700010101010101010101010100202020202A1
:1025800002888888888888080808080808080808D1
:10259000080808080808080808080802020202409B
:1025A000000000000000000000000000000000002B
:1025B000000000000000000000000000000000001B
:1025C000000000000000000000000000000000000B
:1025D00000000000000000000000000000000000FB
:1025E00000000000000000000000000000000000EB
:1025F00000000000000000000000000000000000DB
:1026000000000000000000000000000000000000CA
:1026100000000000000000000000000000000000BA
:0426200008000000AE
:10262400AAAAAAAA000000000000080045000000B1
:1026340000000000801100000000000031302E3046
:102644002E302E31000000000000000031302E300A
:102654002E302E3200000000000000003235352EEE
:102664003235352E3235352E30000000000C6A012B
:1026740003100101FFFFFFFF0000001000C0014034
:102684000700000051C50000000000000000000029
:10269400000000000000000000C00540130000001E
:1026A40051C5000000000000000000000000000010
:1026B4000000000000000A401A00000051C500009C
:1026C4000000000000000000000000000000000006
:0826D400000080FF0000807F80
:040000030000214B8D
:00000001FF
